:100000000030012001520200696F0200696F020096
:10001000696F0200696F0200696F0200696F020078
:10002000696F0200696F0200696F0200696F020068
:0C003000696F0200696F0200A9F6000071
:10003C002DE9F04F99B0054680780224532800F240
:10004C00CF85DFE810F054009900A800B800C80074
:10005C00DA00EA000C011B01CD052A013801590117
:10006C00CD05CD05CD05CD05CD05CD05CD05CD05F4
:10007C00CD05CD05CD05CD05CD05CD05CD05CD05E4
:10008C00CD05CD05CD0565018A019601A201AD0115
:10009C00BC01D601ED0109023C02CD05CD05CD0513
:1000AC00CD05CD05CD05620278028E02A402BA02FE
:1000BC00CF02E0020503CD05CD05CD05CD05CD055F
:1000CC00CD053A034E036203CD056F037903970305
:1000DC00A003AC03B803C703D103F4031104360423
:1000EC003E0450045D0469048D0494049704EC1CD4
:1000FC00E97A2A7B002320461EF0F2F88DF81800CE
:10010C0006AB65200021012222F038FBDFF8280B1A
:10011C000078012800F26385204629F019FE00289A
:10012C0000F05D8505460079012840F0588529F0DE
:10013C0093FB00274FF400018DF83F008DF8380039
:10014C00000ACDF83A108DF841708DF83E708DF89C
:10015C0040008DF839000EAE214606F10A0029F058
:10016C0078FE2978152233460170697887704170C2
:10017C004520FF2100F031BD29F01DFE6979AA79D7
:10018C000023002425F09AFB8DF838000EAB652077
:10019C00012100F05ABC29F095FB29F017FD01460E
:1001AC000EA8022229F0A7FD8DF8180006AB6520D9
:1001BC00022100F04ABC29F085FB29F007FD01461D
:1001CC000EA8032229F097FD8DF8180006AB6520C8
:1001DC00032100F03ABC29F075FB29F0F7FCEA7911
:1001EC0001460EA80023002427F0C2F98DF8180050
:1001FC0006AB6520042100F028BC29F063FB29F034
:10020C00E5FC01460EA8052229F075FD8DF81800B5
:10021C0006AB6520052100F018BC0020DFF8404A31
:10022C0029F037FAADF85800681DA0478046E81D44
:10023C00A04795F809A0814605F10A07BAF1100FFD
:10024C0000F2B2830EAC5546002D00F0B083384658
:10025C0029F050FE24F8020B013D0237F4E729F097
:10026C0031FB29F0B3FC01460EA8102229F043FD06
:10027C008DF8180006AB65200721E6E329F022FB78
:10028C0029F0A4FC01460EA8112229F034FD8DF8AA
:10029C00180006AB65200821D7E329F08CFD6A7B9A
:1002AC00691D0023002423F071FF8DF838000EAB7C
:1002BC0065200A21C9E302208DF8200029F07BFD7E
:1002CC00ADF81800681D29F015FEEA79064605F10F
:1002DC0008018DF838200EAF781C29F0B1F806A86B
:1002EC0031463A460023002420F02EFC8DF85800AD
:1002FC0016AB65200B21A8E329F05DFD002100243D
:10030C0023F04AF98DF838000EAB65200C219CE3E4
:10031C000020DFF84C4929F0BCF9ADF85800681DF5
:10032C00A047814695F80FA005F11000A04795F85D
:10033C0012B0074605F11304BBF10F0F00F249830D
:10034C000EAE5D46002D00F04783204629F0D2FD0D
:10035C0026F8020B013D0234F4E729F0B3FA29F038
:10036C009FF929F05DF840F04B8306A829F071FD48
:10037C004BE329F0A7FA29F093F929F051F840F052
:10038C00528306A829F065FD52E329F014FD29F0EB
:10039C00FAFB8DF838000EAB6520232100F01CBC55
:1003AC00DFF89418C8208DF81800E81C097800298B
:1003BC0000F0878328F0D3FC8DF81800A9E3687946
:1003CC00EE1CFE280BD1A879FF2808D12878082824
:1003DC0005D3304629F08EFD314625F097FC0EA949
:1003EC00304628F099F9002800F097830546002440
:1003FC00A5E3E81C042126F0BBF9E97929F09CFD62
:10040C00DFF850188DF83800022028F0DDFDDFF8F9
:10041C004818032028F0D8FD0EAB65202621DBE31D
:10042C0029F0C3FC044605F10E0029F063FD297C7C
:10043C006A7C0346E878CDE90012AA1D214625F016
:10044C00C1FEDFF80C188DF83800042028F0BCFD34
:10045C000EAB65202721BFE34FF00208E81C8DF896
:10046C00408029F047FDADF8380068798DF85800C8
:10047C00A81D29F03FFD2E7A044600270935CDE949
:10048C00005716A80EA92246334621F04BF929F045
:10049C0043FA10D1DFF89C078DF84080CDE9005766
:1004AC0022463346C08AADF8380016A80EA921F0B2
:1004BC0039F98DF8180006AB652028218CE302264B
:1004CC00E81C8DF8406029F015FD29F07FFBED79D3
:1004DC0004460EA8002321462A4627F0BFFF29F028
:1004EC001BFA0ED1DFF84C078DF8406021462A46E6
:1004FC000023C08AADF838000EA827F0AFFF8DF8A6
:10050C00180006AB6520292166E329F0DBF9ADF86C
:10051C003800681D042126F02BF96A7AAB7A002486
:10052C00014600940EA825F079FE8DF8180006AB54
:10053C006520302189E229F0C5F929F029FB312207
:10054C0001238DF8580016A8CDE90004DFF8FC064D
:10055C000EA921F0E7F88DF8180006AB65203121C3
:10056C0073E229F0AFF929F013FB322201238DF845
:10057C00580016A8CDE90004DFF8D0060EA921F02A
:10058C00D1F88DF8180006AB652032215DE229F018
:10059C0099F929F0FDFA332201238DF8580016A899
:1005AC00CDE90004DFF8A4060EA921F0BBF88DF804
:1005BC00180006AB6520332147E229F083F9ADF82A
:1005CC003800687B0024691D0094C0F3400200F0E1
:1005DC0001030EA822F0C2FF8DF8180006AB6520AF
:1005EC00342132E229F06EF96A7BADF83800691DCE
:1005FC000EA80023002426F05DFB8DF8180006AB36
:10060C006520352121E22C4614F8030B04281ABF6F
:10061C00E8782C1D02208DF84000204629F06AFC59
:10062C00DFF82466A5780121E278ADF838000023C4
:10063C00002431700EA829461EF0C4FE8DF8180057
:10064C002846347026F072FB06AB65203621FCE19F
:10065C0029F0B1FBADF83800687904218DF8400021
:10066C00A81D26F085F80446AE7AEF7A05F10C0049
:10067C0029F040FCDFF8BC850546214632463B4656
:10068C0029F015F80EA821F029F829F045F910D118
:10069C000220214632463B468DF84000B8F8160041
:1006AC00ADF8380029F003F80EA821F017F88DF8F2
:1006BC00180006AB652037218EE26C7829F07BFBA5
:1006CC000146DFF88005007820F018FA8DF8380024
:1006DC0004F0E000202840F082820EAB65203E2121
:1006EC007AE26C7829F067FB0146DFF85805007850
:1006FC0021F000FD8DF8380004F0E000202840F0D7
:10070C006E820EAB65203F2166E200206C788DF87E
:10071C003800DFF824050078411E022980F0998109
:10072C0002209AE129F047FB29F02DFA8DF83800C8
:10073C000EAB652042214FE2002006908DF83D0063
:10074C00CDF83900E81C06A926F024FF8DF83800F6
:10075C00069850B128F081FF81788DF83B10C17854
:10076C008DF83C1000798DF83D000EAB65204321CF
:10077C00062232E2E81C28F0F2FA8DF838000EABB3
:10078C006520442128E229F016FB6979AA790EF03C
:10079C00D7F88DF838000EAB652045211CE229F006
:1007AC000AFB6979AA791AF0A1FC8DF838000EAB16
:1007BC006520462110E2EC7829F0F7FA0146204634
:1007CC0022F0DCF9B0FA80F0472140098DF83800AE
:1007DC000EABC7E1E87800248DF8384023F046FDD5
:1007EC000EAB6520472130E1E8780EA926F0F6FE25
:1007FC0006468DF8180040000130C5B2284629F095
:10080C007DFB002800F0A981044600F8016B002153
:10081C009DF81820914280F0C0809DF8383001314D
:10082C0000F8023B9DF8393000F8013CF2E70EACC1
:10083C001321204629F06CFAEE7829F0B6FA01461D
:10084C00304626F09BFA002800F08E810021231DF3
:10085C008DF8381028F001FFC11C827818468DF8ED
:10086C003B2028F0EDFD82E10020EC78CDF846002D
:10087C00CDF84200CDF83E00CDF83A0029F095FABB
:10088C00AA79ADF838000F2A28BF0F228DF83A202C
:10089C0022B10EA8E91D033028F0D2FD0EA9204686
:1008AC0001221DF0BDF88DF8180006AB65204B2118
:1008BC0092E128F00DF98DF838000EAB65204C2133
:1008CC008AE1E87829798DF838100EA9032800F010
:1008DC006581022800F06881012840F06C8152206B
:1008EC0021F04CFC6AE129F066FA69790246A81DF0
:1008FC001BF013FB8DF838000EAB65204E216BE11D
:10090C0029F059FA0146687919F0A8FF8DF83800DA
:10091C000EAB65204F215FE1C64D0822E88A05F138
:10092C003901ADF83800C54800788DF83A00A88C2C
:10093C00ADF83B00688BADF83D000EACE01D28F027
:10094C007FFD04F10F0005F11C01082228F078FD51
:10095C00287E5021182223468DF84F0065203CE15B
:10096C00B5480078002800F00781122010E120F033
:10097C0053F834E100208DF83800E87841B2B1F139
:10098C00FF3F06DC10F07F00AA4918BF012081F858
:10099C0068000EAB652053211EE1652049212A46D3
:1009AC00234621F0EBFE3DE180208DF8630097F8A3
:1009BC0000B0BBF1100F53D87E1C4FEA4B0500243E
:1009CC0006AFA5424ED0301929F094FA38530234B0
:1009DC00F7E780208DF8630026780F2E58D80597FE
:1009EC00671C75004FF0000806AC454552D007EB6C
:1009FC00080029F07FFA24F8080008F10208F4E74F
:100A0C00084629F077FAADF81800687E06A928F098
:100A1C000FFD0EA921201BF0D1FB8DF8580016AB51
:100A2C006520212111E0084629F064FAADF8180080
:100A3C00687E06A928F0FCFC0EA922201BF0BEFB48
:100A4C008DF8580016AB65202221012221F096FE6C
:100A5C00C6E0002840F0B680042009F001F8B4E0AC
:100A6C0080200EE0BAF1100F0DD80EA900204A46D6
:100A7C005346CDE9001BCDE9027016A8414615F08E
:100A8C0031FA8DF863000DF1630365200621A3E0B4
:100A9C0080200FE0BBF10F0F0ED80EA90020CDE97E
:100AAC0002645246CDE900B1049016A8059B494654
:100ABC0015F0C0F98DF863000DF16303652020215A
:100ACC008AE016A90EAD2A4618F03CFE04469DF8A5
:100ADC005800F0B1614904EB4400002641F8206055
:100AEC0001EB800046609DF94B00B0F1FF3F03DC49
:100AFC0005F1130023F03AF80EAD1421284629F025
:100B0C0007F90420214614222B4625F097FD8DF879
:100B1C00186006AB652024215EE0182029F0EEF960
:100B2C00002800F083800446BDF83800002118220C
:100B3C00234628F01BFB0546002818BFC8251920A2
:100B4C0029F0DCF9002867D007460130002D4BD086
:100B5C001821FF2229F086F850E0002049218DF859
:100B6C00180006AB652037E001208DF838000EAB7D
:100B7C0065204A21132230E029F01DF9044605F1C5
:100B8C000D0029F0B7F90246691D204625F05CFBE3
:100B9C008DF838000EAB652051211DE0522021F05C
:100BAC00EDFA2748002104E0522021F0E7FA24480E
:100BBC000121017002E0522025F09EFB0EAB652056
:100BCC004D2109E001208DF8380004F0E0002028C8
:100BDC0005D10EAB65204021012221F0CFFD002470
:100BEC00204619B0BDE8F08F3146082228F028FCC9
:100BFC0007F109002146102228F022FC652025214E
:100C0C0019223B463D7021F0B9FD3846192129F0D7
:100C1C007FF8384629F070F9002CE0D020461821D6
:100C2C0029F076F8204629F067F9D8E7C825FFF7B0
:100C3C00DEBB00BFA86D002024260020D02600209B
:100C4C00E52700209A7A0020A5270020882600207E
:100C5C00B96A02007F70020019500100F0330020C5
:100C6C00019F02002DE9F04F99B080466FF007000C
:100C7C00DFF8DCA80630ADF852009AF80000022824
:100C8C0014D1DFF8C808007880B9B8F8080010B1A2
:100C9C001020012101E0302000210AF0E5FD0020A8
:100CAC008DF81C0007A9522021F068FA0DF11C09DF
:100CBC0098F80810D8F804004A4610F089FAE8B100
:100CCC009DF81E609DF81F409DF82050BDF82670C1
:100CDC0028F0BCFD844211D127F003004FF6F871C7
:100CEC0080B288420AD0012D08D8022E06D29AF87A
:100CFC000000022808D19DF84D0028B1D32019F02E
:100D0C0076FC19B0BDE8F08FB8F82800ADF84800B3
:100D1C00B8F83200ADF82A009DF82200D0B1D8F80E
:100D2C0004109DF81D209DF83830012027F034FB6D
:100D3C0008B1CF20E3E7DFF81C08C078012809D1FF
:100D4C00B8F8280028F0A7FF20B1417901F0E7019D
:100D5C00083141719DF8210068B1BDF82610FF20C3
:100D6C0026F00CF89DF82110E0B141F001012C2681
:100D7C008DF8211017E09DF83900002800F0EB8069
:100D8C009DF83D10FF2902D0002940F02681DFF8A4
:100D9C00C807BDF82620C18A8A4240F0278101206D
:100DAC00222607E0082601F00300012808BF46F0C0
:100DBC00110601209AF800104FF6F877012908D88F
:100DCC00B207344658BF64F07F04002808BF34468D
:100DDC0000E034469DF82200DFF87C575FFA84FB74
:100DEC0030B9E87A20B10BF02200222840F0808044
:100DFC001BF0400004901CD0012903D8A87B80076D
:100E0C0000F1D880119801780C2900F2DB800122C6
:100E1C0041F298438A401A4200F0D480032902D14F
:100E2C0040780D2805D007A822F0F4F901283FF4EA
:100E3C0068AFA88CB8F8441081420AD198F84620C3
:100E4C00B8F84210B8F8280000230093002307F0EC
:100E5C0001FE9DF82200F8B1B8F84210B8F828004D
:100E6C0022F0E4FC002800F08F800646D8F804003D
:100E7C009DF81D10F2780844417B8A421EBF002267
:100E8C007260F1700130042125F072FC71688842A7
:100E9C00FFF437AF013070609AF80000022834D2AA
:100EAC00A87B80077FF52DAF9DF84D004FF6F876A7
:100EBC0060B1BDF8280027F0BBFC002800F00781CA
:100ECC00D8F80400417801F0DF0141709DF82E0044
:100EDC00002800F0DF80D8F8040081790139817195
:100EEC008DF82E1004F07F00090640F0D680D3E078
:100EFC000BF0420042287FF41CAF1198007800F0F0
:100F0C00FE0006287FF415AF72E77FF4FAAE95F871
:100F1C002600092802D004287FF4F3AE5FEA8B6028
:100F2C0000F19E80049800283FF4EBAE11989DF8D8
:100F3C0038100078042808BF022900F045810728E2
:100F4C0008BF042900F009810C2840F04D8107A846
:100F5C0015F080FBD5E6BDF8260022F0E7FE02383E
:100F6C00DFF8F415B0FA80F0CA8A4109BDF8260002
:100F7C00904208BF023100293FD09DF81E20002A64
:100F8C0056D001F1400455E09DF84D00B8B3042053
:100F9C0026F0CEF900283FF4B4AE01464FF4B270FF
:100FAC000880B8F828004880DFF8B00500781EF0FB
:100FBC00D5F8A6E611980178A1F10C0212F10C0FEC
:100FCC003FF62CAFE88ABDF8262082427FF496AE1D
:100FDC00BDF8280024F0AAFA90E6109A9DF83C007F
:100FEC0020F0DEFF30B101200026E3E690F8260069
:100FFC000428F8D100260020DCE600241AE095F83D
:10100C006C0001287FF448AF11980078062803D1B2
:10101C00049800287FF440AFF81DBDF82A1080B268
:10102C0081423FF46EAE07A841461EF02BFB68E6EA
:10103C0001F1200422F07AFE0138B0FA80F0400968
:10104C0044EA00069DF81E0000283FF4B2AE119849
:10105C00007827F041FC012818BF04F07E06A8E6B2
:10106C0098F8460028F0D6FA9DF82E00012840F09A
:10107C00B480B8F82800BDF82810814240F0AD804B
:10108C00BDF8260022F052FE022804BF00208DF885
:10109C002E00A2E004F07F000446210702D44FF09A
:1010AC00000A34E0E1B24A0722D4C9069DF82110A7
:1010BC0028D5C1F3820212B1072A18BF013A002ABF
:1010CC0008BF044601F0E30040EA820118E0D32097
:1010DC0019F08DFADFF888040078002800F09F8062
:1010EC00DFF8801451F82000C0EB0010810098E06C
:1010FC009DF8210000F0E00100F0E30040EAD1018E
:10110C008DF82110D8F804004FF4805A017295F82C
:10111C002600092801D0042823D1E98ABDF826002D
:10112C0088420AD022F002FE022806D09DF8210047
:10113C0000F0030001287FF4E4AD9DF81E000028A8
:10114C0047D011989DF838100078042808BF022960
:10115C003AD0072848D1042946D107A817F0C2FF76
:10116C00CFE5E7B214F0610F46D0F80709D0B8F814
:10117C00281007A8A94615F0B5FC002864D004F087
:10118C009F040025E7B2A00609D598F84600D8F8C8
:10119C003C2028F03FFA07A815A905F06BFC78064F
:1011AC0040F12681B8F8281007A80DF152022B4601
:1011BC0010F08AF800286FD00546119800780128A5
:1011CC0008BF4AF0100A13E107A9002010F024FE12
:1011DC0097E598F8460028F01DFAD8F83C2007A8A7
:1011EC0015A905F047FC8CE503287FF48AAD07A808
:1011FC0000210FF079FC84E59DF81E0001285AD1DE
:10120C0011980078032849D0052854D1B8F8281033
:10121C0007A80DF15202002310F056F871E5D148E1
:10122C000168D1480268BDF82800904701287FF476
:10123C0068ADCE480168BDF828008847CC480168E5
:10124C00BDF8280088475CE526F034FC9DF82E108C
:10125C000546BDF8280019B9B8F82810884291D075
:10126C00B9F81610814204D1BA48807800283FF4AE
:10127C0089AFB8F8281007A82A460AF0B9F8002850
:10128C0000F09B8038074AF0040ABDF8260048BFDE
:10129C00F01DADF8520075E70025A9E0BDF8260059
:1012AC0027F0C6FA38B1B8F8281007A80DF1520289
:1012BC00002310F009F89DF82E0088B323F0CAFE25
:1012CC0000287FF41EAD9DF83900A0B3109A9DF84C
:1012DC003C009DF83D1020F063FE002870D09DF876
:1012EC003D00002875D0109928F098FC9DF824300A
:1012FC00ADF8520011209DF823209DF821104AF0E2
:10130C00400A002B08BF0920002A18BF083000290A
:10131C0018BF0130D8F804100A5C013A0A5462E094
:10132C009DF81E0001287FF47EAE119800780328EA
:10133C003FF4E7AC77E69DF82010BDF826000029B5
:10134C00ADF8520000F0D3804020BDF8261009F112
:10135C001D0200EAC4059DF820002B4618F048FE3B
:10136C0038B1D8F804004AF0200A017801F03F01A6
:10137C0001709DF8390048B1BDF8261009F1200024
:10138C0021F02AFF4AF0400AADF852009DF81E00E9
:10139C00012806D0BDF82810BDF82600002214F054
:1013AC00ABFFBDF82810BDF826002A4612F0D2FB80
:1013BC00002818BF4AF0200A15E004F0DF04E0E62C
:1013CC00BDF82610BDF828000B2200231AF033FDBF
:1013DC0097E4BDF82600ADF8520028F05CFC00281C
:1013EC0008BF4AF0400A26F065FB05464FF6F87632
:1013FC00B01DBDF8521080B20F1A5E4818BF2F46B0
:10140C000078012805D1F01DB8F8321080B2814265
:10141C002FD160B2B0F1FF3F3FF773AC002F3FF418
:10142C0070ACB8F8080028F069FD00283FF469ACEE
:10143C00B8F80820D8F80410054628F001F89DF8F3
:10144C001E10002098F80830B8F8282016908DF857
:10145C005410BDF8521015ACCDE9007ACDE9020458
:10146C00284610F065FC70B3284628F045FDFFF7C0
:10147C0048BCB8F828108142CBD0701CBDF826208F
:10148C0080B28242C5D2BDF828008142C1D028F07A
:10149C0002FC0028BDD0017901390129B9D8408856
:1014AC0001218DF85410ADF8600015AD28461EF0E2
:1014BC0059FD0028ADD0281D1DF048FD0028A8D0EE
:1014CC0021F0D4FFA5E72348407800283FF419AC5D
:1014DC0000208DF81870ADF81900DDF826004FEAE1
:1014EC003040059005A827F037FEFFF70ABC3907F6
:1014FC003FF52AAF9DF81E1001293FF425AF0021BE
:10150C0018F036FD20B1407901380228FFF41CAFE9
:10151C00B8F84410BDF8520022F088F930B1807848
:10152C0026F0F8FC01380728FFF40EAFBDF82800B0
:10153C0027F07EF918B104208DF8200004E7BDF8DF
:10154C002610BDF8280002223FE700BFE527002047
:10155C0024260020E8250020A86D00209C7A00207D
:10156C00D727002090B40200942300209C23002055
:10157C0098230020E32700202DE9F0438DB0054689
:10158C0080780224252800F27380DFE810F0260012
:10159C00A400C400D700EA00F8000601B602B602A7
:1015AC001D012E01B602B602B602B602B602460103
:1015BC004B01B602B602540158016101B602B602E3
:1015CC00B602B602B602B602B602B602B6026B019B
:1015DC006E017101740178017F01DFF8D47500246C
:1015EC000E258DF804403878012807D801A81DF085
:1015FC0073F904469DF8040005EB4005EEB2304645
:10160C0028F07CFC002800F087824FF0000805468B
:10161C00431C0021082280F80080012027F0A6FD41
:10162C0028F01AF96872000A0721A872DFF88405FD
:10163C00E972007828733878012800F262829DF8EC
:10164C000420002A6A7300F05E8205F10E0000216E
:10165C002346914280F0578213F8022B013100F897
:10166C00022B13F8012C00F8012C9DF80420F0E754
:10167C00A0F140010D291FD8DFE811F00E00100178
:10168C003F023F021E012E013F023F023A0145017B
:10169C00500165013F02740101ACE91C0822201DB8
:1016AC0027F0CEFE204619F0EDFFBDF806004021D4
:1016BC00ADF828000AABEEE0632800F069816428DD
:1016CC0000F07681E02840F0188200244720E021C9
:1016DC00002200230FE2202028F010FC002800F04C
:1016EC00C1812021FF22044628F0BCFA631C012092
:1016FC000021082227F03AFD0546002818BF0125D5
:10170C0001AB84200021042227F030FD002800F0DA
:10171C000582023506E2E81C28F0ECFBADF804006B
:10172C00832028F001FB014601AA832028F0C6F98A
:10173C008DF828000AAB6720022190E1E81C0421F7
:10174C0025F016F80190842028F0EEFA014601AA43
:10175C00842028F0B3F98DF828000AAB6720032108
:10176C007DE1612028F0E0FA0146EA1C612028F0B6
:10177C00A5F98DF8040001AB672004216FE162200C
:10178C0028F0D2FA0146EA1C622028F097F98DF86D
:10179C00040001AB6720052161E100208DF80400F5
:1017AC00E81C28F0A7FB6A7900F4F851002A00F035
:1017BC004981B1F5A06F04D04FF6FF71884240F01B
:1017CC004B814FF0FF3045E128F06AFB044628F0CE
:1017DC0065FBD949604301ACB0FBF1F1204628F020
:1017EC00F6FA672009210422ABE0DFF8B4632D7907
:1017FC00306840B901AC204627F0F0FE01202146AC
:10180C000EF03AFB3060052D00F06981002D00F0E0
:10181C006981642122F01AFA66E115F8032B67201E
:10182C0010216EE0E87823F011FF8DF8040001AB75
:10183C006720112113E100246720142102E0002409
:10184C0067201521ADF80840019401AB062252E146
:10185C0000246720162109228DF80C40CDE90144A3
:10186C0001AB48E1F52020210BE0F520212108E017
:10187C00F520222105E04FF6F570232108E0F52034
:10188C0024218DF8040001AB6720E8E0F520252128
:10189C00ADF8040001AB67200222E1E0E81C28F05F
:1018AC0029FBADF8060001AC204617F0D7FB231D31
:1018BC00672041210822D3E0E81C0AA926F02CFF5E
:1018CC0000288DF8040000F0CF8001A81821FF2219
:1018DC00013028F0C7F9F4E0E81C0AA926F01CFF37
:1018EC0000288DF8040000F0F1804FF0FF30EFE09D
:1018FC0015F8030F697822F071F9288067204821C8
:10190C0002222B46ACE0E87825F080F801AC0146C9
:10191C00204618F06DFD6720492111E0EC1C204693
:10192C0026F0C6FB002818BF2046B5F80B1019F09E
:10193C0039FA01AC0146204618F05AFD67204A21BD
:10194C00242223468CE001ACE91C0822204627F017
:10195C0077FD204627F04CFB8DF828000AAB67205A
:10196C004B217CE04FF0FF3095F80380691D01900E
:10197C00ADF81000CDE90200FE208DF806002879A4
:10198C0003288DF8300020D10AA828F062FA21E053
:10199C000024E91C08228DF8284001AD284627F0C8
:1019AC004FFD28461DF0D2FA0AAB67206321A1E057
:1019BC00B5F80B006A7B0024E91C8DF804400AF092
:1019CC0085F901AB6720642194E0084628F092FA6F
:1019DC00ADF82800AF7B002F00F0DD807E0095F87D
:1019EC000D90304628F08AFA002800F0D48005F1DA
:1019FC000F013246044627F023FD00940AA9404605
:101A0C004A463B460DF07EFA002800F0BA808378F7
:101A1C0001784278057946798DF806308DF80410F6
:101A2C008DF80520C3788DF809608DF808508DF875
:101A3C00073001A98B1D811D40794200184627F003
:101A4C00FFFCA5E0B1F5A06F03D04FF6FF71884203
:101A5C0002D100205549086001AB67200621012204
:101A6C0020F08CFE002448E0182028F047FA40B300
:101A7C00BDF828100446009006200022182324F0FC
:101A8C00C7FDB8B9BDF8285001AE21461022701C14
:101A9C0027F0D6FC444F05EB450506F1110057F82D
:101AAC00251028F094F907EB8500416806F1150024
:101ABC0028F08DF92046182128F02AF9204628F024
:101ACC001BFA01AB672044211922C9E7BDF8280095
:101ADC00ADF8050001AB672045210322C0E7314971
:101AEC0001220A7021F049FA002467200A218DF89E
:101AFC00044001AB012220F041FE20460DB0BDE8B0
:101B0C00F08385F80D806720002132462B4620F0AB
:101B1C0035FE284628F0F0F97CBBA3E7019800BA03
:101B2C00C4F809000AAB83200021022227F01EFB17
:101B3C0020B1043506E000BF40420F00BDF828007C
:101B4C00A4F80D0004F10F0361200021012227F0FD
:101B5C000DFB002804F1100318BF0835622000218A
:101B6C00102227F003FB0028234618BF10356720EE
:101B7C0001212022257020F001FE204628F0BCF91E
:101B8C0070E74FF6FF70ADF808006FF480300190ED
:101B9C00204628F0B1F901AB67204D210E225FE7FA
:101BAC00287A0020A227002030750020087A002017
:101BBC0024260020D02600202DE9F04F85B0847813
:101BCC000226362C00F2BF820546DFE814F06B01CA
:101BDC00730172007B017800BC02BC0281003700EB
:101BEC004C008C009F00AD00BC02B5008F01BC0204
:101BFC00BC029901AC01BA01BC02BC02BC02BC0221
:101C0C00BC02BC02BC0237004C00BC02BC02BC02D1
:101C1C00BC02BC02BC02BC02BC02BC02BC02BC02C8
:101C2C00BC02BC02BC02BC02BC02BC02BC02BD00B9
:101C3C00EB00CA01FF005B005B00DA0128F0AFF893
:101C4C00242840F0A98102AB352000210422002475
:101C5C0027F08CFA002800F0FB81012002228DF87D
:101C6C0010000020FBE100208DF8100028F097F800
:101C7C000646092C40F0EC8095F8059095F8068006
:101C8C000720EEE0DFF82465306880B1406A70B15F
:101C9C0002A928F08DF80546342C40F02A822846FB
:101CAC0028F028F9002800F02382042042E20320C7
:101CBC0040E2DFF80835612002210A2240E202AC42
:101CCC00E220214624F018FB61200421082287E140
:101CDC0028F065F80446681D28F00CF9242C40F017
:101CEC0086810020F9E1E878032800F29681281D0E
:101CFC0028F000F90246E878DFF8B81431F8101033
:101D0C00DFF8B404007828F05FF887E1E87803285E
:101D1C0000F28881DFF89C1431F81010DFF8980479
:101D2C0000781DF059FE7EE127F06EFFADF808003B
:101D3C0002AB61200C2102E1002661200E21012260
:101D4C008DF8086002AB1CE2DFF8606401208DF8AE
:101D5C0010003068002800F02B810069002800F08A
:101D6C00278102A928F024F8042124F001FD002881
:101D7C0000F0ED81044628F0C1F8002800F01B812A
:101D8C002146054627F0C4FF3068BDF80C102246EA
:101D9C002B4606690298B0478DF81000284628F0AB
:101DAC00ABF808E1DFF804442068002800F0078154
:101DBC008069002800F0038102A927F0F9FF206850
:101DCC00BDF80C10826902989047F9E0DFF8DC73DB
:101DDC003868002800F0FA80C069002800F0F6800E
:101DEC0002A927F0E5FF9DF80850BDF80AB0BDF830
:101DFC000C90044628F07EF8A6788046F72E28BF73
:101E0C00F726B01C5FFA80FA504628F077F80028C5
:101E1C0000F09F81012D044608BFBBF1000F00F0BC
:101E2C009C813868A11C42463346C56902980091D2
:101E3C004946A8470746002840F0958100276120B5
:101E4C003321524623466670277020F097FC8AE1B6
:101E5C00681D28F04FF88146E81D28F04BF88046A5
:101E6C00092002AF242E18BF2F1809EB080508BF54
:101E7C003526304627F058FF854201D9022059E11A
:101E8C00B9F1000F04D1304641463A4623F098F997
:101E9C00304641463A4627F011FE002800F0E58016
:101EAC000A2047E1E878012802D0002840F04A8156
:101EBC0027F02EFB40F259600121ADF8080002AB6F
:101ECC0061203CE00120EC1C8DF80800E22021464A
:101EDC0020F054F930B901200821224627F0EEFDFC
:101EEC008DF8080002AB6120032128E1E878291D58
:101EFC00012800F0E080002840F0E480E020DEE0E3
:101F0C0027F04DFF0446681D27F0F4FF242C0FBF6B
:101F1C0000200146204627F0AFFE8DF8080002ABEA
:101F2C00612012210BE127F03AFF24280CBF00207E
:101F3C0027F0FAFEADF8080002AB61201321022253
:101F4C00FEE0E8788DF8080099488068D0F83024D5
:101F5C0002A9E02090478DF8100004AB61201421F9
:101F6C00EDE0924C206898B3806A88B302A927F000
:101F7C001FFF2068BDF80C10826A0298904701463A
:101F8C0027E08A4C206868B3C06858B327F007FF75
:101F9C002168C968884726E083466938002680B2E4
:101FAC00032838BF0126681D082C40D1057841E074
:101FBC0003208DF8100004AB61203021BFE003201A
:101FCC008DF8100004AB61203121B8E00327CFE07D
:101FDC00002102AC204627F0FAFE612032210422B7
:101FEC002346ADE0032027F0ECFD3621A7E005F1F8
:101FFC000806ED790146A8426BD92046002227F04D
:10200C0057FD09288DF8080069D1002D67D02046AE
:10201C002946324627F052FD61E0022027F0D1FD1F
:10202C000A218CE0022027F0CCFD0B2187E027F061
:10203C0061FF0546584627F077FE0227A84288BF65
:10204C007700CFB100268DF808706120214694E00E
:10205C0002988DF810400422ADF8120002208DF881
:10206C00110004AB612008216AE0012E64D1E2204A
:10207C00394620F083F85DE0401B87B2F72F28BF6C
:10208C00F727B81C5FFA80F8404627F037FF002886
:10209C0061D000F1020A81463946504627F038FEDD
:1020AC00584629463A46534627F060F8054600281C
:1020BC006AD00A2773E00878022814D2522020F044
:1020CC005DF800E002208DF8080002AB61200F21C2
:1020DC0035E02046324627F0EBFC8DF8080002ABC9
:1020EC00612007212BE002A9522024F005F9ECE72E
:1020FC0002359DF8080015F8018B012811D1BDF8A7
:10210C000A0070B9BDF80C7041462A46384623F0D7
:10211C0057F8012F07D1E220294620F02FF801278C
:10212C0001E0BDF80C703068394642462B46466AD1
:10213C000298B0478DF8100004AB612021460122B3
:10214C0020F01CFB0026304605B0BDE8F08F0520C2
:10215C002FE710270CE0102774E7A9F1690003287A
:10216C00BFF45FAE0227204627F0C6FE002FE9D051
:10217C0000268DF80870612033218DF8096002ABC0
:10218C00022220F0FBFADEE789F8017000276120BB
:10219C00214642464B4689F8007020F0EFFA48463B
:1021AC0027F0AAFE002D7FF44DAFCBE76827002067
:1021BC000C01002054BA02009A7A0020F0B90200F7
:1021CC002DE9F04F9DB00446DFF89C05406818B12E
:1021DC008047002800F05682DFF890A5DFF890B514
:1021EC000D940DF138099AF80000411E002C0B914A
:1021FC000BF1180418BF01219BF802800027002561
:10220C008BF80F109BF801100C91C0B287421ED2B4
:10221C00B84517D0FEB200214A460423304627F0B9
:10222C00D7F80E9810F4403F40F00400C0B218BF2D
:10223C0001357C2806D130460621F82226F03CF8E0
:10224C00F82020709AF800000C340137DDE7E9B271
:10225C0001380024884204D19BF80500002800F0C6
:10226C007F82DDF83490CDF82880DFF8FC84B9F15A
:10227C00000F484608BF1020059015AD00200190B6
:10228C00DDE90B740026380400F0FE819BF80F008A
:10229C0010B901208BF80F00E0B200210EAA042324
:1022AC0027F096F80E98B9F1000F19D010F4403FB2
:1022BC0019D04FF400509AF800100136013FABF8DA
:1022CC0010009BF80F0001388BF80F00012050FA1A
:1022DC0084F0B0FBF1F202FB11048BF80D40D2E755
:1022EC000021049102E0CDE90B740496C0B20A9E61
:1022FC004FF0000A702804D00C987021C0B222F064
:10230C001BFB5FFA86F900210EAA0423484627F02E
:10231C005FF89DF83800FE2803D04846FE2122F0D5
:10232C000BFB48460621FE2225F0C6FF4FF4005059
:10233C000C9F0BF11601ABF814A000228BF80C606B
:10234C00ABF81000FF2088F800208BF80E00F8B2D4
:10235C008BF80D70400050FA87F001EB8000B0F85C
:10236C0006A04FEA490050FA86F09BF80F6001EB8B
:10237C008002FE20ABF812A0114601F8020F32F8D1
:10238C00060F03910890DFF8E4030292047814A876
:10239C0021F090FD56FA87F0CDF82490013890FB8F
:1023AC00F4F101FB140000905FFA87FB0C97CB450E
:1023BC0000F06281ABEB0900B0FA80F040090790A5
:1023CC00002006900020DDF83490C00740F09E807D
:1023DC001FFA8AF4162C6ED998F80000002840F0E9
:1023EC007381AAF1070758460FAAB9B218F0C0F8C2
:1023FC00BDF84A6006F11000A0423BD89DF846009B
:10240C00962837D1A7EB06099DF8452031465B4647
:10241C001FFA89F840461BF043FE58BB9DF8470055
:10242C00C10701D1800704D40020CA46DFF83883E5
:10243C00C9E7F01D83B2089813FA80F4B4F5005F75
:10244C0001D90120F2E780B2CC4918440A1A584647
:10245C00414626F0BDFF06980130B4F5005F0690AA
:10246C0004D101204FF400510891DEE70020CA4648
:10247C000894DBE7AAF1010ADFF8EC825446A0B21B
:10248C00172836D33628A4F1160658462A4688BF94
:10249C002026A41BB3B2A1B226F09AFF3004EED0D2
:1024AC0015FA86F010F8010C962801D0013EF5E7DC
:1024BC0006EB040A86E7069810B1AD4927F0DBF865
:1024CC000098C0B2834500F0DB800C990120DDF848
:1024DC00249050FA81F0A5490978B0FBF1F202FB87
:1024EC001107A34907EB470001EB8000B0F81CA0D3
:1024FC005AE7A0481499006842689F48904700200A
:10250C0007900C980A90DDF8349008E0069810B10A
:10251C00974927F0B0F8002007900C980A9098F88B
:10252C000000002840F0D08008981021C0F500521F
:10253C00103883B20998C1F2001221F0D7FC98F838
:10254C0000100843149988F800008A480068426813
:10255C008948904707980A9A88B1844800780BEB11
:10256C000001013991FBF0F202FB10128049D0B24C
:10257C00400050FA82F001EB8000B0F81CA0DFF8AC
:10258C00F0B108990298099C01238BF80E20018068
:10259C00ABF81010BBF912209BF80D102046ABF8CD
:1025AC0014A023F05FFDBBF914209BF80E102046FD
:1025BC00022323F057FDBBF81000049CB9F1000F67
:1025CC00C0F5005007D00599DFF8A0A18842A4BF40
:1025DC000121019101E0DFF894A1059988424FF0A7
:1025EC007C01B8BF7821099E304622F0A5F90DF088
:1025FC00E3FE07469BF80F000621FC22C01B8BF85C
:10260C000F00304625F058FE0399FC209BF80E3045
:10261C0008709BF8021017FA84F00C9301449AF896
:10262C000000B1FBF0F202FB10118BF802100A91C2
:10263C000131CAB2B2FBF0F202FB10118BF801109F
:10264C0003EB43010BEB8101898B102906D10C990B
:10265C000131B1FBF0F202FB10100C900B98C01B77
:10266C00B9F1000F0B903FF40BAE019880F0010014
:10267C00C0077FF405AE07E00120CB46079042E788
:10268C0000984BE700246BE07C2022F06FF90446A5
:10269C00FF284ED17E2022F069F90446FF2848D14C
:1026AC009BF8014004EB44000BEB8000807DFF287D
:1026BC003BD09AF800009BF802100144013991FBC1
:1026CC00F0F202FB101434E02A48149900684268B6
:1026DC0029489047264E254F00253878854213D23D
:1026EC00ECB2204615F0CEF898F80010084388F8A4
:1026FC0000003DB138780138854203D020467E2158
:10270C0022F01AF90135E8E7B18B01380024B070DA
:10271C00C0B2F4707470F180FE2122F00DF900202B
:10272C007C2122F009F974711AE020467E2122F0F6
:10273C0003F9E0B2FE218BF80340400050FA84F01C
:10274C000BEB8000808BABF806009BF8020022F0AC
:10275C00F3F800208BF80500BBF81000C0F500540E
:10276C0020B21DB0BDE8F08FA02300209B7A002082
:10277C00B8720020D8010010004003400020001166
:10278C002DE9F04F8FB00C4648070FD4200441D4EC
:10279C00E00400F19781200600F1C081A00700F150
:1027AC00D481200500F1F3810020B4E1DFF820058D
:1027BC000178062900F2AD81DFE811F007009401E1
:1027CC00AB01AB019901AB01A001DFF81055DFF8AB
:1027DC0004152A7891F82B30022A02D19E0600F1BA
:1027EC0098815E0700F19D819B0740F19281042343
:1027FC00037091F82C30DB0700F08B8191F82E30B0
:10280C00002B00F0528225F09EFC0420012101F0E7
:10281C00EFFF57E2DFF8C8040394DFF8BCB4DFF82D
:10282C00B094DFF8C474DFF8AC44DFF8B054DFF8D0
:10283C00BCA448F20208008802909BF800001CF02F
:10284C0031F9002800F03A8106460078D3282DD1C2
:10285C00F089404540F019813878002800F0158146
:10286C0099F80000012840F0108126F031FD002875
:10287C0040F00B817088002840F00781A24604AC20
:10288C001221204627F044FA27F016F8304621464C
:10289C0018F096F9BDF81C00B0F5285FC0F08880E0
:1028AC00012002211FF016F854462AE099F8001076
:1028BC00884217D1012834D0032840F0E6802878CC
:1028CC000138012800F2E180B078012851D00028AD
:1028DC0040F0DB807078002800F0BF8000201DF0F5
:1028EC0059FCD2E00A2811D194F82B00BA46B71C37
:1028FC003071A16909B138468847384625F0AAF8E5
:10290C005746DFF8D853DFF8E4A3BEE02978002956
:10291C0040F0BB80092840F0B880A168B01C884703
:10292C00B3E028780138012800F2AF80707860B1EC
:10293C0094F8330094F83410013084F83300C0B2AA
:10294C00884202D9012000219DE099F8010003285A
:10295C0058D0022871D0012840F097803878002890
:10296C0000F08C8026F0B4FC002800F0928001204E
:10297C0085E07078002875D026F06EFF4FF6FE715A
:10298C00884203D1BAF81600884207D0AAF816106C
:10299C00ADF8281053200AA91FF0F0FB1EF00EFB17
:1029AC0025F0B8F800208AF826001DF03BF96CE001
:1029BC00CF48006809A90AAA16F0C4FE0746029877
:1029CC005446C64DDFF824A3874212D29DF8380036
:1029DC0010B1FD208DF838000420394614220AABC2
:1029EC0023F02CFEC34907EB470001EB80000121CB
:1029FC0041720020012184F83200012001F0F8FE20
:102A0C00B94F42E0A2460AACAB20002122461CF092
:102A1C0071FA042004945446DFF8D0A2AF4D8DF81F
:102A2C00140004A80FF054FB26F046FF9BF800009E
:102A3C004FF4805141F288321DE0012020714FF497
:102A4C008060ADF828000AA818F0E2FD26F034FFEB
:102A5C00A4484FF4805102680BE010F0F9F860695B
:102A6C0098B9A2E702204FF4805140F6B83289F8A9
:102A7C0002009BF8000027F0A7F906E0002084F87C
:102A8C0032000120012101F0B3FE304625F02EFB6F
:102A9C00D3E694F8350020B1E0690028F5D08047E2
:102AAC00F3E70020002102220023ADF828000220C9
:102ABC008DF830000AA825F0D1FCB5E7039880F416
:102ACC00004028E0854800780138012859D8804812
:102ADC00017803294DD0012953D1417800201EF0F3
:102AEC00F9FE4EE0012001211EF0F4FE11E025F06C
:102AFC002AFB0420012101F07BFE0AE00021322296
:102B0C000170744880F82A1073480421007827F06B
:102B1C005BF984F004000FB0BDE8F08F84F0800006
:102B2C00F9E70522027091F82C2092072CD591F828
:102B3C002E204ABB052202600120487000201CF0A8
:102B4C0097F8022024F05CFDE3E764480078013834
:102B5C0001280BD80020CDE90A000AA812F024F8AD
:102B6C0020B15D48022100781BF0CAFA84F0020003
:102B7C00D1E78178022904D10121817000201EF057
:102B8C0085FE84F48050C6E705200021B3E7534846
:102B9C000078002840F08680DFF838A1DAF80C5075
:102BAC00002D79D004A80DF1280B01300BF104068F
:102BBC000390002D6DD0A87A18B10138A8720006C8
:102BCC0046D19AF83180B8F1000F11D00020A91C21
:102BDC0008228DF82800304626F032FC584618F0B2
:102BEC0051FD28B12A88BDF82A00314623F02CFB70
:102BFC00AF1C0DF127015A46384616F0A3FD81464D
:102C0C00384609A923F099F8B8F1000F05D09DF8C2
:102C1C00380040F0020002281CD1DAF80800A0B1FC
:102C2C0003983946082226F00BFC022000220C23C4
:102C3C008DF81000BDF82400ADF81A002648007875
:102C4C0004A90091092120F0D6F928461EF014F8A9
:102C5C00ED68AEE7384623F0CAFD9DF82700012841
:102C6C00DBD15846142127F053F8224A09EB4900CE
:102C7C0000215B4642F8201002EB800014224160D8
:102C8C004172FF2049468DF83800042023F0D6FC11
:102C9C00C3E7DAF80C0028B90F484FF4006100784C
:102CAC001CF09AFE84F4006035E7013A012A09D839
:102CBC00032202600120487001201BF0D9FF012083
:102CCC0024F09EFC287800287FF423AF04205CE7D6
:102CDC000C7A0020AC220020A37A002024260020AD
:102CEC00C0BA020070270020BA270020A86D00206F
:102CFC00EC580020F03300202DE9F04F89B021F082
:102D0C0079FBDFF810158122DFF81485DFF814A5A4
:102D1C00DFF82045DFF814E50A70DFF8FC140860D2
:102D2C00DFF8F804FF2101700020DFF80415A8F883
:102D3C0000008AF80000DFF8F0040968007891F8C8
:102D4C0008B04FF6FE718EF8000059448AB2A168A3
:102D5C00D1F80031DB899A4200F267810422DFF856
:102D6C00DC54A8F80020DFF8D02412689668330EE3
:102D7C00CEF80C60C6F301592B706FF0FF0303EA19
:102D8C001627B3B2D1F8B86047EA1327AEF804702F
:102D9C0036781EB9B9F1020F00F04781B9F1030F73
:102DAC0000F043811B0A03F0070316B1002B00F05F
:102DBC003C81DFF88CC4042B9CF800C008BFBCF12C
:102DCC00000F00F032813EB1DFF878643678862E41
:102DDC0002D1022B40F02981BB0416D4BBB203F004
:102DEC000703022B08BFBCF1000F20D0DFF85414EE
:102DFC000978862909D10020764621F04FFBDFF8AF
:102E0C004004B64690F800C0307800284ED0BCF193
:102E1C00000F4BD1012800F0088103283FD0022875
:102E2C0044D1BEF80400400740F0FF803EE0D1F8EA
:102E3C00D40090F88300022800F0808027460520FB
:102E4C00147BF246A946A8F8000026F0CFFC0546F4
:102E5C00DFF8F003007886286DD1B868016C09683A
:102E6C0011B9D0F84C05804760B20021002623F040
:102E7C0012FDB9680A6C12685077086C0068867786
:102E8C00086C0068C477284626F06BFFBAF804106B
:102E9C0099F8000001F010011CF018FF4EE0BEF88C
:102EAC00040000F00700032840F0BF80BEF80400C7
:102EBC00010700F1BA80810402D4810500F1B580CC
:102ECC009EF80E20C2F38107012F00F0AE80960908
:102EDC00012E00F0AA80B9F1010F11D840F00201C7
:102EEC0001F0070103290BD117B93F2A40F29D804D
:102EFC0037B9A168D1F8AC100978002900F0958099
:102F0C004FF6FB71B9F1020F0BEB010C19D1CF4B42
:102F1C00D95D9B5D03EB01090023402AB7FA87F2C8
:102F2C0038BF012352091A40430616D4002A08BFA1
:102F3C0009F1020915E0284626F013FF25F06EFB77
:102F4C0075E0C14B402AD95D9B5D03EB010908D3A9
:102F5C00420648BFA9F1020903E0002A18BF4FF04E
:102F6C000209C0F300205FFA89F11FFA8CF30A1AE8
:102F7C008EF801009A4258DC60440391B346401A23
:102F8C00A168AEF806007430D1F8501280B28847B0
:102F9C00A6490028886048D07421CDE9019726F015
:102FAC00B7FEA24F0020B870A548007820B9387938
:102FBC0000F020008AF8000078789AF80010DFF80A
:102FCC0078C24FF000092E4600299A493DD00028BE
:102FDC004FF000003AD1B88800F00700032807D062
:102FEC00012832D18868D0F8D40090F8820060B300
:102FFC00C8684069007818B125F06EFFFE280DD026
:10300C008C488068D0F84C02804738B98948806871
:10301C00D0F844028047002800F0F780834F01204D
:10302C00B870DFF814C22E4610E025F0B1FD26F082
:10303C00DDFB814900240A6813681C7112680A6060
:10304C0026F08FFE09B0BDE8F08F0020BC6804F1BB
:10305C00740184F830B06160A1657978BB88FA8816
:10306C000029A381029B228184F83A30337808BF6F
:10307C009946B8F8003097F80EB0019DA4F85C2082
:10308C00FF2284F84990A2735E1A797BCBF3011965
:10309C00A8F8006001F0780160F3820101EB0900EF
:1030AC002074280600F0AE80DCF8000004AF039A10
:1030BC0010FA86F000F10801384626F045FF56FA62
:1030CC0085F0CBF38105A8F80000207C00F04008C7
:1030DC00CDB3B9F1020F06D1B8F1000F03D0B4F89B
:1030EC00440004AF06E0BDF810000237A4F8440019
:1030FC00A4F84200564EF189884203D04FF6FF7176
:10310C0088425ED1032D11D104F13200394626F0EC
:10311C00A0FE464CF11CA068323024F018FC454946
:10312C0000284ED094F80EB008370EE037F8020B9A
:10313C00B1898842608606D04FF6FF713B4C8842BD
:10314C003C493ED101E03B49384CBBF1400F20D308
:10315C00B9F1020F06D16DB9B8F1000F0AD133489D
:10316C00806803E0A068017C490603D439880237E3
:10317C00A0F84210BBF1C00F06D32C4C3946A06806
:10318C00283026F066FE03E0284C3888A1680885B4
:10319C0028498968A088D1F8AC201278B2B1B9F16D
:1031AC00020F13D200F00700012802D003282FD100
:1031BC001E4C6DB9264AA368D289B3F842309342AB
:1031CC0006D01FF01AFA19F011F930E700F00700D9
:1031DC00032806D0012815D1D1F8D40090F882002C
:1031EC0080B1A068D1F848128847104A50B9002025
:1031FC00D17B9070907BC1F3011100F078000844F2
:10320C009168087408F0ECFB11E7084FB87808E7F0
:10321C00064CDDE7B07A0020387A0020B57A002021
:10322C00BE780020B37A0020B27A0020342500202A
:10323C00787A00200C010020D8790020C37A002075
:10324C00C27A0020B87A002048BA020044BA0200C0
:10325C00007900202DE9F04F97B0DFF80C8505467A
:10326C00DFF8086598F800000328307040F04981B9
:10327C00002088F8000030700DAC204626F0F5FDDB
:10328C002046002125F0D8F9DFF8E494B0603A210B
:10329C00484626F03DFD4FF0FF30A9F81400C9F860
:1032AC001000C9F80C0022F0F3FE002029461EF095
:1032BC0065F806F11001F06026F065FDD6E905020F
:1032CC00DFF8B074B0FBF2F1C9B2032928BF0321B7
:1032DC00B2F5005F89F80010397040F00F81B0EB47
:1032EC00413FC0F00B81F068002800F007814FF4DB
:1032FC000050FF224FF000084FF0885BA9F8060041
:10330C00FF2089F8032089F805800590002008909B
:10331C0000200B90002009900020079000200690C0
:10332C0000200A9000200C90FF200290FF200490B7
:10333C00FF200390CCB2A04580F0E6805FFA88F6BF
:10334C00002116AA0423304626F042F8DFF82C445C
:10335C003046002115AAA0473046012114AAA047E7
:10336C003046022113AAA04716996FF06F0050FA4D
:10337C0081F2C8B20E2A06D8012303FA02F245F2F2
:10338C0001131A4203D1A0F1FE02022A04D242F226
:10339C008352B2EB914F1ED0304614F073FADFF823
:1033AC00CC130028087040F0CF803046002116AABC
:1033BC00042326F00DF8DFF8C4433046002115AA8B
:1033CC00A0473046012114AAA0473046022113AA77
:1033DC00A0471699C8B208EB48023D46CA4609EB0D
:1033EC008204C1F30142090AE1759DF8561004F1FB
:1033FC001609FD28627689F80000217601D9102182
:10340C0036E0BDF854104FF6FF72914230D10EA841
:10341C0020F050FD304600214FF088524FF40053FD
:10342C004FF4005725F0D4FF6FF0030313FA87F71E
:10343C00B8B250F80B104A1C01D10328F6D801225F
:10344C000126D3B2042B06D8CBB2FF2B18BF1646DD
:10345C000132090AF5E740F80B10C9480E990068CB
:10346C004268C848904757FA86F081B299F8000034
:10347C00A1839DF852107028A176BDF85010E183FD
:10348C009DF84E10E176BDF84C10218411D07828AF
:10349C00D14614D07C282F4616D07E281AD0FE2870
:1034AC001FD0FF2823D10898CDF80C80013008904C
:1034BC0020E00A98D1462F4601300A901AE006986F
:1034CC002F460130069015E00798CDF8108001309A
:1034DC0007900FE00998013009901FFA88F00290CC
:1034EC0008E00B98CDF8148001300B9002E00C989A
:1034FC0001300C90397808F101081BE7012088F89D
:10350C00000017B0BDE8F08F0C98984E00060BD158
:10351C000B98C0B2012807D80A98C0B2012803D86A
:10352C000998C0B2012811D99348042200240270D2
:10353C00CAB2E0B2904210D214F0A4F9317801343E
:10354C00084339783070F3E7884E1BE0089BD8B2FB
:10355C00A04219D1884800220270002089F803008B
:10356C0089F80100481E7E2189F80200B9F81C0078
:10357C00A9F80600002021F0DFF999F80200FE21DD
:10358C0021F0DAF93078BCE70A98000624D00B98C1
:10359C00059A000603D1039A180600F08480764839
:1035AC0002210127D5B289F80220017017FA82F0A6
:1035BC00B0FBF4F101FB140089F80100284614F06B
:1035CC0061F930702846FE2121F0B6F989F80570B2
:1035DC000020FEF7F5FDD5E70B98059A000621D0E3
:1035EC006548012189F80220017011FA82F0049AD1
:1035FC00B0FBF4F101FB140091B2FF2989F8010032
:10360C001FD10299FF2919BF89F8031001EB410062
:10361C0089F8030000EB400009EB8000808BA9F8CF
:10362C000600AFE7DDE90620104300063FF47CAF4F
:10363C0022F002FDA04280F085804F4803210170EA
:10364C003EE0480089F8032010FA82F009EB800074
:10365C00818B1829A9F8061094D30739D0B20EAA79
:10366C0089B216F085FF9DF843004007B0D5B9F834
:10367C000610BDF84620002399F80300009303239D
:10368C00891A0EAA073989B206F0B0FF00287FF418
:10369C0079AFBDF8441000293FF474AF9DF8480091
:1036AC001DF0D6F86EE722F0C7FC0621A042324886
:1036BC0038BF03210329017002D0062952D061E7DB
:1036CC0022F0BAFC054689F80C0000EB400009EB2F
:1036DC008000408BA9F80D000CF06EFE3978284460
:1036EC00B0FBF1F202FB110089F802000130C2B20A
:1036FC00B2FBF1F202FB110089F801007C2021F0F1
:10370C0035F9FF2812D17E2021F030F9FF280DD198
:10371C00FF2021F02BF9FF2808D1782021F026F981
:10372C00014699F80100FF2918BF0846C1B289F873
:10373C000300490051FA80F009EB8000808BA9F856
:10374C0006001AE70898000609D099F80200FE2135
:10375C003C46374621F0F0F82478039A40E70648B7
:10376C0006210170FEE700BF98270020A02300204F
:10377C00B87200209B7A0020A77A0020F7950200EF
:10378C00D8010010004003402DE9F84305460C46D3
:10379C00480413D4A00024D4A0075CD460057ED4C4
:1037AC00200500F10681200700F13B81600040F10B
:1037BC00F6801AF009F824F08044F0E026F016F8B0
:1037CC00DFF81C140F6D3FB1D7E90A1202F0E0428A
:1037DC0001F00A01891849D026F0C3FA24F4804478
:1037EC00DDE0BB48DFF8FC73016841F0800101604B
:1037FC00B878012804D1042021F020F90020B870F9
:10380C0025F0F4FF0646042026F098F8DFF8D813CC
:10381C000A68904219D12A7EBAB1FA68AAB1DFF8C7
:10382C00C003806C002800F09780C16840F603024A
:10383C000988914206D0C06840F60401008888428D
:10384C0040F08A8005F1140088E040F6C41208604C
:10385C00C5E9042284E009F0ABFBDFF88403006CBB
:10386C00002840F09D8024F0020498E0D7E90A6516
:10387C00D7E90A12AA43B143C7E90A1226F071FA32
:10388C00B8680028AAD056EA0500A7D0D7F808C017
:10389C003869B7F9301032462B46E0479EE725F0E1
:1038AC00A5FF054623F0E6FD002800F0B780CC48C4
:1038BC00876B002F00F0B280DFF828830420CB49FF
:1038CC00002288F81800C64825F0FCF926F076FA94
:1038DC00C74826F040FAC7480068006B8047C8F814
:1038EC0010000125042088F8025021F0DFFE386911
:1038FC0090F82810C8F80400490703D5436A04213E
:10390C000022984701201BF055FCD8F8040045769E
:10391C0013F096F8D8F8040081680B461A465B68D9
:10392C004BB11E88A6F60306072EF7D805FA06F645
:10393C0016F0830FF2D0537B03F0F0030133537373
:10394C000023FD6853602D88A5F60305012D00F2B8
:10395C008A80C8F810309FE005F110001EF0FEFAC6
:10396C00304626F0FEF921F0B9FE78B12E6A2846D1
:10397C006FF4807100224FF00073B0479848806B51
:10398C0010B119F021FF01E044F00204EE69284661
:10399C00002100224FF08063B04724F0005434B172
:1039AC00974821462830BDE8F84326F0BDBABDE85B
:1039BC00F8838C4EB078012804D1042021F03EF815
:1039CC000020B07021F08AFE38B170686FF48071FD
:1039DC0000224FF00073056AA847306950B1854842
:1039EC000068006B804732697168801A000BC860F0
:1039FC00002030617A4D81490022284625F062F979
:103A0C0002203076286C20B17D480221283026F027
:103A1C008BFA19F0D9FE24F40064C0E726F0CEF935
:103A2C0041E025F0E3FE054623F024FDA0B1DFF8CC
:103A3C00B48198F8000000070ED498F90000002813
:103A4C000AD4684613F038FA08B1009820B1DFF8B0
:103A5C00B49199F8610048B326F0B0F919F0B4FEAE
:103A6C0024F008049BE7034633F8385FA5B190F8BF
:103A7C00445090F8456005F0F00580F8445006F08D
:103A8C00F005013580F8455000255360C563458726
:103A9C00507B00F0F000507357480022C261016067
:103AAC00012024F027F924F4806478E7002601270C
:103ABC00602E0FD009EB0600817A31B18772407A03
:103ACC0007FA00F0C0B220F0D3FF2036F0E700BFB9
:103ADC00CC210840032088F81800454826F03BF913
:103AEC0026F06CF9444F3E4D002278690020786135
:103AFC00F968F8602846444925F0E4F83D48006828
:103B0C00006B8047D8F80C10D8F82020411A02EB33
:103B1C001130B0EB113F38BF4FF0FF3098F8241044
:103B2C00C8F8200021B1D8F80810B0EBC12F20D96B
:103B3C0024F0F0F8B8B140F60900414621F83C0FEA
:103B4C00002048804A7B02F0F00201324A730A7B63
:103B5C0002F0F0020A734860F8613960B8F83E0070
:103B6C0010F4406FFAD00020C8F82000012088F82B
:103B7C0024001DF0BBFB2548002101600220002120
:103B8C0024F0B8F8022020F059FF102012F008FBA6
:103B9C0098F8010020B9D8F80400503026F0C0F98C
:103BAC001B48807810B90D2012F0FAFA98F825000D
:103BBC0028B1002088F82500052020F03FFF0020C8
:103BCC0088F818001348C8F81C000220B5F85610E5
:103BDC00B5F85420914208BF072018F077FF3DE755
:103BEC0030210020D01E0020E02600205D74020051
:103BFC00387100208C01001000100440F50C0100FD
:103C0C0070200020206E002039D8010000000460D4
:103C1C009CB90200D50501002DE9F04F8DB08478D8
:103C2C000226142C00F21F820546DFE814F029004E
:103C3C00150015004A0085001C021C021C021C0207
:103C4C001C021C021C021C021C021C021C028E0008
:103C5C009C00AF00BE00CC0001206A78022C8DF8CD
:103C6C003100089240F0C080E878291D03288DF8B7
:103C7C002C0040F0E18009A8082225F0E1FBE0E0EF
:103C8C0010208DF82400102026F038F998B1044645
:103C9C00DFF8E00321466060E81C10F017FC8DF89B
:103CAC00240028B9204623F087FC8DF8240010B19D
:103CBC00204626F021F9002609AB642000210122C0
:103CCC00C2E10020CDF82A00ADF82E00CDF8260078
:103CDC0002208DF82C00E81C26F00CF9ADF824001D
:103CEC006979A8798DF82D1025F03AFC8346E81DEA
:103CFC0026F000F995F80C908046687AAC7A95F825
:103D0C000BA04FEA49078DF83100384626F0F6F83B
:103D1C00002800F01081CDE9074806464FF0000856
:103D2C0005EB0800474570D00D3026F0E3F826F877
:103D3C00080008F10208F3E7E87820F083FF8DF81B
:103D4C00240009AB6420042189E1E978032900F2FD
:103D5C005281281DDFE811F00400510155015D016D
:103D6C0018F056FF76E1E81C26F0C4F8C04C6668E3
:103D7C00002E00F0E4806A79002A00F0E4803368B9
:103D8C00A91D184425F05CFB0020D9E0B84EEC1CB2
:103D9C0004212046376822F0EBFC002F4AD0B9688A
:103DAC00814200F0A0803F68F7E7A888ADF82400B6
:103DBC00E87809A924F07CFB8DF832000DF1320370
:103DCC00642013214BE10026E878ADF8246009A9A2
:103DDC0023F08AFDBDF824000DF1320314210222D8
:103DEC00ADF8320064202FE1E81C02218DF82C1074
:103DFC0026F080F8ADF82400002005F10608ADF897
:103E0C002E0068798DF82D0026E0BBF1000F00F034
:103E1C00B580437B0DF131010E30CDE90496CDE92F
:103E2C00000107985946CDE9020A09A8089A1DF025
:103E3C00DBFEA4E0012000E1084626F05BF8ADF8BB
:103E4C002400287B8DF82D0005F10D0026F052F88A
:103E5C00ADF82E0005F10F0898F8000025F080FB56
:103E6C00054608F1010026F045F898F8036098F82B
:103E7C0004A098F805B08146022C8DF8326009D167
:103E8C0008F1060026F036F8074608F1080007F19D
:103E9C000A0104E098F8067008F1070039464DB1A4
:103EAC000A3189B2FB2907D3DFF8C481D8F80400A2
:103EBC0000286ED0022009E00DF132018DE8030CD0
:103ECC0009A84A463B46294603F012FD089E8DF888
:103EDC00310006F0E000202840F0C4800DF13103E1
:103EEC0064202146BBE0EC1D204626F003F86D7AD9
:103EFC00002D00F0978005F102098246484625F016
:103F0C00FDFF002800F098800026457080462A4668
:103F1C000670786800EB0A0108F1020025F090FAAF
:103F2C005FFA89F26420122143461EF027FC4046BA
:103F3C0025F0E2FF97E010208DF8320024E01020ED
:103F4C008DF8240016E0D6F800C0F38AB28A3169E5
:103F5C00757EB77E06F11800CDE900C0301DCDE9A5
:103F6C00025703F0C5FC8DF82400606825F0C4FFEF
:103F7C000020606009AB6420112170E002208DF8F4
:103F8C003200304625F0B8FF0DF1320364200321D6
:103F9C0065E007F11C0025F0B1FF0028C8F804000B
:103FAC0055D000F11C010C22016000208DF831006D
:103FBC00D8F8040009A9043025F042FAD8F8040016
:103FCC000F214FF47A7205612A4DC17680F81AB030
:103FDC0080F819A00676C782A0F8149008212878DA
:103FEC0025F0F2FE089E00283FF473AF28780821D4
:103FFC001AF086F86DE702202CE000781AF0B0F881
:10400C0028E0007825F0ACFA18B324F0ABFF0020C0
:10401C0020E025F06FFFA97925F0C0FCB0FA80F004
:10402C00400917E03068B84201D138683060384632
:10403C0025F062FF002000E0102000262070642094
:10404C0012210222234666701EF098FB0BE0102012
:10405C003CE701208DF8240009AB642010210122DB
:10406C001EF08CFB002630460DB0BDE8F08F00BF73
:10407C00682600209A7A00202DE9F04F8FB00C466C
:10408C0008040CD4A00426D4DFF88853287802281E
:10409C002DD1E10740F00381A10641D558E0DFF8AE
:1040AC006C0300781AF0FEFC90B10178DFF8602305
:1040BC0005460020602808D0135C08308B42F9D1EB
:1040CC00104450F8041C28468847284624F00EF863
:1040DC0084F4004595E11DF08DFC28B10546FCF7F4
:1040EC00C1FD284624F002F884F4005589E1A106AC
:1040FC002ED4012814D8E10600F11781610600F1D5
:10410C002F81210600F13D81E10500F13F81210560
:10411C0000F14181E10400F15481610400F15B8103
:10412C00A10700F1E280A10500F1FA80210700F15E
:10413C001181610500F11981E0034FF0000540F198
:10414C0060811BF037FFB648C57084F4803558E1A8
:10415C00AE4F202138781FF02FF9DFF8C4824FF0D2
:10416C000109D8F80810084317D025F099FE054628
:10417C0025F094FE68434FF47A71B0FBF1F0D8F857
:10418C000810401A4FEA500938BF6FF0004900255B
:10419C00002964D0B9F1000F61D000200421002265
:1041AC0022F08CFE06464FF0060A4FF0FF0B4FF63E
:1041BC00FF7802AD002E4ED0304604210022374647
:1041CC0022F07CFE06463889B0EB090038BF00208F
:1041DC0038810004EED1B87BD0B301280AD178899C
:1041EC00400707D4386887F80DA0B721407B1DF035
:1041FC00B9FBDFE739682A468DF806B0ADF80480C4
:10420C00086AC97F0CF0E4FF01281BD1B87BB97A8E
:10421C008DF838000907788A40F08002ADF8362016
:10422C0006D540F4C070ADF83600387B8DF83A00F6
:10423C00786910B1007BADF81800284601A900225E
:10424C0002F018FC387B87F80DA016F091F8B1E756
:10425C0001207873AEE7DFF8C8816C4F4D4622F031
:10426C007AFF00200121002222F028FE18B13878B4
:10427C00202119F045FF002004210022002622F005
:10428C001DFE002847D006890421002222F016FECC
:10429C00A0B1B1B20689B14238BF0E46F4E764480A
:1042AC0090F82C100F2906D190F82600022802D382
:1042BC00002021F0CBF984F00105A2E0A8B2B1B244
:1042CC00814223D9D6FA55F0202180B242003878A9
:1042DC0025F07AFD25F0E4FD054625F0DFFD684369
:1042EC004FF47A71B0FBF1F615E05248007808B340
:1042FC0002AD284625F0D3FC25F09CFA4E490B78EC
:10430C004E490A7829461AF0D1FE20E0387820214F
:10431C0019F0F6FE0026C8F8086084F0200570E05D
:10432C0015F062FC84F400756BE008F04FFA84F031
:10433C00100566E03E48418B012025F0D5FD28781C
:10434C00022804D13148012100781BF045FB84F090
:10435C00020556E03248012184F00805817050E0D6
:10436C000CF0B6F984F040054BE0022808BF15F0BC
:10437C00FFFE2F480121808C25F0A8FD84F4806578
:10438C003FE024F0B5FA84F080053AE022F0B6FB69
:10439C0084F4807535E01BF073FB2048007801280D
:1043AC000CD11D48007848B14FF47A7100FB01F232
:1043BC0016484FF40061007825F003FD84F4006585
:1043CC001FE01748017819B1002101701BF058FB50
:1043DC0084F4805515E01448006880B111490978BF
:1043EC0001290CD180471148006800B1804707486B
:1043FC004FF480414FF47A72007825F0E2FC84F49B
:10440C00804528460FB0BDE8F08F00BF9C7A002095
:10441C00BCB2020024260020CC270020CD2700208F
:10442C00E8250020CA2700208423002090230020A8
:10443C00A86D0020A7270020D0270020D22700201D
:10444C002DE9FE4F8846080426D45FEAC87004BFE5
:10445C000020BDE8FE8FE548056825F021FD0446E7
:10446C0025F01CFD60434FF47A714FF6FF72B0FBE0
:10447C00F1F14FF6FF70002D00F01A812B886C883B
:10448C00CB1A9BB29C4240F21C81E31A94B2A34219
:10449C00B8BF1A46ED68EEE7DFF840A3CDF804800C
:1044AC009AF800001AF0FEFA002800F0FC8006468C
:1044BC000078012840F0EC80DAF8041096F833907C
:1044CC00D6F814B096F8138021B1484688470028D6
:1044DC0040F0DE80718896F83100022222F05AFA00
:1044EC000546002842D0287A297CA0F10108FF2932
:1044FC0000F0BB80707F4F46C00718BF0027E97CD7
:10450C00287D0144B94204D8E974FF2101FA00F076
:10451C006874A969A87C96F83020896A10FB07108A
:10452C00F16A24F08DFF287D697CB7FBF0F202FB69
:10453C00107001228240D2B20A436A74C8457CD101
:10454C0096F83010AB7C13FB0713A9698B844FF4DE
:10455C00FF7303FA00F0C0B21043FF2868746CD1EB
:10456C00287C1AF0FBFDFF2028747FE0707FC007C9
:10457C0000F08E80B07F24F0F3FF002800F08880DC
:10458C0004461C2025F0BAFC002800F081801C2178
:10459C00054625F0BDFBB07F02A923F0A5F99DF8D7
:1045AC00090002212875284623F0F4F9708896F842
:1045BC00312096F8301096F83330A880287DEA71B7
:1045CC00FF2202FA00F0687460680078A9742874FD
:1045DC00302013FB010080B222F0AAFE0028A86153
:1045EC005DD004461A20B11C2060708CA080A01DE8
:1045FC0023F06CFFF27F04F13000B17F96F8283085
:10460C00C4F81CB084F81980A062307CE273744A40
:10461C00217563750121A075928C2282F28EA28580
:10462C00F28C6282B6F81100A4F817009AF8000018
:10463C0085F8089019F064FD55E725F031FC044627
:10464C0025F02CFC60434FF47A71B0FBF1F0654916
:10465C0028806348097800794843642148436249BB
:10466C00097800FB0100688000E04F46E87C297D5A
:10467C006A7C01440139B94218BFFF2A0CD186F873
:10468C003300708806F11C0186F8342016F085FF83
:10469C00304623F02BFD03E7C845F9D1EFE7284658
:1046AC0023F088F9F4E7019880F40040BDE8FE8F10
:1046BC0092B282424BD049480121007825F084FB0C
:1046CC0045E0A879022806D1287CFF2837D0A869B4
:1046DC0023F00CFD33E025F0E3FB044625F0DEFB74
:1046EC0060434FF47A71B0FBF1F03F49288095F8A4
:1046FC003800097888421BD295F83620FF2A06D15B
:10470C0095F83720013085F8380085F8362095F873
:10471C00351095F8394082F0FF0300200126C7B20E
:10472C00A7421DD206FA07F71F4214D10130F6E753
:10473C00EA8BA87E95F82A10E9231EF087FF2846FD
:10474C0023F038F925480121007819F0D9FC88F0BC
:10475C000100BDE8FE8FFBB201441A4385F83620F8
:10476C00AB8F95F83440C8B204FB10339EB2A6420E
:10477C0003D2FF2285F8362002E0FF2A08D1234617
:10478C00184A174E1278367972436426724302E047
:10479C0095F83A2023466A802A8D0E0606D022F020
:1047AC00200244432A852A6C224404E042F0200172
:1047BC002A6C2985297A85F82E10E9796A6285F8A0
:1047CC002D10D9B269840549496811B18847002870
:1047DC00B8D105F1100004F011FBB3E74826002016
:1047EC00A86D0020C0270020C62700206C53002095
:1047FC007FB50138072800F24C810C46DFE810F039
:10480C0008002C0054006E0089004901A600C90064
:10481C00CB4800780138012800F23B81002C00F0D5
:10482C0047810020032100241FF02CF9C64DC74EF0
:10483C000420042132222870307825F0C5FA082093
:10484C00002107F011F830786C704FF4805104B0EF
:10485C00BDE870401BF0C0B80020002524F088FE95
:10486C00BB480121017004208DF80D0074B1B548CE
:10487C00B34C45852078012803D1072023F08AFA10
:10488C002078022802D1062023F084FAAE480421B5
:10489C0032220570AD48007825F096FAA94890F8B8
:1048AC002B1001F0FE01F2E0A54800780138012838
:1048BC0000F2EF80A54804213222007825F084FA1A
:1048CC00002C00F00F819F4C9F4801210170206942
:1048DC00002800F0EC801FF0E5FCF8E70120002C2C
:1048EC008DF80D007BD0974800219B4A80F82A1048
:1048FC00984824F0FFFF924C2078012803D1072020
:10490C0023F048FA2078022870D1062023F042FACE
:10491C006CE002208DF80D008A48002C73D0002129
:10492C008D4A80F82A108B4824F0E4FF00200321E4
:10493C001FF0A8F8824C2078012803D1072023F01F
:10494C0029FA2078002877D1092073E07C4D0020CB
:10495C008DF80D00002C28787BD018B9092023F095
:10496C0019FA2878022806D10820002106F07CFFCD
:10497C00042023F00FFA10F095FF73480021C82291
:10498C00017070480D2180F82A10704825F0A3F9A9
:10499C0078E005208DF80D0069480078022878D160
:1049AC00002C00F0C38068480022C178C2700170EE
:1049BC0042F20800002106F057FF62480D2190F8E2
:1049CC002B2080F82A10C17802F0DF02002980F831
:1049DC002B200CBF04200D2023F0DCF959E05848A3
:1049EC00007818B95748022180F82A10564800213F
:1049FC0032220170554825F06EF9524890F82B1070
:104A0C0001F0FD0143E0082180F82A104C49097897
:104A1C00012911D890F82E0070B900200DF10A016F
:104A2C008DF80A0052201DF0A9FB24F031FB1EF07A
:104A3C002DFC002023F0AEF94348002132220170F6
:104A4C00424825F048F93F4890F82B1001F0FB0143
:104A5C001DE03C4C022812D194F82E0078B194F849
:104A6C002B00002140F0200084F82B0005208DF84D
:104A7C000D00082006F0F8FE0A2023F08BF9022026
:104A8C0084F82A002F4890F82B1001F0EF0180F8E1
:104A9C002B102C480022032390F82A008DF80C00D0
:104AAC002A48007803A900910A211EF0A4FA7FBDC0
:104ABC00244C0720254D4FF4805184F82A00012006
:104ACC008DF80D0028781AF087FF0020002622F0C0
:104ADC0069F92878022141F2883284F82B6025F09C
:104AEC0073F9D6E7174C022000218DF80B1084F8CF
:104AFC002A001548017094F82B000DF10B0100F001
:104B0C00FD0084F82B0001208DF80D0052201DF0C3
:104B1C0035FB24F0BDFA1EF0B9FB002023F03AF966
:104B2C0020690028B5D01FF0BDFBF9E7054802212C
:104B3C0080F82A1090F82B1041F02001A7E700BF55
:104B4C0024260020AC2200200C7A0020A37A00201E
:104B5C00BD270020A86D00209027002092B0DFF820
:104B6C00EC92D9F8000010B1002180F845104830C3
:104B7C0020F094FF24F03AFE8046072011F0AAF8AA
:104B8C0017F0DAFF10B1B24824F0D4FF1AF06AFB28
:104B9C0001AD284624F0C4FC0427002029468DF8DA
:104BAC00047024F0C5FCAB4C206024F031F90AAD44
:104BBC00284624F065FB002029468DF8287024F047
:104BCC0067FBA54E306024F02DF906AD284624F085
:104BDC0067FB002029468DF8187024F069FB3168BA
:104BEC009E4D286019B99E4824F0A4FF286810B97E
:104BFC009C4824F09FFF206810B99B4824F09AFF32
:104C0C001CF0D8FDD9F800004FF0FF3438B1CDE9D5
:104C1C00104410A9082223F05DFB01281BD1CDE91B
:104C2C001044082025F06AF9002846D005460026D5
:104C3C00052E04D824F0E8FFA8530236F8E74FF607
:104C4C00300029460822E880884824F0F9FB2846E1
:104C5C0025F052F909E0D9F80010CDE910440029EB
:104C6C00DFD08248082224F0EBFB10AA0120082197
:104C7C0024F01EFF092800D0D8B921F075FE80075A
:104C8C0012D4CDE91044CDE90E440EAB0120002125
:104C9C00082224F06BFA60B90EA810A9082223F0A0
:104CAC0019FB002800F0CB80704A0120082124F069
:104CBC0005FF6E49E2201DF061FA12F0CBFB2820B3
:104CCC0025F01CF96A4E0028306055D0694F6A4CAB
:104CDC0007F10C0524F0FBFF24F042FB3068056063
:104CEC0007F1100524F0F3FF64498968D1F84C13DF
:104CFC0088473068456007F1140524F0E8FF1CF084
:104D0C0083F93068856007F1180524F0E0FF19F08D
:104D1C00B5FD3068C56007F11C0524F0D8FF1FF005
:104D2C0007FD3068056107F1200524F0D0FF1EF067
:104D3C007FFB3068456107F1240524F0C8FF1DF0A6
:104D4C0095F93068856107F1280524F0C0FF23F040
:104D5C0053FE3068C56107F12C0524F0B8FF20F034
:104D6C0025FE3068056207F1300524F0B0FF38707D
:104D7C0024F05CF93068456218F0B6FE40484149B1
:104D8C004FF00009CDF8409001603F48032111908D
:104D9C0010A820F043FC24F0BBFC404624F0E1FFBB
:104DAC0017F0ECFA24F058FF01201DF0C7FE19F0A3
:104DBC0031FF37480078022808D1344800780128A0
:104DCC0004D14FF40040012106F04EFD294F4FF461
:104DDC008041387824F0A6FD2E484FF0FF31006852
:104DEC000DF022FCDFF8B08078684FF0FF310DF049
:104DFC001BFC3068002550F82510096821B9691C86
:104E0C00092D0D46F7D3EFE724F0F9FE316851F880
:104E1C0025100C68C1F8009024F0DFFF58F825200D
:104E2C00002021469047044624F0E9FE316851F8F1
:104E3C0025100A6822430A6024F0CFFFD4E70B4800
:104E4C000EA9082224F0FCFA33E700BF68270020E3
:104E5C00B4B60200F4790020F8790020FC79002027
:104E6C0068B802007BB80200B2B80200B679002024
:104E7C00707A002088210020E14902000C010020FA
:104E8C009C23002001CA0100008D1500E52700209D
:104E9C00242600204C7A0020A4B502002DE9F04F06
:104EAC0089B08A4608040DD45FEACA7040F01F81AD
:104EBC005FEA8A7000F12D815FEA0A7000F135819A
:104ECC00002044E1A34F387819F0ECFDDFF88C9208
:104EDC00A64DA14C06464FF0000B48F21508002ECB
:104EEC0000F00281307831283AD032284BD0D328C8
:104EFC0040F0B480F089404574D0382840F0AE8042
:104F0C00CDF820B0CDE906BB304606A920F0A6FCB2
:104F1C009DF81C10052969D8307B002840F09E8034
:104F2C009DF81D00002800F09980052800F296805D
:104F3C00069823F0E8FE002840F09080707C8849A9
:104F4C00AC467870708808809DF81D0021460138A9
:104F5C008DF81D0006A890E82C002CC165467DE05C
:104F6C00B87803287AD899F82E10284623F0CBFE6F
:104F7C00002873D1FF207C49607170880880B0884C
:104F8C00784908806AE06079FF2814D0002016F078
:104F9C0051FA0246B9F8701078783346CDF800B063
:104FAC0012F0A0FD6079002858D038780821322200
:104FBC0024F00AFF52E099F81810706820FA01F2F8
:104FCC00D2071ABF3144097A002100221B2A43D090
:104FDC0020FA02F3DB0703D0B3181B7A99421ED8D0
:104FEC000132F3E7304621F03DFE37E0FF293DD09A
:104FFC00FE2956D199F872109DF81E00884202D8ED
:10500C0060BBFF292AD11CF0BBFE069900201B288F
:10501C0059D021FA00F2D20757D10130F7E7B9F88D
:10502C006E004F49334608804E4802884E4801882E
:10503C0010200090002012F055FD0120F870B87877
:10504C0040B93C2002214EF66022B880387824F01A
:10505C00BBFEB8780130B87084F805B0304623F048
:10506C0045F8387819F01EFD064638E799F87210A5
:10507C009DF81E00884203D80028EFD1FF29EDD1FE
:10508C001CF07EFE069838B1D9F82810814203D066
:10509C00C9F8280022F08EFEBDF8200023F0DCFCBD
:1050AC00DCE7307B0028D9D170882D498022002381
:1050BC000880707CCDE900BBCDE902BBCDE904BB17
:1050CC0011F01CFBCAE71B2000E0C0B299F81810C5
:1050DC008142C3D02649087099F80700642100FB6F
:1050EC0001F23878012163E78AF400402FE020496F
:1050FC001A4C08782076E1201DF040F822F05AFE78
:10510C000020A4F87000012016F094F98AF0010038
:10511C001DE010488188B1B101394EF660228180C2
:10512C000078022124F050FE0FE00B4C607938B16E
:10513C002179206823F0E7FD10B96079013860719E
:10514C008AF0080003E0002181708AF0020009B0A7
:10515C00BDE8F08FCC24002058790020A86D0020E9
:10516C009279002076760020F272002000F8FF077A
:10517C009F7A00202DE9F04F85B08846080418D49A
:10518C00AA480078012802D85FEAC87156D15FEAB4
:10519C0088714DD4022807D1A5480078012803D185
:1051AC005FEA487000F18A805FEA087059D40020E9
:1051BC002DE1DFF860A29AF8000019F073FC0028CA
:1051CC0000F023810546807FD0B9688C132817D155
:1051DC00DFF844926E880021D9F81C000F1D0029BD
:1051EC0008BF09F11C0758B101884468B14204D1C9
:1051FC003C6024F081FE2046F5E701462046EDE7B1
:10520C00A87A05F1020B022840F0E580DFF808923D
:10521C0095F83170BBF8006009F11C000068A0B172
:10522C000188B14202D18178B94243D00430F5E70C
:10523C0079480121017088F00200E8E07648406965
:10524C0000B1804788F00100E1E0D9F81C0000288B
:10525C0058D0012204464068114601320028F9D189
:10526C0052E07048DFF8B091807BD9F81C600007E1
:10527C0060D424F015FE044624F010FE6A4A604304
:10528C004FF47A71B0FBF1F0D9F818101288411A6A
:10529C0091427AD3B1FBF2FB0BFB02F2511A084498
:1052AC005E49C9F818001FFA8BF00978884288BF4C
:1052BC008B4641E059490978C170A3E05E495D48CD
:1052CC0000224FF6FE7300240978023079B130F8D1
:1052DC00025C9D4208D04588013D45802D0406BFE7
:1052EC00027020F8023C012401390630EEE734B19B
:1052FC00484804214FF4FA72007824F065FD88F0D8
:10530C00040084E000240021454889B200888142D1
:10531C0061D2082024F0F2FD00285CD00021068028
:10532C00877041603D490978C170D9F81C1079B378
:10533C0060603FE04FF0010B00205FFA8BF44FF000
:10534C00000A071D002808BF09F11C0796B1F07868
:10535C00C0FA5BF1A042F17006D8756830463D602A
:10536C0024F0CAFD2E46F1E7716830460AF1010AB5
:10537C000E46E6E75FEA0A4007D100200821C9F88B
:10538C001800244800781AF027FB88F008003EE04B
:10539C00C9F81C002348807B00070BD424F080FD47
:1053AC00044624F07BFD60434FF47A71B0FBF1F0BE
:1053BC00C9F818001B48807B00070CD59AF8000030
:1053CC0008211DF0F9FF30B91748082102889AF816
:1053DC00000024F0F6FC2878022810D0012811D106
:1053EC00297EAA89EB7C05F11C006C696E7E8DE828
:1053FC005A0005F11003594605F08EFA02E02846D2
:10540C0015F01CFC284622F071FE88F4004005B013
:10541C00BDE8F08F997A00202C240020C5270020AD
:10542C008A270020A86D00208E270020242600202B
:10543C00E5270020B45F0020A12700202DE9FE4FB6
:10544C00074608680024B0B1D7E9018A0E4624F05B
:10545C00CDF98146D8F8E800082888BF0124B06847
:10546C00204202D17068204208D003203074484694
:10547C0024F077FC00242046BDE8FE8FD8F8C0103D
:10548C0069B198F8F8100029EFD006213174D8F8DA
:10549C00C410C8F8C4604E6198F8FC100DE00021EF
:1054AC000522C8E93066C8E93411C8E9361198F804
:1054BC00FC10002908BF01223274002201297261FC
:1054CC0009D102204FF4E02188F8FC0098F8FB0089
:1054DC001FF0B4FF706889490138884205D8042050
:1054EC0020F0E4F8062020F0E1F8022020F0DEF8AD
:1054FC0098F8F80040B9DAF83C003168814203D2E0
:10550C0098F8FC0000286CD0D8E9361009B118B90D
:10551C0000E028B324F0E3FBDAF80000416941F025
:10552C0001014161484624F01CFC98F8F80008B1D0
:10553C000124A0E708F16C05D8F8EC10284624F0FB
:10554C0077FB0028F4D0D8F8C0000321017438464A
:10555C0012F0B2FF28460021002424F069FB8AE7F0
:10556C009AF8040024F0A8FC654CDAF8101002221A
:10557C00206991FAA1F1B1FA81F14368D8F8CC0015
:10558C004068006898472069DAF8141002224368D2
:10559C00D8F8CC0091FAA1F1B1FA81F14068006819
:1055AC0098479AF8040022F045FA9AF8040024F07F
:1055BC0085FC24F094FB0020C8F8E000D8F8C0006B
:1055CC000068B0F5806F01D924F089FB98F8FE00D3
:1055DC000028A1D1DAF80000416841F002014160D5
:1055EC009AE798F8F90020B1D8F8EC0001307FF474
:1055FC008BAF484624F0B5FBB2683AB1D8F8E80056
:10560C000221092838BF0121009103E008F1F402BE
:10561C0000200090746834B1D8F8E80002270928FB
:10562C0038BF012702E008F1F6040027DAF8000081
:10563C00334D416841F002014160D6F800B0D946C3
:10564C00BBF1000F40D0D8F8E800019209284FF0C8
:10565C00010011D22A68B9F1000F1FD0C0071DD06C
:10566C002178DAF800009268904700281EBF3C446D
:10567C00A9F101090120EDE72A68B9F1000F16D054
:10568C00C00714D02188DAF80000926890470028EF
:10569C001EBF3C44A9F101090120EDE7DAF8000036
:1056AC00D26802A99047DDE90120107007E0DAF812
:1056BC000000D26802A99047DDE901201080009813
:1056CC00ABF1010B0244BBE7D8F8F000DAF800109C
:1056DC00CA680240102802D1002AF9D101E0002A40
:1056EC00F6D0706822F040F8D8F8C0100020C8F846
:1056FC00C400C8F8C00008741AE700BFFEFFFF0F13
:10570C00C40100102DE9F04F87B0851C8346284654
:10571C0024F01EFB01AC06461821204624F0F8FAB2
:10572C009BF801A004F10B002946009524F091FB95
:10573C006FF001009BF80A1002240122ADF818004A
:10574C0000208DF81A408DF80C0001F00800C1F310
:10575C00C007890782EAD00507D40028B946A846B5
:10576C0008BF01240027002507E004244FF000099E
:10577C004FF00008002808BF03248548007850EA41
:10578C000A000BD0834890F82600082809D123F092
:10579C009FFD00285AD0BAF1010F57D14FF0C30921
:1057AC0001E04FF0C2090025BAF1000F10D07F487C
:1057BC00007890B9BAF1010F0FD1002E63D0002000
:1057CC00214601228DF81A0001A814F0D1FA0AE042
:1057DC0001A81BF0DFF986B91CE001A8214652464E
:1057EC0014F0C6FAB6B17179BAF1020F41F0400269
:1057FC00727104BF41F0600171719BF80A10490687
:10580C0003D5717941F080017171B17900240131B6
:10581C00B17100E00124B0FA80F149090D423AD18E
:10582C0007D1002D18BF814641F20100494621F0F5
:10583C00B0F814B9009819F089FBBDF818004FF6B0
:10584C00FE71884218BF24F063FB24E0DEB332798A
:10585C00A24218BFBAF1020F20D1D01EC0B201284B
:10586C0002D857EA050006D1501EC0B2012822D832
:10587C0059EA08011FD0308821F0F8FA20BB308893
:10588C00ADF8180022E00220214601228DF81A0002
:10589C0001A814F06DFA07B0BDE8F08F4FF00009C5
:1058AC00009953468DF81A903088ADF8180024F002
:1058BC000FFB012578E7012802D8308824F028FB5B
:1058CC00009819F043FB0026BDF818004FF6FE7146
:1058DC0088421ED121F086F810B1BDF8180011E0F5
:1058EC00BAF1000F04D02C4D288821F0BFFA30B14A
:1058FC009BF80A0000F002001FF008FF00E0288867
:10590C00ADF818004FF6FE71884202D14FF0C7096E
:10591C0049E79BF80A200099534624F0D9FA10B1B4
:10592C004FF001093FE71D48016811B1BDF818009F
:10593C008847BDF818000099224606F0C7F90646BC
:10594C00174818490A6800784FF4803124F03CFA63
:10595C0001211548C17096B1AAF10100C0B201280D
:10596C0007D81020BAF1020F08BF0820717908433C
:10597C0070714FF0000901258DF81A9014E74FF65D
:10598C00FE7000254FF001090026ADF818000BE75A
:10599C0004250020A86D00208027002098230020DB
:1059AC009C7A0020ACBA0200E825002024260020B6
:1059BC002DE9F04F8DB0044600209A4616460F464E
:1059CC00CDE90B00CDE909008A488568804615F0C1
:1059DC0061FA1C2803D015F05DFA1B281BD1308806
:1059EC0040F60201884218BFB0F5C15F03D1F07BCD
:1059FC00022810D93EE043F6070188420BD196F8F5
:105A0C002400032807D330697B4940F0806020F0E4
:105A1C00604088422ED100206FB366B3387825FAE7
:105A2C0000F0C00726D03046002124F061FA7348FC
:105A3C00C4E90176006880B109A800900CA90BAAF2
:105A4C000AAB304609F0D6FE0B980B214FF6FF72CD
:105A5C00502322F08FF8FF280CD023F0C7FE684F9C
:105A6C0006467878012802D840B1012070E0304613
:105A7C0024F077F900200DB0BDE8F08F09F02EFE70
:105A8C0060480DF10409016841F0020101605E48B3
:105A9C00C8F80000484623F033FDDFF870B15D49CB
:105AAC004A469BF801009BF8005003905848283058
:105ABC001EF0D3FD584859494A461EF0CEFD4846C3
:105ACC0023F02EFCDFF85881564A19214B460295DB
:105ADC0040461DF045FB544A08F11C001A214B4668
:105AEC001DF03EFB5148524924F009F951485249E6
:105AFC0024F005F95148006810F4402F06D0504AA4
:105B0C0007F128000421002321F07EFC9BF8020001
:105B1C0010B10D2010F0DEF808F1400023F0DDF894
:105B2C0008F1380023F0D9F84649002007223876CE
:105B3C00B8843862386181F860200521C7E9021009
:105B4C004149F96138700420002122F0D3F87878AB
:105B5C002F4941F8204001307870304624F001F98B
:105B6C00BAF1000F02D0DAF8000008E00DF1040AD7
:105B7C0036492022504624F0E7F94FF0FF30DAF88E
:105B8C000420BAF81010DAE90635002AB2FA82F6C7
:105B9C0008BF40F6C412206001207609618325639A
:105BAC0060762B4826764FF4FA766261C4E903627C
:105BBC00C4E90700C4E90903DAF80C0000B120625B
:105BCC00DAF8140000B16062DAF8080000B1E061A4
:105BDC0004F13800C82124F09BF804F15000002196
:105BEC0022F0C8F81B4904F1B80024F088F82046CC
:105BFC0041E700BFCC2108400F00000580260020A3
:105C0C00D01E002000200940110000E09CB90200C9
:105C1C00702000206D83020040720020714C010046
:105C2C003021002039D8010049B901007C710020D5
:105C3C00397402003871002019830200B44F0050EF
:105C4C00B1000200206E0020D505010094B60200C0
:105C5C00236E0100059E02002DE9F04F87B0002451
:105C6C000293002A00F03A81074603A892460E469A
:105C7C004FF0200B10300190504610F8011B2529D5
:105C8C000CD0002900F02781022EC0F0D680013EF6
:105C9C00002F00F0D18007F8011BCEE09AF801002C
:105CAC002D2806D19AF802000AF103034FF0010CDB
:105CBC0003E00AF102034FF0000C30280CBF13F87C
:105CCC00011B01462A2920D1029D2A68111D296039
:105CDC00D2F8009013F8011BB9F1FF3FDCBFC9F1FA
:105CEC0000094FF0010C2E291ED11A4612F8011B87
:105CFC002A291CD1029D2A68111D29609D1C12683D
:105D0C0059782B4622EAE27821E04FF00009A1F104
:105D1C003002092AE7D809EB890201EB4201A1F113
:105D2C00300913F8011BF2E74FF0FF380FE04FF08A
:105D3C000008A1F13003092B08D808EB880301EB0C
:105D4C004301A1F1300812F8011BF2E71346302889
:105D5C004FF0000241F0200008BF4A466C2808BFF3
:105D6C0013F8011B9A46692901D0642909D1029BB9
:105D7C001868011D196090456FF00903C8BF4246B1
:105D8C001BE075290AD0A1F16F00092858D8DFE86B
:105D9C0000F005695F5F835F5F5F5F05029D2868A8
:105DAC00031D2B6090454FF00803C8BF424678296D
:105DBC0008BF1023752908BF0A23DDF80480016889
:105DCC004046654616F062FCAC460546A8EB000161
:105DDC00A9EB0100BCF1000F0DD109E0022E05D397
:105DEC00013E17B107F801BB00E000270138013470
:105DFC000128F3DA01380A465AB1022E06D3013EC5
:105E0C001FB12B7807F8013B00E00027013A013560
:105E1C00F2E70C44BCF1000F3FF42EAF0128FFF663
:105E2C002BAF022E05D3013E17B107F801BB00E0E2
:105E3C00002701380134F1E70027013482461BE7C3
:105E4C00632905D1029A1068011D1160006804E0F5
:105E5C00AAF10100022E3AD300788DF80C00012132
:105E6C0003ADB5E7029ADDF804801023CDF800C02D
:105E7C001068011D11601099082200290168404624
:105E8C0016F004FC05464FF04000DDF800C005F8A4
:105E9C00010DA8EB05019BE7029ACDF800C0106834
:105EAC00011D1160109905680E480029002D08BFCE
:105EBC000546284623F048FC8045014638BF41463C
:105ECC0018F1010208BF0146DDF800C080E700218F
:105EDC0003AD82467CE70FB100203870204607B036
:105EEC00BDE8F08F7CBA02002DE9F04F8DB006466C
:105EFC00806A447874B18D4909788C4280F01281A3
:105F0C008B49023022462AB130F8023B013A21F883
:105F1C00023BF8E78748C18A708988422FD18348B1
:105F2C000078A04240F2FE80B589814A214628467D
:105F3C0022F078FA284617F017F8064682480778B8
:105F4C00BE4204D14FF6FE7017F00EF80646BE4264
:105F5C0080F0E880DFF8F48108EBC6094F4657F86B
:105F6C00040F08B123F0C8FF002C00F0B1806000D2
:105F7C0023F0C4FF0028386040F0AC80D2E0B27C43
:105F8C00002A00F0CF806A4F0025AC4205D037F8CC
:105F9C0015208A4203D00135F7E7A04600E0A84659
:105FAC00002113F0E5FF002800F0AD808146407918
:105FBC00012840F0A88099F8060010F0180F00F0A6
:105FCC00A280B9F80210204622F01AFBA54202D397
:105FDC00002800F098805848CDE90498B6F80C9049
:105FEC004FF6FE7A00780890544800780A9000200A
:105FFC0006960B9052481130099052480430079085
:10600C0000200C90DDE909564FF0000BF6B135F885
:10601C00117C574518BF4F4502D1013E1C35F5E7A1
:10602C002046394622F0ECFA0028F6D128780138BF
:10603C000528F2D80C980BF1010BC007EDD00B988A
:10604C005FFA8BF1C0B28142E7D356E0DDE90786F7
:10605C002EB338F8047C574518BF4F4503D1013E89
:10606C0008F12408F4E72046394622F0C9FA002842
:10607C00F5D198F8050001380528F0D898F80000FB
:10608C0001380228EBD30C980BF1010BC007E6D0BA
:10609C000B985FFA8BF1C0B28142E0D32DE05FEA3E
:1060AC000B6028D00B98000625D101205FFA8BF5E8
:1060BC000B90012D4FF001000C90A3D023F0A4FD08
:1060CC00C0B2B0FBF5F101FB15000B90012098E775
:1060DC00002038601E4989F80140A9F8025009785F
:1060EC0008F83610F4B1E8B1114962000DB0BDE802
:1060FC00F04F23F0A5B94FF6FE770498069EDDF815
:10610C00148047800A4FB37CF47CB269B1890125B5
:10611C00581EB07470895FFA88F68DE8D00003952C
:10612C0010F032FD0DB0BDE8F08F00BFD8BA020000
:10613C0008780020A86D0020E3BA0200D1BA020052
:10614C003056002020450020D7BA0200503D0020D8
:10615C00DE2700202DE9F04F87B005462C200E4697
:10616C0023F0CCFE002844D0778B044623F074FB3C
:10617C000021E1840121874208BF02212170707B3C
:10618C00A0703169081A6060204618F0B9FC3178AB
:10619C00834F01F00301387B012908BF0520607093
:1061AC00C0B223F09DF94FF0FF316077A182217FBF
:1061BC00326908440A44317D3261081A3075E07046
:1061CC00A069013017D0207C032816D8DFE800F036
:1061DC0002170209062021466082284617F064F94E
:1061EC0010B3042021466082284607F027FD05469F
:1061FC001BE01025CFE0A32517E0A12515E000201A
:10620C00B3256082F87A80B997F8410001280CD147
:10621C00A07D4FF6FF7619F06DFF0025A082B042ED
:10622C0008BF6FF05E0500E000252078022807D13A
:10623C0004F1080622F05AFE0146304623F009FE0E
:10624C00280640F0A580574F3878013801281AD815
:10625C0094F8260010B994F82700A0B1A078E17842
:10626C00227F08441044043023F048FE58B1A17832
:10627C00E2780646207F114408446168021D3046CE
:10628C0023F0DEF800E0002620460EF00BFB05465E
:10629C003878012802D12DB9002575E0022873D178
:1062AC00002D71D0002E73D00DF1080800274FF08F
:1062BC00010B4FF4D00908F1080A94F8260018B91C
:1062CC0094F8270000285FD0A178E278207F114451
:1062DC0008443146021D606823F0B2F894F8260099
:1062EC0020B184F82670C4F8129007E094F82700C7
:1062FC0020B12D4884F82770C4F8120020460EF007
:10630C00D1FA10B10021054639E04046142123F0A2
:10631C00FFFC608A8DF819B0F0B9A08A40F2031125
:10632C00884216D0682817D16068C17B052929D10D
:10633C002A30FF21082222F0F1FC18B34FF0FF3075
:10634C006946CDE900001948006823F082FDFC2065
:10635C0000E0FF208DF81800504669460022002509
:10636C0013F0F0F901469DF8000038B10420142216
:10637C00434620F063F90321002500E003210329A3
:10638C009BD101E00221FAE716B1304623F0B4FDAF
:10639C00204623F0B1FDE8B207B0BDE8F08F00BF96
:1063AC00A86D00202426002000000301EC580020DA
:1063BC002DE9FC470446019007788A48C65D8A4857
:1063CC00F840ADF80260C00740F00A810D2F13D1E0
:1063DC00864D0DF10201A868D0F82824532090476F
:1063EC00BDF802104FF6FD70814214D8208990B18F
:1063FC004FF0000A25469CE00C2F0ED0072F13D02F
:10640C00052F0ED1A078012800F0EA80207C3044C2
:10641C0000F1240916E0A868BBE06068C08AC005DA
:10642C000AD44FF0000A09E0A07848B1A07D00EB37
:10643C00C00006EB800905E04FF0010AB14605E00B
:10644C0006F11B09ADF802904FF0000A484620F007
:10645C006FFF00B30546072F3CD120782870607879
:10646C006870A078A8700028E178E970D4F805105D
:10647C0069604FD0A07D0028287241D0A169002905
:10648C003ED000EBC00005F110068200304622F031
:10649C00D7FFEE6037E00C2F40F0A280254655F870
:1064AC00040F002800F09C8023F0A0F980464F4890
:1064BC008068D0F8541328468847484620F038FFA7
:1064CC000546404623F04DFC002D00F0898023F05A
:1064DC0055FB2EE023F052FB052F2AD105F11806AF
:1064EC0069682422304622F0ABFF69692A7C05F1E9
:1064FC003C006E6022F0A4FF68682430686118E0EC
:10650C0000202872E860A06998B123F0F5FC002007
:10651C00A0750DE01B2005F110061B2228723046D9
:10652C00A16922F08DFFEE60A06923F0E5FC00204C
:10653C00A0612F48016819B128468847002844D12A
:10654C000D2F2BD1606801788A0720D4294AC1F31A
:10655C008301927C91421AD140783F2817D894F845
:10656C003000022813D195F8470005F146011DF0C3
:10657C0045FE01984FF6FF72418E91421DD1406845
:10658C008079022819D3284619F01EFC40B317480D
:10659C008068D0F8541301A8884721E00C2F0CD147
:1065AC0060781A2809D0686838B1C08AC00704D04E
:1065BC00287C05F10F011DF021FEBAF1000F04D16A
:1065CC000D482946007818F0C9FD0C2F08D1019808
:1065DC0050F8041F21B105498968D1F85413DBE741
:1065EC00BDE8FC878EB8020019C206000C01002021
:1065FC0064270020A86D00209C7A002014F074F809
:10660C008848DFF824B2DFF824A2DFF82482894D11
:10661C00894E0027006818F013F8DBF800004FF0E3
:10662C00FF310CF001F823F0EAFA9AF802109AF80C
:10663C000420D8F800409AF806308AF802708AF8DC
:10664C0004708AF80670002918BF44F00404002A6C
:10665C0018BF44F08004002B18BF44F00204C8F8A3
:10666C00004023F0BAFBD8F80000010644BF20F02C
:10667C008000C8F80000287818F014FA002848D0D8
:10668C00DAF80C10044651B19AF80100012804D034
:10669C00022804D1204688473BE020468847204604
:1066AC0016F09CFEA8B304460C20B1462F4623F0EE
:1066BC0025FC80B1064623F0A2FA05462078B4608A
:1066CC0098B1304623F018FC606821F00FFD20468D
:1066DC0023F012FC16E0606821F008FD204623F040
:1066EC000BFC3D464E46002713E0D9F8000031461E
:1066FC0023F00EFAD8F8000040F01000C8F80000A3
:10670C0023F0E1FA28463C464E46002723F065FB71
:10671C002546D8F80000C10631D5306823F0F2F9CF
:10672C00F0B923F0B1F8D8B9A94623F068FA0446B9
:10673C00306823F0E1F978B10546806841884068FB
:10674C0017F04EFCA868406821F0D0FCA86823F034
:10675C00D3FB284623F0D0FB204623F03EFB4D46CE
:10676C00306823F0CFF930B1D8F8000020F01000D9
:10677C00C8F8000003E023F0A6FAD8F8000081075F
:10678C000FD508F001FE21F005FA20B123F09BFA99
:10679C00D8F8000005E0D8F8000020F00200C8F896
:1067AC000000010725D5706823F0A6F990B1DAF83E
:1067BC000810044641B19AF8000028B1022826D0EE
:1067CC00012804D1A0688847A0681AF0B3FD2046C0
:1067DC0023F092FB706823F095F930B1D8F80000E3
:1067EC0020F00800C8F8000003E023F06CFAD8F899
:1067FC00000041077FF511AF20F00400C8F800003D
:10680C00306823F07FF900287FF407AF02E0A0681E
:10681C008847DCE7D8F8000040F01000C8F800000A
:10682C005846F7E64C7A0020507A00204425002088
:10683C00547A0020BD7A0020302600202DE9F04F3C
:10684C0093B004461EF006FC08B1112006E1207F2F
:10685C004FF6FE75B8B183480078810041EA4010CC
:10686C0061882077FF2020F089FA002180B1E08A2E
:10687C0005F1010B012640F00400E082207F40F07E
:10688C000100207707E0002000264FF6FE7B08E091
:10689C0000264FF6FE7B74480078022838BF012191
:1068AC0088010490678838461DF040FA08B1002032
:1068BC00607694F81AA0BAF1000F04D16B4890F8E6
:1068CC0000A084F81AA094F90000C5B2B0F1FF3F03
:1068DC0007DDE07E40B966480178E1760131017050
:1068EC0002E005F003052570207EDFF88491012875
:1068FC0005D199F80B0010B90DB900202076DFF8FE
:10690C00688198F80000012831D899F80E008007AA
:10691C002DD5E6B1E08A410606D5BAF1010F03D1B7
:10692C0020F00400E08222E0A188E07E627DADF8D8
:10693C0022708DF82AA0ADF824108DF82B0006A833
:10694C0004F056FD00283FF480AF25780FE0384660
:10695C001DF0ECF958B1002DDCD0206900780A2824
:10696C0005D8012101FA00F010F4836FD2D14FF653
:10697C00FE7A012D07D120690078022803D1E08A24
:10698C0040F04000E082EEBBE08A10F0400039D1CC
:10699C0098F80000012835D899F80E00800731D5F9
:1069AC00049DA71D6188607E3A462B4613F020FBA0
:1069BC0028B100206076E08A40F02000E082387830
:1069CC0070B1618804F108001CF006FC83466088F5
:1069DC00834504BF00203870E08A40F04000E0821C
:1069EC002078012804D0A18860882A460FF084FC06
:1069FC00A18860882A460DF0ADF818B1E08A40F005
:106A0C002000E0820DF11701204605F07DFB0646C3
:106A1C001FFA8BF0504508BFB4F802B0EEB12078E5
:106A2C00617D94F82C50B9F816209DF81730079416
:106A3C008DF81800608DADF81A00E08A06ACCDE92F
:106A4C000254CDE900101FFA8BF130460BF070F9AF
:106A5C00102803D1304623F04FFA102013B0BDE8B4
:106A6C00F08F00BFC327002024260020CBBA0200E1
:106A7C00A86D00202DE9F04F99B012AF8A4604465C
:106A8C001C219346384623F043F9204639460CF036
:106A9C009BFA9DF855009DF85C10084307D09DF8B3
:106AAC00480041060CD560891DF040F930B140F228
:106ABC00351013F09CFD19B0BDE8F08F9DF848001F
:106ACC0000F00C0510F0200FC0F3401918BF042D76
:106ADC0021D1E08D9DF8483010F080010CD15A0680
:106AEC000AD59DF84920920706D143F0040202F022
:106AFC000C020C2A40F0CA804FF00008012213F05F
:106B0C0003031ED0012B46D0022BD4D1A08912A98D
:106B1C001AF098FECFE7A68922F09EFE864202D19B
:106B2C00E08D010609D4A68922F096FE864200F07B
:106B3C008B80E08D010600F18780000679D4A08956
:106B4C007BE0544EF37A012B02D1A379002B78D041
:106B5C000223A7898DF84430ADF83C7081BB042D1D
:106B6C0075D1207C4E4D8DF85E0028680028A2D08F
:106B7C0022F072FE87429ED1E08D217994F830206C
:106B8C002D684346CDE903028DE8020A0FA812A92D
:106B9C005246A8478FE7002918BF012152EA01008D
:106BAC0003D1A08912A914F0F8FCA0890797ADF8BD
:106BBC001800A0798DF81A0006A819F0ABF97AE73D
:106BCC00ADF8300016989DF84A109DF84B208DF8C2
:106BDC00203094F832300B9060898DF82310DDF85A
:106BEC004E108DF8222094F830208DF83830ADF806
:106BFC001800B08CCDF826109DF85C108DF837205D
:106C0C00ADF82400207CADF82A10A17C8DF8320060
:106C1C0020798DF834109DF85F108DF833009DF8B5
:106C2C005D008DF836108DF8350006A802F0E6F8F8
:106C3C0041E7A089ADF86200608912A91EF03EFB05
:106C4C0010B14FF49A7034E74FF0010941E71AB9CB
:106C5C0012A9384614F0A1FC10480078022809D17A
:106C6C000D480078012805D1204611F04DFB002875
:106C7C003FF421AFA07CE17CB28C53468DE8020A34
:106C8C00039012A80FA90EF075FF14E74FF001083E
:106C9C00002234E7A86D0020E527002024260020E0
:106CAC003C2400202DE9F04F95B0044680690DF18D
:106CBC0053020021002690F800A09C200BF07AFAD9
:106CCC007D480078012808D8002004211CF086FF9C
:106CDC0006469DF85300304400E00120C1B2002567
:106CEC008DF85300514540F28180A0EB0A005FFA09
:106CFC0080F90220B9F1020F28BF81461A2009FB46
:106D0C0000F023F0FBF80027002800F0C380079464
:106D1C0009A90496F6B28346D04600240590CDF816
:106D2C0018A004310891E0B2484566D25FFA88F0A9
:106D3C00B0425FD21FF06AFE002853D05F4905466F
:106D4C00888C393122F0D0FD4FF60270ABF8170069
:106D5C0028888DF82470ABF81200ADF82600A97ABB
:106D6C008BF8191009A812F079F901460BF10A00F9
:106D7C00012903D1089923F06CF803E04FF0FF319F
:106D8C0041600160287950B14C4991F838100131BB
:106D9C0002288BF8181015D80221012814E0474856
:106DAC00022190F838008BF81510298800290A4622
:106DBC0018BF01228BF8142018BF411E00208BF83D
:106DCC0018100BE0012103288BF8141003D18BF859
:106DDC001570012002E001208BF815008BF81600CD
:106DEC000BF11A0B08F1010801349CE74FF0000974
:106DFC0000274FE00498CAFA50F830480DAD4FF018
:106E0C00020AAE1C00F13907E0B248453ED25FFAE7
:106E1C0088F187202A460BF0CDF9BDF83E003946A3
:106E2C0022F062FD0BF10A00314623F012F8BDF896
:106E3C0034002149214B012208F10108ABF8120062
:106E4C000978022938BF022293F838308BF81520C4
:106E5C00A3F1010238BF4FF0FF3202294FF00001BD
:106E6C008BF8182038BF01218BF817A04900002897
:106E7C008BF8161018BF01209DF8461001348BF8C2
:106E8C0014008BF819100BF11A0BBDE7079CDDE908
:106E9C00057A0025607C9DF85330A11C0022CDE9B9
:106EAC0000A9CDE902750AF007FB17B1384623F0AB
:106EBC0023F815B0BDE8F08F24260020A86D002023
:106ECC002DE9F0478AB0DFF8C0810446D8F80000FD
:106EDC00416E02A88847DFF8B4A1DAF80800016C0B
:106EEC00096811B9D0F84C05804769480121017037
:106EFC00DAF80C00C068007830B9DAF80800002124
:106F0C00D0F858240120904722F033FE47680589B9
:106F1C003878C0F3401128460FF09AFADFF87491D4
:106F2C000790D9F8101019B122F023FE0C308847C5
:106F3C00D9F8080008B18047089057480078F0B19C
:106F4C00D9F82010B9B1884755490028554B0A4645
:106F5C0008BF023212781A708DF82420CA1C00283F
:106F6C0018BF4A1C10788DF825004C481978022956
:106F7C0008BF023000E0494801880131018016F059
:106F8C00C3F84A48484E0078F57350B122F0F1FD31
:106F9C00007D30B1284622F08FF81FF047FA002808
:106FAC006BD000253761758022F020FC0746758078
:106FBC00059524B1012C31D13D483E49C1613C4875
:106FCC003949027B437BC47D416045804D6002F0B2
:106FDC00F002027303F0F0020232427304F0F0028A
:106FEC000432C2754A7B22F00F02531C4B73DAF841
:106FFC0008301B6C1C6864682478A40608D52E4CD9
:10700C0042F002024C601B685B689B784A73A37366
:10701C002A4E7060707B00F0F00070732848D8F82E
:10702C0000100822274B0C6D00210068CDE90021CF
:10703C0002AA3146A0472449B0F1FF3F088007DD82
:10704C00224819490160224801780131017010E091
:10705C00D9F8004044B1DAF80800002100220023DE
:10706C00006C00680C30A047012041F2883114F00C
:10707C002DF9384622F075FE02E0E1200BF046FBBC
:10708C000AB0BDE8F08700BF347A00200C01002064
:10709C00B327002054B502002C250020AC7800202A
:1070AC00BE790020AA7A0020C0770020A0270020FB
:1070BC00B8750020006A180048780020742500205C
:1070CC00E4260020F59600008E7A00203025002062
:1070DC0029250020B0B5784C20780E2850D8DFE850
:1070EC0000F0E34F4F5E084F4F4F4F4F584F08087B
:1070FC00080073480078B0B1A078012830D1E0784E
:10710C000130E070C0B2032851D870484FF6FF71BF
:10711C00808C88424FD06C48012101704FF4417033
:10712C00A4F8010049E06C480021E17001700020D6
:10713C001CF0D8FF18B120780D38012862D86148AE
:10714C000078022803D10820012104F08DFB0520D2
:10715C0020F020FE42F21070BDE8B04020F0D2B911
:10716C0003282AD157480078022826D156480121F5
:10717C00017003200021A070544880F826101CE0F8
:10718C0015F05AFF554810210078BDE8B04016F0B4
:10719C00B7BF4A48008800F007000128A9D1484829
:1071AC000078F8B10020BDE8B0401AF06FBB484839
:1071BC000078012801D10020A07019F0FFFE20F00A
:1071CC00A9FC3E488078000703D542480078012886
:1071DC006AD1A078032867D108200121BDE8B0400E
:1071EC0004F042BB3D481021007816F089FF0020C6
:1071FC001CF078FF334D297810B361B32078012946
:10720C002AD036E0062020F0C5FD2C4CA0780007D3
:10721C0004D54FF40040012104F026FB29480078E6
:10722C00012809D8208800F00700022804D000208B
:10723C000021002222F0ACF8BDE8B04015F0FCBEF5
:10724C00022903D10820012104F00EFB052020F0B7
:10725C00A1FD0120A7E720780A280AD11748008849
:10726C0000F00700022813D01848082180F82610D7
:10727C000EE003280CD115F0DFFE19480078022827
:10728C0006D101201FF08EFD02200121FDF7B0FA7E
:10729C00062020F07FFD2878012805D807480088B3
:1072AC0000F00700022800D1B0BD00200021002210
:1072BC00BDE8B04022F06CB8D02600203E7900200A
:1072CC00BF7A002024260020A27A0020A86D00207E
:1072DC00977A0020CA270020AE2200209D7A002039
:1072EC000C7A00202DE9F04F93B01C9C08901D46A1
:1072FC0006928B4620461EF0A9FC074620461EF03F
:10730C008DFC00260790002F00F0E980002D18BF9F
:10731C0001256801BBF1000F00F140014FF0000B9B
:10732C0008BF69014FF6FE7503914FF00A0108BFC3
:10733C000821029109A90431019100F108010C30D6
:10734C0005910490207C834580F0C480380600F0C1
:10735C00C18004EBCB0898F81C00C00740F0B78044
:10736C0061480078012820D898F8160028B10F96AB
:10737C00CDE90D664FF0010A1FE0B8F8180022F0B5
:10738C008AFC90B1007940F0020003280DD198F8E6
:10739C001C004FF0000A40F0800088F81C00079891
:1073AC00000604D10020079091E04FF0010A98F8F4
:1073BC001600CDE90D660F96C0B14C49089CB8F883
:1073CC00180091F86810012908D1FF21ADF834009C
:1073DC00059841F2080988F81A1024E0A080681C6E
:1073EC004FF00C09ADF8340004981CE0B8F8180004
:1073FC00089CA84213D104208DF8240098F81D0095
:10740C00ADF8300009A818F0ADFD0198002100225C
:10741C000023A580ADF8345016F062FF01E0ADF802
:10742C003400DDE902908DF8360001208DF839002A
:10743C00207D8DF838000DA807F018FF9DF8480046
:10744C0078BB109806994176417DA0F8169088F883
:10745C001B1098F8161019B1244991F8681001778F
:10746C001C9A51890185518A4185117D80F82C1017
:10747C00517980F83A1098F81A1080F83B1021894D
:10748C00A0F84010617D80F8491062682169C263E0
:10749C00406C227D21F0D4FF0DA81BF0AFF89DF8B5
:1074AC00480098F81C1041F0010288F81C2020B10B
:1074BC0041F0090088F81C0005E007998AF00100EA
:1074CC00013F091A07911C9C4FF6FE7500260BF123
:1074DC00010B37E72046002117F070F906463046BD
:1074EC0013B0BDE8F08F00BF24260020A86D00204B
:1074FC00BFB581780446481E0B2812D8DFE800F08F
:10750C0006525C6A26788590A430B23900208DF83A
:10751C000400E0780F28C0F0B28002208DF804003F
:10752C00B3E0FF2940F0D3800025E01C04218DF846
:10753C0003501FF01DF96C4908606C48058011F070
:10754C00E1FE0DF103036F20FF21BDE000208DF85B
:10755C000800E07802F084FA02AB6F200521B3E05A
:10756C0020F058FC8DF80E000DF10E036F200A214F
:10757C00AAE000208DF80F00E01C22F0BBFC0546B1
:10758C00601D04211FF0F4F8014628460DF028F97F
:10759C00504A3520282122F091FA0DF10F036F206B
:1075AC000C2191E000208DF80600E0780F2870D3B4
:1075BC0002208DF8060072E0E07847490DF10703D0
:1075CC00002818BF01200870002003218DF8070047
:1075DC006F2079E0E2780020211D8DF80A0004F17B
:1075EC000C00022A68D0012A6AD117F017FF65E057
:1075FC0000208DF80C00E078002818BF012020F046
:10760C0081FF03AB6F2006215EE0E078211D19F0AD
:10761C0059FB8DF80D000DF10D036F20072153E080
:10762C000020E57804218DF80900201D1FF0A0F83A
:10763C00002D014618BF0125284621F01FFD0DF134
:10764C0009036F2008213FE000208DF80B00E07843
:10765C00002818BF012022F0E9F90DF10B036F206F
:10766C00092131E000208DF80500E07804281BD2B8
:10767C001B4A01211070512022F020FA17E0194A00
:10768C0001211070522022F019FA01AB6F20012158
:10769C001AE0124A01211070532022F00FFA0DF15A
:1076AC0006036F2002210FE002208DF805000DF17A
:1076BC0005036F200B2107E00BF09AF88DF80A00F8
:1076CC000DF10A036F20042101221BF057F8002052
:1076DC0004B0B0BD08750020BE270020D2270020C2
:1076EC00DC270020D8270020182500201425002096
:1076FC0070B590B00446807821F026FA002800F08E
:10770C00D38005466078A0F1E101E873102906D911
:10771C001A2818BFCD2808D01D2806D04BE001220E
:10772C0002FA01F16C4A1142F2D06C4E3078012809
:10773C0002D8688900056CD42846002108F072F93B
:10774C00C0B3307801282BD86548807B800727D5BB
:10775C002968086A20B3C97F03AA09F039FD60784B
:10776C00E92808D12868E27B01234189008800932D
:10777C00E92301F06FF92868BDF8161001809DF817
:10778C001120BDF81810BDF81600002A18BF0122F0
:10779C0092010CF0DFF918B1688940F02000688183
:1077AC006A896178288920F0C5FB28813078012806
:1077BC0031D971E060788DF81000A07B03958DF8BD
:1077CC001100287C00283ED003A811F0FDFF9DF885
:1077DC001030E92B00D03BB92868E27B01264189A7
:1077EC000088009601F036F93C480078012853D8FF
:1077FC003B48807B80074FD5687B022802D1688983
:10780C0040073BD46078E92846D128461BF0B6FAED
:10781C0042E0052068736078E9283DD03148006863
:10782C0000B18047304E3068B0B32D48807B800764
:10783C0032D52868418900881BF0F8FF60B3617865
:10784C003268904728E003A805F044FE23480078EE
:10785C0020B19DF81030012802D0BAE79DF8103005
:10786C00002BB6D1286800881CF060FA0028AED135
:10787C001C4800680028AAD08047A8E72868008820
:10788C001CF054FA002811BF032028684FF6FF7132
:10789C00018008BF05206873687B022804BF06209E
:1078AC006873A07812F064FD1FF055FC0B4800784B
:1078BC0002280ED10D48007858B900200DF10B01AB
:1078CC008DF80B0052201AF059FC2020012103F0F6
:1078DC00CBFF10B070BD00BF0101010024260020B9
:1078EC00A86D00207C23002080230020E5270020A9
:1078FC002DE9F04F8BB0002900F0EC80DDF858A09A
:10790C000746007A0D46994690465FEA0A718DF853
:10791C00060012D4387A02240F2800F2DC800121F0
:10792C00814011F00B0F19D003288DF8100024D1D1
:10793C0002A8394622F08DFA22E0022840F0CA80D3
:10794C003C8821F089FF8442E4D03888012103224D
:10795C0013F0CCFB0028DDD0CD24BCE048F20400B1
:10796C00014200F0B88038881CF0E0F9002800F0E3
:10797C00AD800F2038728DF810003888ADF80800F3
:10798C005FEA8A7014D40020ADF8180054480068DF
:10799C0088B14168A942FAD1826862B12978022083
:1079AC00904768B10188ADF8181022F0A5FA07E0ED
:1079BC004FF6FF7002E0A86810B14088ADF81800CF
:1079CC00CAF380121798DDE9141B8DF805209DF879
:1079DC001020531E18BF01230F3A18BF9A001AF03B
:1079EC00100318BF13464FFA8AF2002A0AF040021D
:1079FC0048BF43F0100343EA92125FEA4A73ADF8B2
:107A0C00202044BF42F04002ADF820208DF8240025
:107A1C000791ADF81A90ADF8168000229BF8000083
:107A2C007C7A7E895FEA8A618DF804202D498DF875
:107A3C00220028788DF81340ADF8146009788DF881
:107A4C00120048BF04218DF8231021F029F828B129
:107A5C00016919B102A888477C7A7E893046214693
:107A6C0021F09CFF28B121F019FA48450DD20224CF
:107A7C0013E001A821F0F8FA48450AD21A48016827
:107A8C000029F4D002A8884706E002A806F0C4FE3C
:107A9C0002E002A801F0B2F904469DF81000022899
:107AAC000CD1BDF8086021F0D7FE864206D19BF8B8
:107ABC0000102878424623461BF0C8FD5CB99BF8A1
:107ACC000000002401308BF8000004E0387A0F2805
:107ADC007FF42AAF022420460BB0BDE8F08F00BF24
:107AEC00247A0020E71D002000270020F8B57B4EEB
:107AFC000446B068D0F8B8100A78CAB18A6BBAB12B
:107B0C00896DA9B10DF1030142F21A009047B068DA
:107B1C00D0F8B800806D8047002738B19DF803007D
:107B2C0020B1A4F1E100B0FA80F04709B06800E0A0
:107B3C000027D0F8401400208847C07B012502287C
:107B4C0008BF0525B168086C0068002800F0C480E7
:107B5C00E92C12D01B2C03D06CB90021417077E0BA
:107B6C00027D052A05D0D1F8D41091F88210002995
:107B7C00F3D017B96BE0002F49D0F068816DF1207C
:107B8C008847B068016C09688A7E2AB1CB8A5B078A
:107B9C0020D4501E887633E0D0F83C058047B1687D
:107BAC000A6C126888B3D08A40072ED4D1F8D4005E
:107BBC0090F834009076D1F8D40090F82220531C21
:107BCC0080F82230086C006840688270F068016AA6
:107BDC00284664E00A7E02F07F020A76016C09688E
:107BEC000A7D032A5DD1CA8A22F00402CA82006C83
:107BFC000068817E01398176394801880131018024
:107C0C00F068D0F8AC008047F8BD547020E01C2C14
:107C1C004FD0E12C1BD1D1F83C058047B26801460E
:107C2C00106C006899B1C18A490710D4D2F8D410ED
:107C3C0091F834108176D2F8D40090F822104B1CB5
:107C4C0080F82230106C006840688170BEE7447088
:107C5C00B068D0F86C12006C00688847B068016C92
:107C6C000A68D28A120614D5D0F8B810097839B936
:107C7C00D0F8D400F16890F84300096B8847B068DD
:107C8C00D0F8D400F16890F94200496A8847B0688E
:107C9C00016C00200860B068D0F8281310208847C9
:107CAC00F8BDF068816DF0208847B068816C096878
:107CBC00D1E7096E09680029D0D08847B068002147
:107CCC00006C0160F068C068007828B9B0680021C9
:107CDC00D0F8582400209047F8BD00BF0C010020BC
:107CEC00822700202DE9F04788B004464FF0FF3082
:107CFC0002214FF6FE79CDE90200E089002808BF89
:107D0C000821A66916F801A030B1704835880088A2
:107D1C00854213D16E4E06E06D4831461FF017FEBA
:107D2C0090B36A4805884D4518BF002E29D1207B99
:107D3C00002840F0C8806848406843E065480078F7
:107D4C0001281CD8284621F0A6FFC0B101790026D5
:107D5C0001292DD140880DF110088DF81060ADF877
:107D6C001C00404618F0FEF80646002818BF08F123
:107D7C000406BAF1000F18BF4FF0FF3AD3E7002604
:107D8C0016E05548406825E05248007801280DD887
:107D9C00304621F0DDFF48B101790139012905D8C0
:107DAC00BAF1000F18BF4FF0FF3ABBE74FF6FE7564
:107DBC00207B002840F08780474840684D4518BF1D
:107DCC00002E07D1E1894FF0810881B100F8018BB9
:107DDC0002AE11E05FFA8AF1022902D24FF00008DC
:107DEC0007E0217B01296ED04FF0800801E009F1FA
:107DFC00010500F8018B0EB1314600E002A922F01A
:107E0C0028F80570064605803248007838B10B27F3
:107E1C0001284AD15FFA8AF0012804D045E05FFAC4
:107E2C008AF0012822D10B27B8F1000F3DD1274849
:107E3C00A9B20088814238D100250DF107008DF8D8
:107E4C00075016F049FD98B1E1890322002908BFBB
:107E5C000922A1698A5C9DF8071091420BD9891AF5
:107E6C000D238DF8071003EB410708E00B271CE0EE
:107E7C000C27B57019E000210D278DF80710F27052
:107E8C005200331DB17009060DD0815C03F8021B42
:107E9C0081180232497803F8011C9DF8071001394A
:107EAC008DF80710EFE722F027F8E2890A4D102031
:107EBC00A11CFBB2A87004F1110042F4004217F0AF
:107ECC0005FB0020A87008B0BDE8F0878879002079
:107EDC00E079002024260020882600202DE9F04F90
:107EEC008DB00746C08914468946073086B23046A5
:107EFC0010F09AFA0546FF280AD13046FAF760F9D5
:107F0C00B04205DA70480778002F08BF0527A3E0B8
:107F1C006D4E3078C0B91CB1022C15D1FF2D13D188
:107F2C00387A002203238DF81C00786800920690A2
:107F3C006648C188C07805AA02F058FB9DF8240059
:107F4C003874BDF82000B881DFF880B1002104231B
:107F5C009BF80340BBF806A00CAA204621F038FA87
:107F6C009DF830007E2805D120467C211CF0E4FCD5
:107F7C009DF830007C286BD1FD8905F107081AFAB1
:107F8C0088F0B0F5005F65D8BB88C5F38512049006
:107F9C00F88849461FFA88F94FEA850C8DF82DC0F0
:107FAC0042EA83128DF82A00C0F301208DF82C20B0
:107FBC009A088DF82B203A7A05EB0A07B9F10D0FC8
:107FCC0040EA82008DF829004AD23F482A460197A0
:107FDC00CDF80CC000F11C06304621F0B5FFDDF8E1
:107FEC002900711900220027029170519DF82D0073
:107FFC000871681D81B2304621F04CFCDDF8291067
:10800C0032464B46715196212F4D8DF82F10039906
:10801C0021F015FB02998DF82E000B98C1F8030086
:10802C00204651461BF062FF04EB4401049A287071
:10803C000BEB81018A83BBF806104144ABF80610A8
:10804C0050B1019881B2204618F002FC2F7803E061
:10805C00012700E00527377038460DB0BDE8F08FDA
:10806C00894608462946002221F014FC0DF129010D
:10807C00052220F063FA96214A462B468DF82F10E4
:10808C009DF82D1021F0DBFA51468DF82E0020467C
:10809C001BF02CFF3070B9B220460DF129020723DA
:1080AC001BF024FF317851EA00073770D4D104EB70
:1080BC004400049900270BEB80008183BBF8060079
:1080CC004044ABF80600C7E7A0230020B87200209C
:1080DC002DE9F04F8BB0876904463D88B7F80290C4
:1080EC0028461BF023FE01280DD1207C617C002248
:1080FC008023CDE90052CDE90220A21C48F20600F3
:10810C0017F034F9D1E028461BF010FE20B969486D
:10811C000088854240F0C4803E7905375EB170001E
:10812C0021F0ECFE38B10246304639460A9221F075
:10813C0079F8074602E0002000260A9017F8015B48
:10814C0055B1680021F0DAFE30B182462846394636
:10815C00524621F067F802E04FF0000A0025A819FA
:10816C001421564F01EB4000C0B2079068000690F6
:10817C0070000590A01C0890002009903F68002F0B
:10818C006AD0786801780029F8D0BA7BD207F5D08C
:10819C00D7F80880B8F1000F03D00120C047834600
:1081AC0001E0D0F808B0BBF1000FE7D0BBF802003B
:1081BC00814503D04FF6FF70814511D1DBF80830B3
:1081CC009BF807200A9930461DF041FE78B9DBF880
:1081DC0010309BF80C20284651461DF038FE30B963
:1081EC00B8F1000FCAD0584621F086FEC6E70798B2
:1081FC001FF09EF838B30146D220087008980491FD
:10820C0000880D730E7148803EB101F11400059A7F
:10821C0088600A9921F014F901E00020886055B1BA
:10822C000499069A01EB460014300861514621F07E
:10823C0007F9049902E00499002008617868406805
:10824C00007816F08BFF099B9BF800001C4AD9B2F2
:10825C00013350540993C3E7099B0A9D180610D0AB
:10826C001448DBB2227C617C0088CDE90003144801
:10827C000023CDE9020248F20600089A17F076F8BE
:10828C0001E0207BA0B115B1284621F035FEBAF1F2
:10829C00000F0AD050460BB0BDE8F04F21F02CBEB9
:1082AC000548007802283FF420AF0BB0BDE8F08FF2
:1082BC000023D5E78879002024260020247A00208A
:1082CC002C7300202DE9FC47D0E900588246D8F8E1
:1082DC000000D0F8409019F4F06FC0F8449035D0FD
:1082EC005FEA495117D5D5E91401411A50461DF0E2
:1082FC003DFFD8F800008169C90605D401688DF8E6
:10830C0007109DF80710F6E7296801312960A97B51
:10831C0009B90121A973696C40684FF0004600F05F
:10832C000F0404EA0100B0FA80F126FA01F10140D1
:10833C0005D02F6C1FB12A68AB6C5046B847B4FA05
:10834C0084F026FA00F020404042A863D5F858018A
:10835C00D8F83C1009F0400740680068D0F80425B4
:10836C001140394347D0DAE90064504614F030FE2E
:10837C00D7B1F07C90B90BE0316F69B10068B16E88
:10838C00B26F8854306FB16F01310138B16730670B
:10839C0020688169C906EFD5F07C28B1D6E91401B3
:1083AC00411A50461DF0E2FE96F86400E0B13079B7
:1083BC00022819D017B1B179012901D0316F99B9BF
:1083CC000024B16E0128346786F86440B46607D186
:1083DC00B36CB26FD6F8CC6050460094B04703E053
:1083EC0006F17C0021F09CFD504609F0C9FAD5F845
:1083FC0058014068006800F204500068D8F8381042
:10840C00084228D0D5F8F80028B3DAE900765046AF
:10841C0011F02EFE50460CF0E1FC7879012812D1B7
:10842C00D7F8F40078B997F8E80060B1002087F825
:10843C00E800BB6CD7F8EC10D7F8FC20D7F850410B
:10844C0000905046A047D7F8F80020B93068816BEF
:10845C0041F4006181635FEA095023D5D8F800002C
:10846C0081690907FCD4016B21F480710163297ABD
:10847C0091B10020287295F84400800606D52C6C2A
:10848C0024B1AB6C504620210022A047504601215C
:10849C001EF098F9D8F80000816B21F4006181631B
:1084AC00687908B1BDE8FC8705F58070BDE8FC472C
:1084BC0021F036BD2DE9FE4F1D4614460F46814670
:1084CC0021F094F9DFF8C0A183464FF6FD78DAE984
:1084DC000010494518BF084660B1B83021F0E4FCE3
:1084EC0040B19AF82400CAF8209040F004008AF8B1
:1084FC0024009FE01FF0DEFB002868D0064663488E
:10850C00CDF808B0DDE90CB821F025FC604908F085
:10851C00200EB1F8540001306FF31F30A1F8540055
:10852C00B5605C480025C6E903792268D4F80C8054
:10853C0086F83250C6E908550BEA000C207C7263B1
:10854C002279C6E906CEC6F8408086F8440086F843
:10855C003820B1F8541086F83350D4E905533186DD
:10856C00A168C6E91253F163A18BA6F8501028B983
:10857C00B8F1000F1CBF012086F844004AB9387BC3
:10858C0000F00F00022804D1012086F83800B868EA
:10859C007063DDF808B00822FF2353FA82F23C46E0
:1085AC00D0B2851A18BF01257F680FB1002DF4D108
:1085BC00208800F47C40B0F5305F0BD196F8330086
:1085CC000022082340F0100086F8330004E008F184
:1085DC0001082FE0002202234CEA03004EEA0201BC
:1085EC002B4DC6E90601DAF82000484507D19AF868
:1085FC002400C1071CBF00F0FE008AF824002648A6
:10860C00046854B1A96CEA6C05F1400005F138031B
:10861C0000903046A047033013D1FD209AF8241067
:10862C00CAF820904FFA80F841F004018AF824101F
:10863C0020F0E6FE584621F094FB0FFA88F0BDE8D6
:10864C00FE8FB6F83080B5F85410414501D020F0BB
:10865C00D7FEC0B2012801D8FE20DFE7002089F840
:10866C00FC0096F8330040F0800086F83300A86BCD
:10867C00B04205D0F068007B00F00F000228D9D181
:10868C0015F0A2F8D6E700BF70200020387100204A
:10869C0030210020FFEFFF9F902600202DE9FF41A5
:1086AC00DFF8BC81002003900290D8F83840B4B3B6
:1086BC00D8F84C0010B9D8F8480070B3D8F8480076
:1086CC0060B12069D8F848100969814206D194F844
:1086DC003300C00602D5D8F84C0090B1002702A890
:1086EC0087F0010103AA10F085FD0546FFB9F5B12D
:1086FC000299002900F09D805A4820F065F9002766
:10870C0014E0D8F84800C06840880028F9D0D8F8A0
:10871C004800C06840880128F3D00127DFE75248A1
:10872C000221283021F000FC0027002500242CB366
:10873C004E48466816B30298B0FA80F040092840BB
:10874C0001281BD1D8F84800D8F84C10039A87F0B0
:10875C000103CDE9003208F1380208F14003B047BB
:10876C00012868D0022809D1D8F848000122012339
:10877C000069D8F84810B1F9301065E0002C20469B
:10878C0018BF01203840012851D13948216940686F
:10879C00814203D034484FF4806145E002980028B0
:1087AC0018BF01202840012806D1D8F8480018B974
:1087BC00D8F84C0000284DD008201FF0C3FD94F8C9
:1087CC0033004C25C00608F1380058BF48251FF06F
:1087DC0047F848F80500274BD4E90601C2439A60D4
:1087EC00DA681043D860C8431860586808432146BB
:1087FC0058600820E5681FF07DFA28461FF0AAF99A
:10880C00288843F60601411A022906D3B0F5C15F48
:10881C0003D040F60201884203D1012029461FF003
:10882C0069FA11484FF08041283021F07DFBBDE8FA
:10883C00FF8100277BE70398002818BF044601221C
:10884C000023B4F9301020690092002205F0BEF824
:10885C00BDE8FF8108201CF00BF9BDE8FF8100BFCB
:10886C00302100207C7100207020002090260020F8
:10887C00D01E0020081004402DE9F0478AB0684D46
:10888C002868416E02A88847664FF87918B1B87904
:10889C0008B10020C0E020F0A9FFDFF88CA18046D1
:1088AC0000249AF8000080074FF0000005D47D20CA
:1088BC0000210DF0CDFD8DF818408DF80C40029480
:1088CC005A4C0790616911B19AF800008847E0682A
:1088DC0008B180470890387A98B1606A88B18047AF
:1088EC005349544B8A1D002818BF0A1D12781A7060
:1088FC008DF82420CA1D002818BF4A1D10788DF849
:10890C0025004D4EDFF8349100200590317BF27E2E
:10891C00B0607080D9F8080001F0700180313173BB
:10892C0002F08001D0F82824F4206331F176032181
:10893C008DF8181006F11C019047387980B99AF817
:10894C00000080060CD52868C06B8047317BB06076
:10895C00029001F0F0010231317301218DF80C10FD
:10896C0029683748344E384B0D6D4FF080710068D4
:10897C0001913449009102AA3146A8470546334873
:10898C00B5F1FF3F058035DDB879002100240130B9
:10899C00B871787901307871FE60F8790130F8712E
:1089AC00022012F093FC3C712948D9F80820018868
:1089BC00D2F8AC30D2F8D4201C7841EAC411D48C53
:1089CC000180D2E9117193F800C0538D7486C48173
:1089DC00C0F80710C0F803708381508DC6E90A7186
:1089EC000CF001013086308B20F0800040EAC11081
:1089FC00308309E0626812B1002000219047022008
:108A0C0041F2883112F062FC404621F0AAF90020B4
:108A1C00B5F1FF3FC8BF01200AB0BDE8F08700BF29
:108A2C00347A002024250020B17A002054B50200AD
:108A3C00BE790020A97A0020007200200C010020D1
:108A4C00E426002020004300E90F01008C7A00206E
:108A5C00007900202DE9F843994617460C468046CC
:108A6C001AF0E4FE089D06463DB936B9404621464B
:108A7C003A46BDE8F84318F07BBA6EB3002D3ED0F1
:108A8C00624C207808B1012803D16148806800B19C
:108A9C008047B9F1000F4BD02078012800F2A58057
:108AAC005C48807B800740D55948C26812B130467B
:108ABC0049469047584831780078884224BF0131A4
:108ACC0031700024C9B2814230D1404619F056FFB2
:108ADC007470012701242EE04C4800240127B9F1C1
:108AEC00000F007829D0012D27D1012825D849481D
:108AFC00807B800719D5404619F040FF15E0B0780F
:108B0C00B9F1000F0AD1C1194808022938BF012058
:108B1C007178B07011B94149097871704049097880
:108B2C00884202D90027002405E00024012702E036
:108B3C0000270024377035480078012D08BF022823
:108B4C002BD084F001010F424DD1012812D83148AD
:108B5C00807B80070ED5404621F09DF850B11FB99F
:108B6C00417901F0FE014171ECB3417941F0010111
:108B7C00417100E0BCB3254C2078012821D8254850
:108B8C00807B80071DD540461FF046FEC8B10020F3
:108B9C004146BDE8F84321F0A7B9A9F11901022912
:108BAC00CFD3B9F1000F08D0B9F1E10F18BFB9F16B
:108BBC00F10FC6D0B9F1EB0F1AD1154900220A708A
:108BCC00BFE71448408B40450DD10120414621F0B0
:108BDC008BF92078022806D14FF400500121BDE812
:108BEC00F84302F041BEBDE8F88300240127A4E756
:108BFC00074A0C49137809780133DDB28D4228BF3E
:108C0C000023137028BF01249BE700BF24260020FB
:108C1C0074230020A86D0020CDBA0200CCBA02004B
:108C2C00A3270020D62700202DE9FE4FD0F8008086
:108C3C00994614460E46824613B10020C9F800002E
:108C4C0020F0D4FD834698F8070038B198F86400FA
:108C5C0048B121F09BF86FF00805B4E021F096F8CC
:108C6C006FF00E05AFE0002C4AD0504614F0B0F96E
:108C7C0000200121C8E91A64C8F87040C8F87800CF
:108C8C00C8F8380088F80C0088F80A00504688F8B4
:108C9C0064101BF0EFF9504608F072FE08F14C041A
:108CAC0002AD204629461EF0FDFDD8F87810D8F804
:108CBC0070707218B84238BF0746029910463A468F
:108CCC0021F042F9204639461DF093F8D8F870008F
:108CDC00D8F87810C21B3944012FC8F87020C8F896
:108CEC00781001DBB842DCD198F8041002290CD1C1
:108CFC000020C8F8680088F86400C8F870001CE010
:108D0C0021F044F86FF009055DE0B84215D1002060
:108D1C00D8F86860012988F86400C8F868000CD19C
:108D2C000124584688F8104021F01BF898F80F00E1
:108D3C0000284BD020F05AFD834621F027F898F8F4
:108D4C00040008B100252FE0D8F8701008F17C0061
:108D5C0031B30C9920F06CFF10B1012088F80C0095
:108D6C0020F044FD0446504614F032F90020C8F8B7
:108D7C006800C8F8700088F86400504608F000FEDF
:108D8C0098F80A6098F80C50204620F0EAFF002D65
:108D9C0018BF6FF00C05002E18BF6FF00D0503E027
:108DAC000021002520F044FF20F020FDB9F1000F38
:108DBC0007D098F8041001291CBFD8F87810C9F80E
:108DCC00001020F0CEFF2846BDE8FE8F002598F855
:108DDC0010000028AED020F009FDA8F80F4020F0BC
:108DEC00C0FFD8F84830D8F87820D8F8CC70504666
:108DFC0031460095B84788F80F50E8E7F0B587B0D2
:108E0C0004466F48007878B1228B0020E57A012166
:108E1C000390CDE901008DF80910500706D402F03B
:108E2C0008030121002008E0BA20ABE0402012F03A
:108E3C0008038DF8060008BF0321402606EA8206C7
:108E4C004BB1C02093068DF806004FF0010358BFBC
:108E5C0002238DF80730530903EA121202F00802BC
:108E6C00324342EA0106217A03290AD8DFE801F0ED
:108E7C000215112640F0040720F0EEFC8DF8067068
:108E8C0008E00F291ED140F0080046F004068DF8CA
:108E9C0006002088ADF8040014E04A4991F86810E7
:108EAC00002900F08180278840F0080006F58056E4
:108EBC00FF258DF80600ADF8047004E001A92046EA
:108ECC001CF014FA0027208BC0070ED09DF806006A
:108EDC0010F00C0F58D09DF8060000F00C0104297E
:108EEC0004BF40F020008DF80600A07C8DF808002F
:108EFC0001A806F0BBF99DF81800002842D104988F
:108F0C00C682B4F81B10A0F81910217A012903D1DC
:108F1C002C4991F868100177A17EE37F0185228BA3
:108F2C0080F82C301306428508D5D20506D5417D34
:108F3C0094F820001DF0D9FCA17E0498878780F856
:108F4C003B5080F84A10A17A80F83A10D4F80E10F1
:108F5C00C0F83E10A17F80F84B10617F80F849105B
:108F6C00406C6169628A20F06BFA208B400604D554
:108F7C001548016809B101A8884701A819F03EFB02
:108F8C009DF8180007B0F0BD208816F0CDFD48B153
:108F9C009DF8060040F020008DF80600208BC007DD
:108FAC0099D1A2E7BB20EDE727884FF6FD7140F081
:108FBC000C0046F00406ADF804108DF8060082E7AC
:108FCC002C240020A86D00206C2700202DE9F04FE8
:108FDC0089B0714F14460A46064610460492B98C65
:108FEC001AF024FC054610B16878002866D0B06AE7
:108FFC004FF00E09B34690F80180867890F805A0E2
:10900C005FEA886158BF4FF00609B0F8030003907F
:10901C0004981AF0DBFF18F0870F4CD108F01801F8
:10902C00182948D09BF81C10894544D100EB0A0242
:10903C000021BBF80C00B1460091D1B292460E460D
:10904C00049B494632460EF0B5FC032836D008F096
:10905C007801B8BB18F0180F62D05FEAC860884678
:10906C004FF0030058BF012040EA0108BBF80C0088
:10907C00414610F07DFF88B1817911F0180F0DD0A9
:10908C00417901290AD14DB1B98C40881AF0CEFB37
:10909C0020B1407810B1697888420FD320F0C1FA22
:1090AC0088B94FF0FF3020809BF8080000286BD067
:1090BC00DBF8181069E0D32011F099FA002009B000
:1090CC00BDE8F08F884620884FF6FF718842F5D1B5
:1090DC000121BBF80C00324600914946049B0EF06E
:1090EC0069FC0398414685B2284618F0FBF9F98AC9
:1090FC0088420CD1284620F0CEFD20B300790138EF
:10910C00012820D805A928461CF000FE21E0DBF838
:10911C00280080F805A009B0BDE8F04F1EF0CABCCD
:10912C00787B884608B120F07CFA03984FF6FE71E4
:10913C000022434680B203F0E1FF0028C3D14FF672
:10914C00FF702080C4E71FF0D1FE014605A820F077
:10915C0080FE9BF80800012804D1DBF8181007A842
:10916C0020F077FEDBF82810BBF80C00497805AA34
:10917C0007ABCDE9003200224B4641F030010291A1
:10918C00294608F0BDFE99E70021BBF80C003246D9
:10919C0020F098FE97E700BFA86D002070B58AB04C
:1091AC0000F11605044628461BF00CF867480078B9
:1091BC00013801282BD800201021012214238DF80E
:1091CC00110005AE0DF11100CDE90210CDE90062E0
:1091DC000DF11201042000221BF098F950B15C48EB
:1091EC00006804A905AE324610F0ACFAC728ADF8F9
:1091FC0012000CD806F108002946082220F020F9AC
:10920C00BDF812100420142233461DF017FA28461C
:10921C00FF2108221FF082FD10B14E480121017080
:10922C0028461BF0DBFC20790138052800F28B80E6
:10923C00DFE800F00389345C8903A01D00211029AC
:10924C0013D0425C0131002AF9D061791EF036F955
:10925C004348424D90F8410008B12878D8B1607964
:10926C000DF0CAFE0020287015E03D4890F8410032
:10927C0088B905AC002062210025224610F030FC94
:10928C00204600211EF01AF900200DF0B5FECDE9A4
:10929C000755CDE905551FF0EFF854E00DF112011B
:1092AC0028461DF0B9FA60B10DF112024FF6FE70AE
:1092BC0029461CF0DFFF284600210022002315F070
:1092CC000FF8BDF8126005A930461CF027FB059875
:1092DC0028B905A81AF07EF908B905980680A11DD1
:1092EC00284610F005FD13F0FFFC2CE01A4E3078E8
:1092FC0048B30DF1120105AA284610F023FA0146D5
:10930C009DF81200F8B1002501201422ADF82400BC
:10931C0006958DF82650059505AB04201DF08EF9A9
:10932C0006344FF481701021224620F0C1FB28B97D
:10933C004FF481701021224620F0C0FB0120032144
:10934C00357018F0C7FA0AB070BD00BF2426002093
:10935C00EC580020A07A0020B0220020AF22002080
:10936C00A86D00202DE9FE4FD0E90198D8F8001027
:10937C00CA690A62D20740F0AF80D8E904014FF005
:10938C00000A4FF0000B0843D9F8CC104968096863
:10939C00C1F8040509F13000029009F1C8000190F0
:1093AC00BBF1010F00F2A180D9F8C000002800F039
:1093BC009C80D9F8E010DC22D9F8CC70202300294D
:1093CC0008BFD82208BF182358F803404FF02403D5
:1093DC0008BF1C237F68D8F8146058F803303F6826
:1093EC00D7F80455354211D0A46864070ED104682F
:1093FC00D9F8D050A54209D144693CB9D8F80040FD
:10940C00656A25F002056562C7F804659B685B0711
:10941C0002D00BF1010BC3E759F80230002BF8D046
:10942C0049F802A0B1FA81F1D9E93442490900683E
:10943C0049011A448442C9F8D420C9F8E01028BF65
:10944C0082420CD24846414602F0F6FC99F8FE00E6
:10945C000028DED01FF05EFD18BF8862D9E720F02F
:10946C00C5F9D9F8C820D9F8C010019B81F810A013
:10947C0022B113465269002AFBD114331960C9F882
:10948C00D4A04A69C1F814A0D9F8E01000294FF013
:10949C00DC01C9F8C02008BFD82159F80110C9F85F
:1094AC00D01020F05EFCD9F8C00058B148464146B7
:1094BC0002F0C2FC99F8FE0050B11FF02BFD18BF52
:1094CC00886205E0D8F80000416A21F0030141628E
:1094DC00029820F02BFD9CE7D9F8C0203AB103216B
:1094EC001174BDE8FE4F0EF0E7BFBDE8FE8F486873
:1094FC0020F002004860486A20F003004862D8E976
:10950C0004021043D9F8CC2052681268D062C2F819
:10951C000405486920F001004861012008624046BA
:10952C00BDE8FE4F1DF0F1BD70B58CB004460020B7
:10953C008DF82C00CDE906000890A078411E052975
:10954C0025D82220DFE801F00321212C23036248D7
:10955C00007820BB20F058FA40B9604DA168082271
:10956C0005F118001FF06CFF208828805C480078FB
:10957C00022814D1A0680DF1030101AA10F0E2F841
:10958C009DF8140038B1B1206CE01B2008E0B3202A
:10959C008DF82C0059E09DF803000028F3D023200F
:1095AC008DF81C000120A17B8DF81A0020888DF805
:1095BC001D102169ADF81800607B0891012804BFCB
:1095CC0021208DF81A0006A805F050FE9DF82C00FD
:1095DC00D8BB0998456C05202870A0786870A81C29
:1095EC00616819B110221FF02BFF04E00021C1604B
:1095FC00816041600160A078062801D0012803D168
:10960C00E078A874133500E01235A16828461FF0E5
:10961C00DEFFA17805F1080006290AD8012202FA1A
:10962C0001F111F0520F04D02E49096820F011FC01
:10963C0001E0217B017020881AF078FB10B10998A9
:10964C000421C1829DF82C0070B12348007838B9F0
:10965C0020F0DAF920B921480021C0E90611018077
:10966C009DF82C000CB070BDA078042814D1A06813
:10967C0001AD0DF103012A4610F064F806469DF881
:10968C00030018B94FF6FF708642DED0206968B12E
:10969C0006A80DF0C7FF0CE0206918B106A80DF064
:1096AC00C1FFD2E706A818F0A9FFCEE706A818F06C
:1096BC00A5FFA16805F1080008221FF0C1FE0120DA
:1096CC00314614222B46ADF814000020CDE90100E0
:1096DC0004201CF0B3FFB8E72426002050240020FF
:1096EC00BC270020EC580020F8B5634E01211D4624
:1096FC001446F068C0680170604800210170604831
:10970C000170B068016C096811B9D0F84C0580473C
:10971C005C48076847B15C4822462B464188B068D4
:10972C00006C00680C30B84715F0E24F14D0574865
:10973C000178013901705448406818B15448C18906
:10974C000131C181B068006C006840680078800607
:10975C006FD41AF02FF86FE020070CD44A484068F9
:10976C0018B14B48C1890131C18148480178013990
:10977C0001701D205EE0454C42F205422078013814
:10978C0020704448418841F00400904218D13E4872
:10979C00406818B13E48C2890132C2813C484289B6
:1097AC000132428142F20542E120914208BF1C2065
:1097BC0008F0ACFF207800284AD094F9000040E073
:1097CC00314842F606024188914212D0B1F5105F41
:1097DC0049D140693349086019F0B0FA2E48007835
:1097EC0050B32F480168013138BF0160002101815D
:1097FC0022E0406818B12648C1890131C181264850
:10980C000078C8B12548042100780228204808BFF8
:10981C000621425A0132425221484168013138BF77
:10982C0041600189428901318BB20181934288BF29
:10983C004181E92008F06AFF1448017841B190F9A0
:10984C00000000280ADCB068D0F84C05804705E021
:10985C00B0680021D0F8582400209047F06800210F
:10986C00C0680170F8BD406800283FF482AF08481A
:10987C00C1890131C1817CE70C0100202725002022
:10988C00B327002054B50200C07700202925002002
:10989C00AC780020B87500202C250020AA7A002076
:1098AC0064790020487A0020FEB504462C2020F074
:1098BC0025FB002820614BD02C2120F029FA2569AA
:1098CC0020884FF6FF760DF10301AE8211F0F2F90C
:1098DC0048B30DF1030069461EF01EFFBDF80020D1
:1098EC00B24220D0584902EB4200AA8206226A8278
:1098FC00002251F820302A744FF47A72AB6151F87F
:10990C0020300133B3FBF2F541F8203005FB123265
:10991C004AB901EB8000012101724C484FF40061FF
:10992C00007814F0EDFB21692088083111F0C2F9A0
:10993C001FF0CEFC256970B1022028744FF4D000C2
:10994C00C5F8120042480168A9610131016021E0AB
:10995C0010202075FEBDA88AB0421BD13D4F05F1E9
:10996C00080039681DF0F3FF58B93D681FF0BEFAC6
:10997C00014628461DF0EBFF18B91FF0A9FC002882
:10998C005FD02169208802F00DFB256900B1AE8201
:10999C0000202874A88AB04231D12F48C17A11BB5B
:1099AC0090F8410001281ED10DF10B02002001217D
:1099BC003A2301271EF03AFC08B1AE8213E09DF861
:1099CC000B002F74A8754FF46810C5F812002348CB
:1099DC0001684A1CA961026029B91C484FF4007146
:1099EC00007814F08DFB2569A88AB04207D1A1201C
:1099FC002075284620F080FA00202061FEBD287CCE
:109A0C00012801D10E210CE0A06808B10D2108E05D
:109A1C001FF05EFC0D2118B9A078C00708BF052106
:109A2C0025692977A1780C4801F00301007B0129F5
:109A3C0008BF05206870C0B21FF052FD216948773D
:109A4C00FEBD2569A6E700BF307500209D7A002079
:109A5C0008270020EC580020A86D002018250020B5
:109A6C00F0B587B0624C054694F82B0028B9614FCD
:109A7C000421387819F0A0FC30B35F48407808BB5B
:109A8C005E480078022803D194F82B00800619D484
:109A9C0094F82E0005F0C60668B1A8070BD594F80B
:109AAC002B00C00607D41EF04EFB04200121FAF750
:109ABC009FFE86F0020694F82B1006F03F00084338
:109ACC0084F82B0007B0F0BD94F82B0005F00606C7
:109ADC002178304384F82B0051B1E0B34648002183
:109AEC0001703878042107B0BDE8F04014F008BBD1
:109AFC00012004F12E0300210122207055201FF0BB
:109B0C0035FB94F82E0080B33C48007801380128CE
:109B1C0009D83B4D0021082228681FF0FFF810B926
:109B2C001FF0D6FB20B334480721017094F82B00AA
:109B3C000021304340F0100084F82B00002005F089
:109B4C0027F80028BED000201DF02CF9072000219A
:109B5C00FAF74EFEB6E728480721017007200021CE
:109B6C0007B0BDE8F040FAF743BE94F82B00B4E719
:109B7C0028680DF11B0101AA0FF0E4FD05462148F0
:109B8C0000780028CFD09DF81400FD28CBD00228F7
:109B9C00C9D01D480088854217D201AE1421304629
:109BAC0020F0B6F8FF202946142233468DF8140015
:109BBC0004201CF043FD154905EB4500002241F83B
:109BCC00202001EB800042724260002555200121CB
:109BDC0004F82E5F22461FF071FFFF20032119F0BD
:109BEC0051FF054804210570387814F089FA69E7AB
:109BFC00AC220020A37A00200C7A0020242600201E
:109C0C00EC580020BA270020C0BA0200F033002024
:109C1C002DE9F04788B00646109C0020DD099A46D5
:109C2C001746C3F3C308E060A06060602060E9B130
:109C3C00E9462146102248461FF002FC20463146D8
:109C4C0010221FF0FDFB484620F0A3F8002010283E
:109C5C0005D0315C225C514021540130F7E70AF108
:109C6C00800A1FFA8AF04FEA102901E04FEA1A29FC
:109C7C006E46280418D0304621461022013D1FF0B4
:109C8C00DFFB2046394610221FF0DAFB304620F06D
:109C9C0080F80020102805D0395C225C51402154FA
:109CAC000130F7E70744E4E7B8F1000F25D0684628
:109CBC00214610221FF0C4FBB8F10E0F40D3002533
:109CCC00204639464246E560A560656025601FF078
:109CDC00B7FB80202146102204F8080004AE304661
:109CEC001FF0AEFB684620F054F8102D48D0705D84
:109CFC00615D484060550135F7E76E4621461022FC
:109D0C0030461FF09DFB002780201FF04BFF2146A3
:109D1C001022C4F80170C4F80570C4F80970677398
:109D2C00207004AD28461FF08BFB304620F031F834
:109D3C00102F42D0E85DE15D4840E0550137F7E770
:109D4C000026204639464246A681A66066602660FB
:109D5C001FF076FB80202146102204F808001FF02B
:109D6C0021FF04AD28461FF06BFB684620F011F86C
:109D7C00102E22D0A85DA15D4840A0550136F7E712
:109D8C006F462146102238461FF05AFB00253046FC
:109D9C00214610221FF006FF25606560A560A58195
:109DAC001FF04EFB38461FF0F4FF102D05D0705DF0
:109DBC00615D484060550135F7E708B0BDE8F087B4
:109DCC002DE9F04F8BB0DFF8A0810446D8F80800DD
:109DDC00D0F80001807AC00020F090F8002809909B
:109DEC0000F0B6800DF1040A0AF103071FF0FEFC27
:109DFC004FF00009FF2600250090D8F80800EAB2C1
:109E0C00D0F80011CB7A9A422AD2D0F88824D020EC
:109E1C0051468DF80650ADF804409047F0B99DF8C6
:109E2C00100020B1012819D19DF80F1001E09DF808
:109E3C000B1099B100284FF0080008BF0420002136
:109E4C00814202D27E540131FAE707F80090D8F82B
:109E5C0008005146D0F89424D02090470135CCE727
:109E6C004FF6FF7701AE0DF1140A4FF0FF3B4FF0A8
:109E7C000009C9885FFA89F291426BD9ADF80620C6
:109E8C00D0F88824D1203146ADF80440904730B149
:109E9C00D8F8080009F10109D0F80011E9E7BDF87C
:109EAC000800B842F4D0ADF81400D8F808005146B8
:109EBC00D0F88824D4209047002841D10025D8F828
:109ECC000820D2F80001C1888D4216D2D2F888241D
:109EDC00D1203146ADF80650ADF80440904728B972
:109EEC00BDF81400BDF80810814201D00135E6E739
:109EFC00D8F80800D0F80001C1888D42C8D1CDE94E
:109F0C0007BB099AADF81A70ADF81870807AC100C9
:109F1C000020814214D0131808309B88A342F8D13A
:109F2C001118002241F8082C09990844514620F8D0
:109F3C00047CD8F80800D0F89424D4209047A7E7E4
:109F4C0000981FF00EFF09981FF0D6FF192008E0AB
:109F5C001A2006E000981FF004FF09981FF0CCFFB0
:109F6C0000200BB0BDE8F08F0C010020FEB50C46B4
:109F7C0014F036FFA00600F18280200400F1AF80BF
:109F8C00E00607D52E208DF8040060481FF0AFFEC8
:109F9C0001A88847E00707D025208DF804005B480E
:109FAC001FF0A5FE01A88847A00707D526208DF82D
:109FBC00040056481FF09BFE01A88847600707D590
:109FCC0027208DF8040051481FF091FE01A8884706
:109FDC00200707D529208DF804004C481FF087FE78
:109FEC0001A88847600607D52D20ADF80400474826
:109FFC001FF07DFE01A88847200607D53020ADF85C
:10A00C00040042481FF073FE01A88847E00507D5FD
:10A01C003520ADF804003D481FF069FE01A88847C3
:10A02C00200505D53720ADF8040001A81FF0D2FF9C
:10A03C00E00405D53820ADF8040001A81FF0CAFFD4
:10A04C00324CA068D0F898000068B0B11FF0CEFB7D
:10A05C00A168D1F898100A68029200220A601FF0D9
:10A06C0080FEA068D0F8981002984860A168D1F8DA
:10A07C0040138847A0681FF031FC0020FEBD234E22
:10A08C0002ADB068C06B04301DF006F800280290D9
:10A09C003FF473AF1FF0AAFBB168C96B0A7B013A9E
:10A0AC000A731FF05EFEB1680298D1F89810077819
:10A0BC0048608DF80470417839B1162F0BD1B06817
:10A0CC00D0F8541328468847DBE7B168D1F8401321
:10A0DC008847162FD5D0B0681FF000FCD1E70B4D88
:10A0EC00A868D0F89400007814F0DCFC00280290EA
:10A0FC003FF446AFA968D1F898104860A968D1F828
:10A10C0040138847A8681FF0E9FBE9E70C01002021
:10A11C002DE9F04706680446307B022812D196F8E8
:10A12C0023006568D6E904A79146884680B1B168DA
:10A13C0058481FF07DFD40B100206FF0010786F8F4
:10A14C00250055E06FF0060752E0012086F8260046
:10A15C00002052492246F0614F48C6F8008086F82C
:10A16C0021901EF0AFFD297827201EF043F85046B1
:10A17C003946062209F080FA58B196F8260098B3B1
:10A18C0044481FF0CDFE002086F8260086F82500F6
:10A19C002AE0434D434FD5F8800320F00200C5F868
:10A1AC00800396F82000042804D157F84C0C416920
:10A1BC00272088470220C5F8FC0238684168062031
:10A1CC008847C0B1402028608020286096F826007F
:10A1DC0038B130481FF0A4FE002086F8260086F81F
:10A1EC0025000020C5F8FC024FF0FF30F061F76944
:10A1FC003846BDE8F0870220BA461BF057FA002714
:10A20C00B9F1020F0AD0B9F1040F4FF0000006D0DB
:10A21C00B9F1060018BF0120800000E00020C5F84D
:10A22C004C010123D8F80C10D8E90102C5F85011E3
:10A23C00C5F8547186F82430DAF800301D690B46E5
:10A24C00A847256895F8200002281BD00428CFD1F8
:10A25C00DAF80000816915488847B0F1FF3FDCBF90
:10A26C004FF0FF30E8610020EF6985F8240095F885
:10A27C0021100339022928BF85F82500204619F042
:10A28C0059FCB5E708484FF0FF311FF0D1FCEF69DE
:10A29C00AEE700BF98700020CC76002079C7010093
:10A2AC0004440240FC010010E87000200100008012
:10A2BC002DE9F0415A4E04465A4DB068D0F8D410EE
:10A2CC0091F88380297819B1D0F84C058047B06893
:10A2DC00016C096811B9D0F84C058047524F012028
:10A2EC00062C3C7028701ED8DFE804F004042225EC
:10A2FC002B5140004E4800214170B068026CD0F8E0
:10A30C00D41010684B4AC08A40064FF04E0058BF1C
:10A31C002520085C107014BBC97801B3022828BF33
:10A32C00022010701BE0B068D0F84C0580472EE07E
:10A33C0018F0C4FC2BE03E480021417017F0C8FF18
:10A34C0025E03A4800213A4A0170B068006C006878
:10A35C0090F8691090F86A0051703649087008F04E
:10A36C00E3FFB068006C006888B940E0B068324A1E
:10A37C00006C016891F86D1011803049006890F8FC
:10A38C006E00002808BF0120087019F0DFFF284874
:10A39C000078A0B9B268106C016829B9D2F84C05E4
:10A3AC008047B068006C01684968254A097801F05B
:10A3BC002001117023490068406880780870387853
:10A3CC00062814D8012101FA00F010F04C0F0ED021
:10A3DC001FF00CFA0446387802280AD18320287022
:10A3EC0020461FF0BEFCBDE8F04118F067BDBDE88B
:10A3FC00F0811548017819B9144909780029EDD074
:10A40C000221B8F1010F297004D10078832808BF0C
:10A41C0015F0E0F82046BDE8F0411FF0A2BC00BFEB
:10A42C000C010020B87A0020BB7A0020B527002050
:10A43C002D260020B97A0020C6790020BA7A002097
:10A44C00C47A0020C57A0020B07A0020B37A0020AC
:10A45C002DE9F0438BB0DFF884810C4605460020D3
:10A46C008DF81300D8F80010002900F0AD80032DF2
:10A47C0018BF022D03D191F84200904208D15849DF
:10A48C0000201BF081FD3DB1012D03D185240BE093
:10A49C00002099E0032D0DD10121D8F80000032DE7
:10A4AC0080F8411003D114B18DF813400DE0002455
:10A4BC005DB91EE0022D07D1D8F800000CB10221C5
:10A4CC0000E0012180F841100024D8F8000090F839
:10A4DC004190B9F1010F0ED190F8431019B1013927
:10A4EC0080F8431005E090F8481011B1013980F85C
:10A4FC0048104FF0010990F8431049B1426C00F13B
:10A50C002E03074602EB41018A1E00F126010CE0E6
:10A51C0090F8481000295AD0C26C00F10E0300F1DB
:10A52C00200702EB41018A1E811D1E78158802222C
:10A53C008DF828201CBB17B32A4A127880F84220C9
:10A54C0003208DF81C007888ADF8200005AC20465F
:10A55C001FF07FFC7878BB7BCDE90054CDE902601D
:10A56C002120B9F1010F08BF2220BA1D08A911F052
:10A57C0025FE1D481A4900881BF006FD23E0418882
:10A58C000DF1130448F220020123ADF8201041789C
:10A59C00CDE9004108A917F0C5F8D8F8000090F8EB
:10A5AC00401002290DD1418C48F220020123ADF854
:10A5BC00201090F821102030CDE9004108A917F0A7
:10A5CC00B1F815F087FA01200BB0BDE8F0834FF617
:10A5DC00FF75FF2600210027A9E700BF44270020B4
:10A5EC00519C020088260020967000202DE9F04F27
:10A5FC0089B08246129803F0F00403F00F0B002888
:10A60C0018BF0120103C03920025B4FA84F46409AD
:10A61C002040D4880290107A92886FF39F2400F027
:10A62C003F0024036FF39F2244EA0060544C104413
:10A63C0000905248007804AEC2B2ABB2934280F0A4
:10A64C009580A27801355FFA8AF7974273D08AB267
:10A65C000195172A6DD3A1F10709384632461FFA26
:10A66C0089F421460FF084FF9DF81B8008F003004D
:10A67C00022826D1BBF1030F00F27D800398007AEB
:10A68C00DFE80BF0140205109DF8181007E09DF898
:10A69C001810884215D10398BDF81610C08888424E
:10A6AC0004D00EE00498009981420AD10298002847
:10A6BC0054D01298002183688289304615F048FFE7
:10A6CC0060B15FEA48701CD5BDF81E0084421CD9ED
:10A6DC00A9EB000188B21728BDD228E01298808817
:10A6EC00E0B3129BDA8819689B681A440B781578CA
:10A6FC009D42E6D1013802F1010201F10101F5D1CF
:10A70C002CE01F4C0120607104E03846214616F005
:10A71C009FF81B4C00200025F7F752FD1748E178F5
:10A72C0000780131B1FBF0F202FB101A03E0134880
:10A73C000078134C019D5FFA8AF1C2B251FA80F194
:10A74C00013991FBF2F303FB121A5FFA8AF149000B
:10A75C0051FA8AF104EB8101898B6DE7039D96E830
:10A76C001F001FC5002009B0BDE8F08F0399002021
:10A77C0088810A20F7E70420F5E700BF9B7A0020C8
:10A78C00B8720020B0B560480021604C016094F8AC
:10A79C003A01032812D002282ED0012840F0AF80B5
:10A7AC0094F8400111F090F8002084F840015948C9
:10A7BC00817B0220002908BF06209EE054480168D6
:10A7CC00B1F5C060C4F82C01B8BFC1F5C060D4F8B5
:10A7DC001011002900D5494288422ADDD4F8140111
:10A7EC001CF0CAFDD4F818011CF0D8FDD4F82801CF
:10A7FC001CF0F8FD01201DE0454805681EF040FEE8
:10A80C00C4F814011EF044FEC4F818011EF048FEF2
:10A81C00B5F5C061C4F82801C4F8101109D094F83A
:10A82C0030215AB1D4F81401D4F82021D4F82C11C9
:10A83C000AE0002084F8300106205EE0C4F8240110
:10A84C00D4E94502C4F82C110223C4F81C010029D8
:10A85C0001EB410148BF6FF001031944042391FB44
:10A86C00F3F111440029C4F820110FDD1F2931D355
:10A87C00D4F824212AB33E28A8BF3E200130292930
:10A88C00A8BF2921C4F81C010B3909E0D4F82421F4
:10A89C00032A09D111F1140FD8BF6FF01301153130
:10A8AC00C4F82011002113E00128D8BF0120013881
:10A8BC0011F10A0FD8BF6FF00901C4F81C010B315C
:10A8CC0003E03329A8BF33211539C4F82011032123
:10A8DC00C4F824111CF050FD01201CF071FDD4F8BB
:10A8EC0020011CF05BFDD4F824011CF07BFDA5F2CB
:10A8FC00FF510420032938BF0620C4F83C01BDE8F1
:10A90C00B04005F04FBC00BF3C500C40D81B0020A1
:10A91C0008400C4018B802002DE9FE4F074600789D
:10A92C009B468A46029200F00C000C2808D1B8888D
:10A93C00FE211AF0A1F9FE28019008BF012019E0B0
:10A94C0059480568B878FF2808D01EF009FE40B1B8
:10A95C00064600781EF0A4F8054603E02DB16E689B
:10A96C0000E00026FE2001900EE0FE2000250026CF
:10A97C00019009E01EF0F4FD002800F092800646DC
:10A98C0000781EF08DF80546002E00F08A80AA682B
:10A99C004AB13178022090474FF6FE7440B10488DA
:10A9AC001FF0AAFA04E0B0684FF6FE7400B14488B8
:10A9BC0039893078A14211D010B909B900200DE0C5
:10A9CC0028B14FF6FE72013292B2914206D0A1F537
:10A9DC0080714FF6013289B2914244D897F80290B7
:10A9EC00B870387DD7F810803030C0B21CF0A0FCA5
:10A9FC00B8B304461A20514620707868C4F8020097
:10AA0C00A01D1DF063FDBBF80100A4F817000C9805
:10AA1C003A7D397B84F820000E986175A284E06140
:10AA2C000D986076F878E073307820759BF800000C
:10AA3C00A075788BA08578896082029820820F9807
:10AA4C0084F82E0032B104F130004146A0621EF0B1
:10AA5C00F7FC01E00020A06270682146007814F039
:10AA6C007DFB87F80290387800F00C000C280DD094
:10AA7C00B8780026FF287FF487AF286800250026C9
:10AA8C0000283FF481AF466805467DE70199B888F8
:10AA9C00C9B21AF0F1F8FE280146019001D00198D4
:10AAAC0068E7BDE8FE8F00BF247A00202DE9FF4740
:10AABC00D0E901590E4604461EF098FE95F8FD109B
:10AACC0021B97169102901D8032906D81FF049F959
:10AADC000024204604B0BDE8F087012785F8FD70FE
:10AAEC001FF03FF900204E4A85F8FC00C5E9300004
:10AAFC00C5F8C80085F8FE003069C5F8E400706937
:10AB0C00C5F8E800307B85F8F9000028317885F825
:10AB1C00F8107168C5F8EC10B9F80E10A5F8F6101D
:10AB2C00317E52F8211085F8FA1008BF1027C5F8AD
:10AB3C00F07099F80C000BF0CDF8204616F00EF9D9
:10AB4C0099F83B00374985F8FB008A46D4E9018720
:10AB5C003A6B97F83A000DF01FFC7A6B98F8FB00F3
:10AB6C0051460DF019FC98F8F91097F838000129A6
:10AB7C0015D1FA6A51460DF00FFCBA6A97F83900F4
:10AB8C0046F202010DF008FC98F8FB0026491DF076
:10AB9C0023FB98F8FB0021461EF06CF90AE0BA6A18
:10ABAC0046F202010DF0F8FBFA6A97F839005146AB
:10ABBC000DF0F2FBE84640461EF0B2FB99F805009A
:10ABCC001A4A4346CDE90040284699F8041018F07B
:10ABDC00C7FA40461EF094FCD9F8080014494246C6
:10ABEC000094029005F1300019F037FD12F082FE4E
:10ABFC00104AC5F8CC0005F11C00042123461CF0BA
:10AC0C0003FC95F8F80008B1B06805E005F16C009C
:10AC1C0000211DF0AFF80848C5F8BC0059E700BF8B
:10AC2C00B8B7020002600020ED0E01007193000025
:10AC3C0045110200E19A0200259D02002DE9F84F12
:10AC4C000CF088FD5F4800254FF0000A0478A542FF
:10AC5C0011D2E8B21BF0DAFE58B1017941F00401CF
:10AC6C00042906D1807A1DF055F9002818BF0AF185
:10AC7C00010A0135EBE700271BF0B4FC0546002662
:10AC8C00F8B285420AD91AF0B1F928B1807C1DF0CE
:10AC9C0041F9002818BF01360137F1E706EB0A0924
:10ACAC005FEA096032D04FF47F7000EA89073846BA
:10ACBC001FF024F950B33946FF2280461EF0D2FF14
:10ACCC0000275FFA8AFA4FF0000BA7422AD25FFAEC
:10ACDC008BF0504526D2F8B21BF098FEA0B1064678
:10ACEC00007940F0040004280ED1B07A1DF012F95E
:10ACFC0050B10146727A30885FFA89F3009343466B
:10AD0C0015F00EF80BF1010B0137DEE74FF00008E0
:10AD1C004FF000092C48007BD8B11EF0E1FBC0F1CC
:10AD2C00540017E000245FFA89F7E0B28542F1D9AC
:10AD3C001AF05CF958B10646807C1DF0EBF830B186
:10AD4C000146727C30884346009714F0E9FF0134C9
:10AD5C00EBE76220C1B203224546B1FBF2FABAF12D
:10AD6C001F0F28BF4FF01F0AC0B25FFA89F72A469F
:10AD7C00002818BF0120410101F14004574588BF4C
:10AD8C00440128BF57462146384612F0F4FA0646CD
:10AD9C0014F0400040EA0601A7F1010008BFA9EB3E
:10ADAC000009C0B208BF05EB800500200029DBD0EC
:10ADBC00B8F1000F02D040461FF09EF83046BDE8B7
:10ADCC00F88F00BFE3BA0200A86D0020FEB5044660
:10ADDC005A480078A04213D908780D46012801D1B1
:10ADEC00686868B16878012801D1A86840B1544FEF
:10ADFC0057F834601EF0FAFCF17921B11EF0B1FF66
:10AE0C0000242046FEBD07EBC40401216768F171E4
:10AE1C001EF0A7FF002005F1040C7074F081B060E7
:10AE2C0030602988B180A98BC6E93D00C6E90E00C7
:10AE3C0086F86400B186297D2B69B1719CE80610F7
:10AE4C00C6F85021BCF1000FC6E910C34FF0FF3219
:10AE5C00C6F8CC10A969C6E93B203163A97F86F8F6
:10AE6C003610296AC6E91A00C6E91C00B16486F8D6
:10AE7C00E800C6F8580102D13249C6E9101097F81B
:10AE8C0040000AF027FFD7E9031206F14C001EF030
:10AE9C001FFBD7E9051206F1D0001EF019FB2A4959
:10AEAC0038680968C96888477A6C97F8240046F2B4
:10AEBC0002010DF071FA254DBA6C97F82000294665
:10AECC000DF06AFAF86901280CD1FA6C97F8280091
:10AEDC0029460DF061FA3A6D97F82C0046F2020102
:10AEEC000DF05AFA12F006FDC6F85801204605F08E
:10AEFC0079FD174A06F5AE70042123461CF084FA3E
:10AF0C006D4628461EF00CFA387A7968114A2B46A1
:10AF1C000094019006F1140018F022F906F17C005F
:10AF2C0000211CF027FF06F5807000211CF022FF89
:10AF3C003868D7E90C121060486062E7C6BA0200A4
:10AF4C002CBA0200C3730100D00100100260002073
:10AF5C00AD8F0200D18200002DE9F84F81460868C0
:10AF6C008B469046D9E90045476806895548E16803
:10AF7C001EF05EFE18B16FF00100BDE8F88F52486C
:10AF8C0052494FF0000A4A46C4F814B084F80980BC
:10AF9C00C4F804A084F802A01DF094FE29782720A0
:10AFAC001DF028F938463146062208F065FB40B101
:10AFBC0044481EF0B5FF4FF0FF3084F801A0BDE807
:10AFCC00F88F434F57F84C0C416927208847414E66
:10AFDC000220C6F8FC02386841680620884760B138
:10AFEC00402030608020306036481EF099FF0020F1
:10AFFC0060704FF0FF30BDE8F88F02201AF056FB5E
:10B00C003A68DBF810009BF82010D26990473A6838
:10B01C009BF820009BF821101368A8F10102B2FAEA
:10B02C0082F252099847DBE90610C6F8500100205D
:10B03C00C6F85401C6F8581159B13A68DBF8040047
:10B04C00002315690022A84738688169224801301D
:10B05C008847207A042804D057F84C0C0169272023
:10B06C0088473B68DBF81C10DBE902021C690B46C5
:10B07C00A047D9F8004001206070207A022815D032
:10B08C0004281BD13868144D816928468847B0F1D3
:10B09C00FF3FDCBF4FF0FF30606000206070A81CE9
:10B0AC00C6F88403484610F071FF04E00B484FF0DB
:10B0BC00FF311EF0BDFD6068BDE8F88F0020BDE8D3
:10B0CC00F88F00BF98700020CC76002051D401007E
:10B0DC00FC0100100444024001000080E8700020D4
:10B0EC00F0B587B05C4E0446306848B390F8401019
:10B0FC0001293FD1022180F840102030214612F066
:10B10C001DFE05463068C169436B90F83220007E05
:10B11C0016F078FAB5FA85F137684D09002887F8EA
:10B12C00430043D040001EF0E9FE37687864C8B392
:10B13C0097F843104A0049491EF082F9376835E008
:10B14C0050201EF0DBFE306050B3502105461EF03F
:10B15C00DFFD2846214612F0F1FD08B330680121CD
:10B16C0080F840103E483F49008807B0BDE8F040E9
:10B17C001AF00ABF02200DF10F0148F22002012340
:10B18C008DF8180088208DF80F006088ADF810003D
:10B19C006078CDE9001004A9204616F0C3FA49E006
:10B1AC0088201CE0882001258DF80F007B69BA7C73
:10B1BC00F96B97F8380016F025FA316881F84800D9
:10B1CC0058B140001EF09AFE3168C86430B191F855
:10B1DC0048104A0021491EF033F96DB386208DF8D2
:10B1EC000F0002200DF10F0548F2200201238DF80B
:10B1FC0018006088ADF810006078CDE9005004A903
:10B20C00204616F08FFA306890B190F84010022961
:10B21C000ED1418848F220020123ADF81010022112
:10B22C008DF818104178CDE9005104A916F07AFA7E
:10B23C0014F050FC07B0F0BD306890F8431019B909
:10B24C0090F848000028C9D000200021002207B047
:10B25C00BDE8F040FFF7FCB8442700202C73002019
:10B26C0096700020519C020070B5604D0446A86891
:10B27C004169497F002973D0D0F8D420B4F842102A
:10B28C00D28C91426CD1D0F86C1304F12800884711
:10B29C00002865D0A868002241694A77D0F8D410FC
:10B2AC0091F8291021B1E868816A02208847A868C2
:10B2BC00006F90F82B0018B1E868816A012088476C
:10B2CC00207CC00608D5E868816A10208847A868E9
:10B2DC00D0F8281380208847E868C16B2020884765
:10B2EC00A868D0F8FC14C068103088476268A86859
:10B2FC0013785278416902F00F064E76C2F30011B2
:10B30C004269917603F00F01426991771909D0F8DF
:10B31C00D42082F82C10D0F8D410426991F84F3018
:10B32C00927F0F2B05D09A4203D26668F67806B945
:10B33C001A464A730022C16881F83020D0F8D41024
:10B34C00497B0F290DD14169C97E022908D1D0F85A
:10B35C0064018047A868D0F86C01BDE870400047D4
:10B36C0070BDD0F80C2520469047A9684869C07E6E
:10B37C00022814D1C868D1F8FC148847AA684FF485
:10B38C007076D2F8D430D2E90301D2F8F0245B7B8A
:10B39C0031F8131006FA03F3591A9047A968D1F83B
:10B3AC00D400D1F8B431228990F82C10022098479F
:10B3BC00A968D1F8D400427B90F82C0090420FD0B1
:10B3CC004869D1F8FC148847A8684169D0F87C0119
:10B3DC008860A868D0F8F024406941699047A96852
:10B3EC00D1F828131020BDE8704008470C0100204C
:10B3FC002DE9F84F544B554D93F800B000235B45A5
:10B40C0004D2AC782CB108350133F8E74FF00009C1
:10B41C0097E04FF000095B4500F093804C4B009295
:10B42C004D4A4FF0000885F806901E1D494BB2F8A6
:10B43C0016A04FF6FE721F78012307B336F8044CA2
:10B44C008C4218BF544503D12436013F5B00F4E70E
:10B45C003478042C03D0012C06D0002CF4D109F143
:10B46C00010985F80690EFE702F1010CB0F80AE04B
:10B47C001FFA8CF4A64508BF48EA0308E4E7384CE9
:10B48C00DFF8D4E0354B2678BEF824700A33B6B119
:10B49C0033F80A4C8C4218BF944202D11C33013E43
:10B4AC00F5E71C88BC42F9D1DC79002CF6D01C7A6B
:10B4BC00002CF3D009F1010985F80690EEE7294933
:10B4CC005FFA89F309788B4284BFA9718946009A87
:10B4DC005FEA096102D0817C012901D1002102E0DF
:10B4EC009EF80210013129719EF801109EF8073068
:10B4FC00B8F1000F6A71E9708189C07CAB7029804A
:10B50C00E87111D0184D194BBBF1000F0CD01E78FF
:10B51C00284619462EB14B1C051DABF1010B96426A
:10B52C00F2D1C0F800800A70114C4021207817F03D
:10B53C0043FF20B92078402164221EF042FC4FF0DA
:10B54C0001094846BDE8F88FCEBA0200AA6800206F
:10B55C0020450020E3BA0200A86D002030560020E0
:10B56C00D1BA0200D4BA0200306D00205876002007
:10B57C009C7A0020F8B50446007D50B15A4994F9E4
:10B58C001800C968D1F880108847013004BFE82042
:10B59C00F8BD554EE27BB568D5F80011E86B09781B
:10B5AC000AB1807A00E0C07A81429CBFF120F8BDDC
:10B5BC00636A94F8392094F83810A08DD5F88C5221
:10B5CC00278C0097A84700285ED0054600202880CD
:10B5DC006868A28DA16A1EF0B7FC04F1300005F179
:10B5EC0084010CC80CC1028880788870B0680A800D
:10B5FC002146D0F8442505F1900090476089B36846
:10B60C00A5F89A00207B85F89C00607B85F89D004E
:10B61C00A27DD4F80E00D4F81210D3F84835984710
:10B62C00A5F89E00E07D85F8A000207E85F8A1009D
:10B63C0094F83C0085F86C00228CA5F8A8202AB35D
:10B64C00E169D5F8A4001EF07FFC1DF0E1FEB5F811
:10B65C00A800E8B1D5F8A400D0B16868411E6960B3
:10B66C00F82100F8011C6868411E6960002100F88F
:10B67C00011CB5F8A8006968091A6960A9652989CF
:10B68C0008440230288103E01A20F8BD1DF0C0FEEA
:10B69C00B5F89E10C8051DD594F83B20E8202AB1BA
:10B6AC0011F0040208BF11F0010100D0F8BDB1681F
:10B6BC00486ED1F8FC14884794F83B004FF47A712B
:10B6CC00B268484309490978B0FBF1F1506ED2F8E1
:10B6DC00F4249047B0682946D0F89400007813F011
:10B6EC003DFD0020F8BD00BF0C010020B47A002005
:10B6FC002DE9F84F0446B0F82490C17B008A1EF067
:10B70C004DF948B9A07B032806D009F1140A1FFA99
:10B71C008AF0F128C0F09E8009F11E0A1FFA8AF007
:10B72C00FB280AD309F110001EF0E8FB40B30646D3
:10B73C0010304FF01E0A706000E000264FF08208B7
:10B74C004FF0010B1FFA8AF01EF0D8FBB0B1074680
:10B75C00A078BBF1000F3870E07878702079B87061
:10B76C006079F8700ED0A07BA11D3871A07B0328E6
:10B77C0010D1781D08221DF063FE0FE0002E64D15D
:10B78C00BDE8F88FA079FD1D3871E0797871E07B08
:10B79C00B8710BE0087878714878B871E07B07F1E4
:10B7AC0010057873207CB873607CF873207D28704A
:10B7BC00607D6870A07DA870607EE870281DE169CE
:10B7CC001EF005FB0020BBF1000F28720FBF05F126
:10B7DC000A0B4FEA1920A87205F10B0B85F809909A
:10B7EC00CEB11F481F4D4FF47A72016831600F21A2
:10B7FC0006602878317308211EF0E6FA18B1287813
:10B80C00082112F07DFCE069A16A4A46B0607068BC
:10B81C001DF016FE05E0A16A58464A461DF010FEC2
:10B82C00CB4494F82C005FFA8AF241463B468BF8E5
:10B83C00000094F82D008BF8010094F82E008BF882
:10B84C000200442016F09AFF3E463046BDE8F84F01
:10B85C001EF052BB4FF0000B4FF08108002671E731
:10B86C00682600209A7A00207CB5594D594E4CF62A
:10B87C00C0722B78347883F0010384F002042343E4
:10B88C00554C08BF104000295349898C0CBF21EA44
:10B89C000000084301B2A084B1F1FF3F08DC012095
:10B8AC000DF103018DF80300522016F067FCA08CFB
:10B8BC0081046BD401B2B1F1FF3F2ADD010465D0E4
:10B8CC004FF0FF310191317802295FD1297800299D
:10B8DC005CD121682346013101A908BF0B46C20780
:10B8EC0008BF0B4622461D6852F8046FB54298BF3C
:10B8FC001A46050758BF1A46C30606D525461368CF
:10B90C0055F8086FB34288BF2A46830607D41346FE
:10B91C000CE080B2400439D504F110003EE023461F
:10B92C00156853F80C6FB54298BF1346420401D406
:10B93C001A4606E022461D6852F8106FB54298BFB1
:10B94C001A46C30401D4134606E02346156853F87F
:10B95C00146FB54298BF1346820701D41A4606E00D
:10B96C0022461D6852F8186FB54298BF1A46400718
:10B97C0001D4104606E02046136850F81C5FAB4219
:10B98C0098BF1046884218BF002807D1002001211B
:10B99C0020621248007814F01FF87CBD226A0168FE
:10B9AC0012B11268914211D00C4D206201292878F5
:10B9BC0003D1012112F0A4FB7CBD012114F00CF881
:10B9CC00216A28780A6801211EF0FBF97CBD00BFB2
:10B9DC00E527002024260020087500209C7A0020F2
:10B9EC00F8B5554F554E564D38883168EC8808449B
:10B9FC00224600F10801A868806D1EF0A5FAA9681E
:10BA0C003888504B8A6D2044388022448A653268CD
:10BA1C0081B20832565C811C398089B2515C197034
:10BA2C00C11C0730398089B2515838806846009162
:10BA3C0004211AF09DFE00901CF08EFDA968C863CD
:10BA4C0000981CF027FAA968A1F840003E4800783D
:10BA5C0018B11EF025FAA968C863EA2019F074F928
:10BA6C003A48426812B1A86801219047384802212F
:10BA7C00384C0170E0684069007830B1A87B8009CF
:10BA8C0017F08CFB08B10120A870A968A8780A7C73
:10BA9C00002870B218BF42F0040200270A7400217B
:10BAAC001AF0F9FE0146A86880F8461000F17401FE
:10BABC00B0F85C2080F8486080F847708165018997
:10BACC00511A426811444160417B890709D5A1682C
:10BADC00D1F808138847A868416E11B1B0F8681006
:10BAEC00F1B190F8601049B1A168D1F80C138847F6
:10BAFC00A868C16C11B1B0F8501089B1A168D1F827
:10BB0C00B820137823B1926C12B19047A868A16841
:10BB1C00D1F8581288470020A8601CF07FFDF8BDB2
:10BB2C00A068D0F8541205F1080088470020A860DE
:10BB3C0010F05CFCF8BD00BFBE780020D879002066
:10BB4C0034250020B57A00209427002054B502003B
:10BB5C00B07A00200C0100202DE9F84FD0E90054F8
:10BB6C00994616468A46834613B10020C9F8000050
:10BB7C0076B11DF03BFE0746E87968B195F8E80010
:10BB8C0088B138461EF0EDF86FF00800BDE8F88F6C
:10BB9C006FF00900BDE8F88F38461EF0E2F86FF040
:10BBAC000E00BDE8F88F0020012105F58078C5E96D
:10BBBC003BA6C5F8F460C5F8FC0085F8E810E8630E
:10BBCC006873E872404600211EF032F820461DF0E2
:10BBDC00FDFE38461EF0C5F81DF069F808B9687905
:10BBEC00C0B395F84400C00606D52C6C24B1AB6CE0
:10BBFC00584610210022A0471DF0F8FD0446584677
:10BC0C0009F0ECF820461EF0ACF8687960B90A9996
:10BC1C0040461EF00DF808B10120687358460EF02E
:10BC2C0027FA002085F8E800B9F1000F1CBFD5F801
:10BC3C00FC00C9F80000E87A28B10020E8726FF027
:10BC4C000D00BDE8F88F687B002818BF6FF00C0062
:10BC5C00BDE8F88FDBE9005495F84400C00614D514
:10BC6C002F6CAB6C584610210022B8470DE0D5F86C
:10BC7C00FC0031460AEB0002204618F047FFD5F8CD
:10BC8C00FC10361A0144C5F8FC10002EEFD12046EA
:10BC9C001DF056FC0028FAD020461DF08BFE95F8BE
:10BCAC004400800605D52C6CAB6C58462021002234
:10BCBC00A0470020B9F1000F85F8E800C8D0D5F8EE
:10BCCC00FC00C9F800000020BDE8F88F2DE9FF4703
:10BCDC0015460F46814639B138461EF039F818B171
:10BCEC000446A5F1010A4EE04A48A0F124014A4855
:10BCFC000678701C01386DD001F1240491F82810DD
:10BD0C00FF292146F6D1002C64D0E81EC0B20128D0
:10BD1C000DD84248B0F80080B8F1000F07D00320CE
:10BD2C00042117F05BFFA6EB080181426FDDA5F142
:10BD3C00010A5FFA8AF001280DD83948B0F8008062
:10BD4C00B8F1000F07D00120022117F047FFA6EB36
:10BD5C00080181425BDD0120E8463946ADF80290CE
:10BD6C008DF8000008F104001DF031FC404605F090
:10BD7C007FFE0020A071BDF80C0060802948818CEA
:10BD8C0048461AF092F84AF6012100202571A4F8D1
:10BD9C000090A4F8091080212082E060E072E0712C
:10BDAC0084F82110204909780131490821725FFA81
:10BDBC008AF1042938BF01208000012960710BD859
:10BDCC001A48007858B11A4951F82000C0EB0010FD
:10BDDC00800006E0002409E06FF0010004E0144844
:10BDEC000068012184F82010A061E061002004218A
:10BDFC00002517F0F3FE08490978884224BF0D4846
:10BE0C00057008F0B1FD204604B0BDE8F0870024B1
:10BE1C00F9E700BF20450020E3BA0200BABA0200DD
:10BE2C00BCBA0200A86D0020CDBA0200D8270020B1
:10BE3C0090B40200972700202DE9FC4FD0F8C08069
:10BE4C00D0F8D0C0D0F8E820D8F80030C346E64689
:10BE5C009C4511D3D8F814B0BBF1000F00F08980C9
:10BE6C0090F8FC3005244FF0000E002B08BF012485
:10BE7C00DBF800308BF81040A3EB0E05A2F1080A9A
:10BE8C00B5F5806F28BF4FF48065D0F8D82032B15B
:10BE9C0001F1200301F12402C0F8DC5005E0C0F8E8
:10BEAC00D85001F1180301F11C020026BAF1000F61
:10BEBC00C8BF0126DBF8044012681F68CDF800E00B
:10BECC007CB1354B53F82630BB6005FA06F30126DE
:10BEDC00BAF1000FC8BF02260EFB06332344013B08
:10BEEC0005E02E4B53F82630BB6000F1F6033B60A7
:10BEFC0043F6F0740191D1F8009004EB051626403E
:10BF0C0009F1080EC7F804E0BC683443BC60002497
:10BF1C00BAF1000FC8BF0124DBF808709FB161466D
:10BF2C00DFF87CC05CF824308C46936005FA04F38F
:10BF3C000124BAF1000FC8BF0224009901FB04319F
:10BF4C0039444C1E05E0154951F8241000F1F40455
:10BF5C0091605460C2F800E0916831439160C34530
:10BF6C0004BF05EB0C01C0F8D01090F8FE10019A3C
:10BF7C0009B1BDE8FC8FD9F8241041F00301C9F8D0
:10BF8C002410D0F8CC00D2E90412406811430068A8
:10BF9C008162BDE8FC8F00BFA0B70200A8B7020009
:10BFAC00B0B70200F0B58BB0ADF80A00002001F17B
:10BFBC0008070C468DF8080038461CF079F808B3D1
:10BFCC0006AE0DF10701384632460DF0BBFB0546B7
:10BFDC004FF6FF7085421FD09DF8070000B39DF807
:10BFEC002800002844D0FF280AD0022848D0FD2879
:10BFFC0006D001284DD13F4800780138012844D99A
:10C00C003E4844E002A80DF029F8012802D102A80C
:10C01C0018F010FCA1205AE03848C4F8120055E082
:10C02C0006F10800394608221DF00AFA40F2FF100A
:10C03C00ADF828001DF0E8FD00F00F0000272946A0
:10C04C00142233468DF82A000420CDE906771AF025
:10C05C00F5FA2B4905EB450041F8207001EB800007
:10C06C002649C0E90177C4F812100121417210E091
:10C07C00052060829DF82B0000F07F00A08208E074
:10C08C001C480078411E022923D24FF08170C4F85D
:10C09C0012001B4A05EB4501002052F821305D1CB3
:10C0AC0042F82150A3610A232074B5FBF3F303EB90
:10C0BC008303A5EB430353B902EB81000121017209
:10C0CC0010484FF48061007812F01AF800200BB081
:10C0DC00F0BD30B90848C4F812009DF82A0084F865
:10C0EC00280004F11E0006F1080108221DF0A8F931
:10C0FC00CFE700BF2426002000000101000003014F
:10C10C00F03300209D7A0020F8B50D46417F04469F
:10C11C00827F1020002908BF082060700AB1083007
:10C12C006070217F09B101306070A17921B1217A51
:10C13C0000EB410002306070267E4749002E18BF8C
:10C14C000E26097802290BD142490978012907D119
:10C15C002178012904D04149097809B1012100E075
:10C16C00002184F83410217D314408442870217E4C
:10C17C0031B13B48007B1DF0B3F929780844287095
:10C18C00C0B274283DD81DF0B9FED0B30546344872
:10C19C002178677E237F94F806C094F818E0627FBC
:10C1AC00807C002B41EA800007F00301A77F40EA66
:10C1BC00811094F83410287018BF012340EA032032
:10C1CC0040EA4E2040EAC22040EA073040EA8C2088
:10C1DC0040EA4130000A6870A078A870E078E870F6
:10C1EC002079287160796871A07EA871E07EE87171
:10C1FC00607F40B1216A05F108001DF02AFE10276E
:10C20C0002E0002523E00827A07F20B1616AE8192D
:10C21C001DF01FFE0837A07970B1207AE855E81997
:10C22C000237617A4170E819227AE16852001DF0F8
:10C23C0007F9207A07EB4007207F08B1F9B2685460
:10C24C006078227D2169284430441DF0F9F8284695
:10C25C00F8BD00BFCA27002024260020DC270020C0
:10C26C00A86D00202DE9F04F85B007468A46581876
:10C27C00D7F80880D8F80410884202D96FF003056B
:10C28C007BE04E4D7C68DDF838904FF0FF319B46DB
:10C29C00164628681DF0CCFC6068B8F82010C5E97B
:10C2AC0001015FEAC97014D15FEA897023D5D8F80F
:10C2BC000C0000287AD0D8F81010002976D0012272
:10C2CC008DE80700384651465B46324613F0D2F8EB
:10C2DC000EE0A068C14300EA0B0211EA0B0F1CBF71
:10C2EC00D8F808100A4400EA0A01384606F0FEFDA8
:10C2FC0008B105463DE0D8F800005C46354603968B
:10C30C0000EB0A09ECB3384612F0E0FC78BB384677
:10C31C0019F07CFB58BB02208DF813908DF810009F
:10C32C004FEA19208DF812004FEA19408DF81100D0
:10C33C002248018938461CF036FF5FFA89F0C0F5B7
:10C34C008076B44238BF264604A8042113F094FC2E
:10C35C0068B92846314613F08FFC40B91748A41B26
:10C36C00B144018938461CF027FF3544CAE74FF029
:10C37C00FF35124800681DF0D3FD284605B0BDE816
:10C38C00F08F0E98400701D40025F2E7D8F80C0086
:10C39C0060B1D8F8101049B100228DE8070038467A
:10C3AC0051465B46039A13F065F8A2E70348006810
:10C3BC001DF0B6FD6FF00705DFE700BF0C24002071
:10C3CC002DE9F0418AB0514F05463878022804D146
:10C3DC004D480078002800F09480DFF8348198F8FC
:10C3EC002600082802D0042840F08B8007AC284691
:10C3FC0021461CF009F8387802280BD11CF076FD88
:10C40C00A11C1BF0A4FA28B1BDF81C601DF024FA85
:10C41C00864276D01DF084FC0234BDF81C00214607
:10C42C0008F050FE01286CD06E4630461DF037FCEB
:10C43C00304621461BF08BFA68B1BDF81C601DF02C
:10C44C00F9F9864207D0BDF81C00414621F81A0FB5
:10C45C004B2015F093FE3878012819D8AD8A1DF0C1
:10C46C00FBF9854214D020461DF072FC30B10079E6
:10C47C000138012802D8204612F068FD26480168D0
:10C48C0031B124480078012802D1BDF81C0088473E
:10C49C00BDF81C00002100261AF011FEB8F824107B
:10C4AC00BDF81C0019F001FDBDF81C008DF80C60E6
:10C4BC00ADF80E0003AD28460CF0D0FD70B1CDE9FF
:10C4CC0000662E1D684631461BF041FA30B13046ED
:10C4DC0021461DF07CF803A805F0CAFA281D214658
:10C4EC001DF075F828460FF0CDF850B1BDF81C00C2
:10C4FC00BDF80E10814204D0ADF80E0003A805F073
:10C50C00B7FA0AB0BDE8F081E52700202426002008
:10C51C00A86D0020CA270020982300202DE9F047A1
:10C52C00012816D1DFF830A1DAF83401012813D133
:10C53C000220CAF8340119F0C1FD0120012419F0C0
:10C54C00F5FA60B1CAF834411BF094FB4FF0FF349C
:10C55C007FE06FF001047CE06FF0040479E09AF85E
:10C56C005A419AF859119AF85801002C18BF012415
:10C57C00002918BF0234002818BF043401201DF014
:10C58C00DDF9013818BF01209AF83811B1FA81F1A0
:10C59C00490910EA010902D1002007F03DF9DAF847
:10C5AC0008002E4D10F0010807D12D4F286A816824
:10C5BC00384688470428F9D0064640461DF029FB2A
:10C5CC00B8F1000F08D1012E04D1286A012142686C
:10C5DC00234890471CF04CFF286841692046884747
:10C5EC009AF8540118B14FF480601DF0ADF99AF827
:10C5FC00530118B14FF481601DF0A6F919480121BF
:10C60C00016003200021CAF834011748016020465C
:10C61C0015F0FAFB0128FAD1144E3068042019F0F9
:10C62C0085FA044612480125B9F1000F05603068FF
:10C63C0002D1012007F0F0F81DF039FB082019F0A9
:10C64C0075FA0443CAF8345118BF4FF0FF341BF08D
:10C65C0011FB2046BDE8F087D81B0020B801001064
:10C66C0000400340282008600C2008402C20094082
:10C67C000C4009407CB54B4EB068016CD0F8D4200E
:10C68C00096892F8835019B9D0F84C058047B06806
:10C69C00D0F8B800007800B315F01AFE43494248B0
:10C6AC0009680068096C884705461DF09FF8044628
:10C6BC003F48017811B93F49097821B33E4902221C
:10C6CC000A700078832808BF12F084FF1DF064FB09
:10C6DC001DF06DFA0420884757E01DF087F80446DA
:10C6EC003348017811B933490978C9B30222324968
:10C6FC00012D0A7004D10078832808BF12F06AFF5C
:10C70C001DF04AFB41E01DF052FA00208847B0684A
:10C71C000DF10701D0F82824F42090479DF907006B
:10C72C00854223DB254D287800BB1DF035FB2548C1
:10C73C000078042803D0B068D0F84C0580471E4818
:10C74C00042101702878013028701DF030FA09B1ED
:10C75C00032088471C48032101801DF01DFC14E0B8
:10C76C001548832101701DF017FB0CE01248832142
:10C77C000170002017F022FE1DF00EFB1048F1682E
:10C78C0080780969087016F099FBF068C068007829
:10C79C0000B17CBDB0680021D0F85824002090472F
:10C7AC007CBD00BF0C010020E4260020347A002060
:10C7BC00B07A0020B37A0020B87A0020B527002088
:10C7CC002D260020BB7A0020C67900202DE9F84FD9
:10C7DC00494C1021207816F0EFFD28B92078102153
:10C7EC004FF47A721DF0EDFA44480178013901706A
:10C7FC0009065AD043484FF000084FF6FE79002640
:10C80C00041D41480578AE421DD22078C0B1FF28E6
:10C81C0016D001382070000612D16078032807D199
:10C82C0034F8041C34F8020C022211F031F8607850
:10C83C0001281EBFA4F8018024F8029C24F8049C53
:10C84C0008340136DFE73148DFF8C4A0314C4FF033
:10C85C000008002790F800B05F4519D007EB87005F
:10C86C000AEB4005287A0138287200060ED12046C2
:10C87C00294619F0A3F9064610B1304619F09CFE72
:10C88C00002EF4D185F80080A5F802900137E3E77B
:10C89C0021482249007830B10A780AB1013A0A706D
:10C8AC0008310138F7E7BDE8F88F154900220978FF
:10C8BC000170002005211AF001FB04460626002C0D
:10C8CC0098D020460521002225461AF0F7FA044696
:10C8DC0028890028F3D0013828810004EFD1688919
:10C8EC00400702D5287B18F029FF2868F0216E73C9
:10C8FC00407B15F037F8E2E79C7A00202F79002076
:10C90C00DCBA02004C500020D6BA0200D5BA0200A4
:10C91C00B25C0020AF1B0200D7BA0200503D0020D1
:10C92C002DE9F04F85B006464D48DFF83C91144692
:10C93C000D464FF6FE774FF6FE7800780190494889
:10C94C00007804900120029000200390474800F1E9
:10C95C00110B47480430009099F800C04FF0000EBE
:10C96C000020C00774D1049B5946C14603B331F86B
:10C97C00118CB84518BFB04502D11C31013BF5E70D
:10C98C00A84518BFA045F8D00A78501E0628F4D840
:10C99C00072A01D1C146F0E702980EF1010EC0073B
:10C9AC00EBD103985FFA8EF2C0B28242E5D351E02C
:10C9BC00BCF1010F2AD8DDE9001ABAF1000F25D01D
:10C9CC0031F8048CB84518BFB04503D12431AAF115
:10C9DC00010AF2E7A84518BFA045F7D04B79581EBD
:10C9EC000628F3D8087801380228EFD3072B01D199
:10C9FC00C146EBE702980EF1010EC007E6D1039891
:10CA0C005FFA8EF2C0B28242E0D323E0C8465FEAFE
:10CA1C000E6002D00398000603D00120B845A0D0C8
:10CA2C0018E000205FFA8EFADFF83C9002900120AB
:10CA3C00BAF1010F03903FF48FAF1DF0E5F8C0B2CF
:10CA4C00B0FBFAF101FB1A0003900020029083E77F
:10CA5C004FF6FE781FFA88F005B0BDE8F08F00BFE6
:10CA6C00E3BA0200D1BA020024260020305600207E
:10CA7C00204500202DE9F04395B0044600208DF8A8
:10CA8C001F00208817F052F9002840F081804B4895
:10CA9C00007810B14FF0B30908E0A078042803D156
:10CAAC001CF016FC002876D04FF0B60900261E208C
:10CABC001AF03EFC0546BEB303209DF852108DF8CB
:10CACC001E0010A808AF08303A4610F077FF0CAEE5
:10CADC000DF11E0008213A46334612F097FBA06870
:10CAEC00314610221BF0F6FBE0B11FFA88F702AEBC
:10CAFC000420002214233946009619F089FD9DF973
:10CB0C001B00B0F1FF3F03DC06F1130017F02EF809
:10CB1C000220394614228DF8180002AB042019F0BB
:10CB2C008DFD01E04FF0AD09B9F1000F17D09DF864
:10CB3C001F00012813D19DF953100020CDE91000DE
:10CB4C00002903D401208DF85100FF208DF85000EE
:10CB5C001FFA88F110AB0420142219F06FFDBDB13F
:10CB6C00092085F81D900822287020886880A078FC
:10CB7C002871681D61681CF063FCA16805F10D004B
:10CB8C0010221CF05DFC0E482946007812F0E6FAE3
:10CB9C0015B0BDE8F08360680DF11F0110AA0CF010
:10CBAC00D1FD80469DF81F0018B14FF000090126F9
:10CBBC007DE74FF0AD09002679E700BF2426002061
:10CBCC009D7A00202DE9F843DFF830810C46914620
:10CBDC0007462246B8F8241013F0A4FB002879D09D
:10CBEC00068905464FF6FE70864204BFC320BDE899
:10CBFC00F8831CF031FE864204BFC220BDE8F883E6
:10CC0C002988B8F8240088421CBFA8F824100846CC
:10CC1C0015F080FBE87A3946013088F8380008F1C5
:10CC2C0039001DF016F902208DF80100684619F044
:10CC3C0051FF002851D007460069062101260170DA
:10CC4C0098F80E104170BE771CF050F978624020B5
:10CC5C00BE7687F81890F88228897880384611F0CB
:10CC6C00C5FE002845D1092008F11A0188F82600D4
:10CC7C002889A8F81A0098F81800A04218BF88F85C
:10CC8C0018401F4C4B20A04708F124015020A0470E
:10CC9C0008F11801E120A04708F116015320A04724
:10CCAC0008200121FEF7E0FD4FF400500021FEF7B3
:10CCBC00DBFD144C4FF48061207812F08DFE13488C
:10CCCC00007802280BD110480078012807D14FF4C6
:10CCDC00DC6208E0CA20BDE8F883102009E00820D7
:10CCEC000EF0FCFF820020784FF480611DF06CF890
:10CCFC000020074900220A70BDE8F883A86D0020C7
:10CD0C00892102009C7A0020E5270020242600209F
:10CD1C00A27A0020F0B58DB00546007C0F2873D3A5
:10CD2C006E68686908AC0021224613F023F89DF860
:10CD3C002000002868D1287C0B2865D3307A022883
:10CD4C0062D1B189C8B2FF285ED19DF8220010F0E3
:10CD5C00FD0F59D1404F97F8263043F00402062AB4
:10CD6C0004D13E4A1268AAB1C90B1FE03B4A1268B3
:10CD7C0012B19579012DF4D0082B01D0042B43D19D
:10CD8C007589002A42D0917902293FD1284618F0A2
:10CD9C00E5FE39E0727C7189308800230093002312
:10CDAC00FBF758FEB089C10B9DF8220032888DF834
:10CDBC000D10B17B9DF824308DF810009DF8255096
:10CDCC009DF83200ADF8082072898DF80C109DF892
:10CDDC0021108DF80E308DF813508DF81400ADF82D
:10CDEC000A20727C9DF826608DF81110E11D8DF8DB
:10CDFC0012208DF80F6002AD082205F10D001CF019
:10CE0C001FFB28461DF072F80DB0F0BDB98CA9427D
:10CE1C00FAD1012806D0E11D07F139001AF097FD6F
:10CE2C000028F1D10E484FF40071007816F0C4FAC6
:10CE3C000028E9D140F20120ADF80D00B86A02904B
:10CE4C0097F82E008DF80C0002A812F003F90028B8
:10CE5C009CD01AF05FFED7E7A86D0020D8260020E2
:10CE6C009C7A0020F0B59DB04668077A10AD044658
:10CE7C00342128461CF04CFF8DF84070294636F8BA
:10CE8C00020B16F0E5F902201A9604F128018DF830
:10CE9C004100608EADF84E009DF8400002388DF8D0
:10CEAC005C0006A81CF0D9F99DF8420003287AD141
:10CEBC009DF843501CF0CAFC854274D19DF8440087
:10CECC00002870D19DF8450000286CD19DF84600D3
:10CEDC00002868D19DF85D00002864D19DF84700BA
:10CEEC00002860D19DF8480000285CD109A81C21BD
:10CEFC001CF00EFFBDF84E001A9A9DF85C30ADF890
:10CF0C002E00154615F8010B00F003018DF82400D6
:10CF1C00032916D100F00C060C2E05D0082E08D1D2
:10CF2C0001268DF8306004E0B2F80150ADF82850BD
:10CF3C00D51C35F8046BADF82A6035F8026CADF8E9
:10CF4C002C60521B0D951344524203298DF8383036
:10CF5C008DF8312027D100F00C01042923D010F0DA
:10CF6C00200120D140B200281DD4FE209DF8531082
:10CF7C00B4F8422000238DF827000C4840788DF837
:10CF8C00260094F846008DF81400B4F84700ADF86C
:10CF9C001500E06BCDE90013CDE9020309A806A941
:10CFAC0005AB08F0E7FD1DB0F0BD00BFCC2600209E
:10CFBC002DE9F047DFF83491D9F840A0BAF1000F11
:10CFCC0000F088800AF10C020820FF2151FA80F051
:10CFDC00C3B21B1A18BF012312686AB163B113885C
:10CFEC00A3F60303012B01D90432EFE7DAF81000A2
:10CFFC0092E8FA003830FAC0DAF808200025DAE9AD
:10D00C000A10CAE90A55B2B110F0E2440CD021F072
:10D01C000F0220F0E2434FF0000852EA030005D063
:10D02C001CF030FBB04701E0884604461CF02AFB9C
:10D03C0042462346B0471CF0D9FB0446B9F85600CB
:10D04C0001306FF31F30A9F856004FF6FD70AAF8A7
:10D05C00300009F140008AF833501AF001FC2046E8
:10D06C001CF07FFEB9F85600B9F85410884231D143
:10D07C001F48204940680D6830B190F8FC2007200B
:10D08C00002A08BF052000E005204C680FF01EFDAB
:10D09C0055B195F8FC00002100284FF0000008BFA6
:10D0AC00286885F8FC1000E0002044B194F8FC20BE
:10D0BC000021002502B9256884F8FC1000E0002549
:10D0CC00A84288BF0546681C04D02DB9BDE8F047BE
:10D0DC001BF01CB9BDE8F0871CF0E0FEB5FBF0F1CD
:10D0EC000548BDE8F0471BF06FBC00BF30210020A5
:10D0FC00D01E002070200020387100202DE9F04750
:10D10C004FF6FC76B04201D100240FE08846002196
:10D11C001D469246002414F0E5F9DFF810910746FD
:10D12C00680606D4B9F81600874202D12046BDE83D
:10D13C00F087384629460CF01BFF30B9B01C002193
:10D14C0080B20CF015FF00285ED0B11C078089B2AC
:10D15C00884505F0010118BFA0F8028045EA81015D
:10D16C00BAF1010F817140D101214171324915F0A1
:10D17C00180F99F8142018BF0A7802714046B9F8B4
:10D18C00241016F053FB0028BED12A482B49DFF897
:10D19C00B0C0274D0022007809788A42B4D0C2EB87
:10D1AC00C20400260CEB8404B0420BD005EBC6077E
:10D1BC0023887F889F4201D00136F5E70132F3B214
:10D1CC009842EAD120461C211CF0A2FDB9F824009B
:10D1DC00A4F8008060814AF60120A4F811001948D7
:10D1EC0000780130400820748EE7417901293FF422
:10D1FC008BAF114915F0180F08BF09F1130109780D
:10D20C0080F805A001717FE715F0180F0CD00949C3
:10D21C0007480978063039B110F8082B013912F09B
:10D22C00180FF8D10E3890E702247FE7A86D002084
:10D23C004C500020D6BA0200D9BA0200D1BA020072
:10D24C0030560020CDBA02002DE9F04186B01D46C3
:10D25C0014460E46022818D0012818D0002876D182
:10D26C00012E6BD0022E72D108201AF093FD3E488D
:10D27C000021437B3D48026840480088CDE90211FB
:10D28C0004913F49CDE9004555E0002000E0012024
:10D29C00032E00D0F6B91CF01BF8032E18BF002883
:10D2AC0035D102201AF076FD2F48304C417B206896
:10D2BC0010F0D6FD2E49897801F00801014345D1C3
:10D2CC002C48017801310170C8B2042849D12A4890
:10D2DC00206046E0711E80F0010018BF0121084358
:10D2EC0035D10A201AF056FD26484FF4806100789B
:10D2FC0012F072FB0DF11601502018F0FDFF2249BF
:10D30C00BDF81600888400211CF0E0FD29E01648C9
:10D31C0090F80D8015480768184806881CF074FCB6
:10D32C0001210022049030464346CDE90045CDE969
:10D33C00022113493A4605F0CBFA07E008201AF00F
:10D34C0029FD2046214600221CF022F848B10F4846
:10D35C0001214FF47A72007806B0BDE8F0411CF060
:10D36C0033BD06B0BDE8F081CC220020747A0020D9
:10D37C003E7900209927002000F8FF079027002015
:10D38C00C02600209C7A0020A86D00209D7A0020E9
:10D39C002DE9F04F8BB00C460690C9881F460792BA
:10D3AC00E07816F08FF900287ED0217D0546C0B2BA
:10D3BC0019F0E4FE002879D00646E188E07805975C
:10D3CC00DDE9177900224FF0000815F0F7FB8346D2
:10D3DC00E0787071E188A07D86F80880227DF1806C
:10D3EC007081F06821691CF02BF886F81490778214
:10D3FC004FF000090027BBF1000F4AD05FFA89F00B
:10D40C00854246D906EBC00A9BF80110504600F83D
:10D41C00168F012904D101270770BBF8020005E023
:10D42C00BBF802008AF81D001BF0AAF9AAF8180034
:10D43C0022789BF8041052068AF81A1005D59AF82F
:10D44C001C2042F002028AF81C20C7B9204AD28A5A
:10D45C00904214D11E48A170DDE90613CDF800806E
:10D46C00828C159801901698CDE90208204608F098
:10D47C0081FB9AF81C0040F005008AF81C0009F1A9
:10D48C000109E188E0785FFA89F215F097FB834691
:10D49C00B1E7304619F0E8F80599DDE91423204688
:10D4AC000096F9F71FFF10E0B92000E010208DF86E
:10D4BC002800E078A17D8DF82300E0888DF82410F9
:10D4CC00ADF8260008A81BF0B7FC0BB0BDE8F08F38
:10D4DC00A86D00207CB50568002D6DD0044647482A
:10D4EC00026842B1217928469047012803D1688906
:10D4FC0020F001006881687B02282DD168898007A3
:10D50C002ED52079CD282BD0F02829D0688A00067A
:10D51C000CD5A87E50B1A8732868008816F006FCBC
:10D52C0040B94FF498700DF062F803E0344800787D
:10D53C000130A8732079002856D00420202168736C
:10D54C00304800882881A87B0138A876A8732E481B
:10D55C00007810F0D5FD687B40F0040006282BD134
:10D56C002B49288BC98A884214D02849097889B15B
:10D57C0029680988ADF8000001208DF80500287B8A
:10D58C00ADF802108DF8040020798DF8060068467D
:10D59C001BF0E2FD6889C0070ED0217928461BF0EC
:10D5AC0016F9688920F0010068812868008816F057
:10D5BC00BDFB217908B121B17CBD39B140F23110EC
:10D5CC0001E040F22D100DF012F87CBD40F22F104E
:10D5DC000DF00DF8002560798542EDD24FF49B706B
:10D5EC000DF005F80135F6E7002660798642A4D2E5
:10D5FC004FF49B700CF0FBFF0136F6E7382400204B
:10D60C00C62700208C2700209C7A0020E9250020CA
:10D61C00A86D0020BFB54A4D044695F82600092890
:10D62C0000F28C80012101FA00F040F20A2108423C
:10D63C0000F084806178F1B141F2030019F0A9F98E
:10D64C004048007802280ED13F4801780B2904BFCE
:10D65C000A2101703D48002101703D484FF4804182
:10D66C00007812F0B9F96178A88C1CF02FFC00201E
:10D67C0085F8260060E00220002119F08AF934F8C0
:10D68C00020FE8825320214614F078FD95F826000D
:10D69C00092802D0A88C14F03DFE01200DF10F01D9
:10D6AC008DF80F00422014F069FD04200DF10704E1
:10D6BC0085F826004A20214618F01EFE05F11C00B4
:10D6CC0021461CF0C6FB204801780B2902D106210B
:10D6DC00017003E0A88C00211CF0F8FB194C207899
:10D6EC0002280AD2688B4FF6FE7188420ED00DF1DB
:10D6FC0007010022FEF7EAFA08E007D1E98A0320C5
:10D70C0019F047F9698B042019F043F9A87B0DF146
:10D71C000F01C0F3C0008DF80F00522014F02EFD45
:10D72C002078022808D1A87B00074CBF4FF400409A
:10D73C0001200121FEF798F81AF054FFBFBD00BF7D
:10D74C00A86D002024260020D0260020DC270020F5
:10D75C009C7A00202DE9F0418846080430D45FEA19
:10D76C00C86000F181805FEA887000F182805FEA16
:10D77C00087000F1818018F4706F00F082805FEA0D
:10D78C00085004D500201BF0B3FA88F400685FEA57
:10D79C00485004D501201BF0ABFA88F480685FEA8E
:10D7AC00885004D502201BF0A3FA88F400785FEAB5
:10D7BC00C85068D503201BF09BFA88F4807862E08F
:10D7CC00324F387811F06EF900284AD00546466879
:10D7DC000078411E05290DD91A282CD024282ED0CA
:10D7EC00D12833D0D32835D0FD2836D128461AF08D
:10D7FC006EFC32E0DFE801F0030B310F311B66B336
:10D80C00304611F0FBFB30461CF076FB25E0284639
:10D81C0014F090FE21E0F478701CE11CC9B21BF0EE
:10D82C0087F9611D56FA81F101F8010C15E02846C3
:10D83C001BF03AF811E02846FDF75AFF0DE0F0789E
:10D84C000530C1B230461BF0E3FF06E028461BF062
:10D85C00EBFF02E0284611F06DF828461AF046FC62
:10D86C00AFE788F400480EE01AF004F988F01008CD
:10D87C0009E088F0020806E00DF0D0FA88F00808FC
:10D88C0001E04FF000084046BDE8F0819A7A002094
:10D89C0070B50C4608041CD4E00729D14448007824
:10D8AC00012805D8A00745D4A00654D4600474D42C
:10D8BC00E0062DD4200744BF84F0080070BDE005BD
:10D8CC003DD460075FD400202146BDE8704009F0CC
:10D8DC00E3BB344E307811F0E5F830B1054607F073
:10D8EC00DBFA28461AF002FCF4E784F4004070BD21
:10D8FC0001201AF04FFA2C480F220F2381782B4865
:10D90C00008800F00700FFF79FFC84F0010070BD59
:10D91C002548007810F0B4FC28480078012806D17E
:10D92C0027484FF40061642200781CF04DFA84F013
:10D93C00100070BD0AF098FA84F0020070BD214806
:10D94C0090F82600082801D0042801D11BF032FBE6
:10D95C0084F4807070BD1748007860B91248007864
:10D96C00062802D107201AF015FA1348007801286E
:10D97C0008BF19F0D9FD0B481021007810F0C0FB3E
:10D98C0084F0200070BDFF20032116F07BF81CF002
:10D99C008AF90D4801210160FEE714F045FB84F47F
:10D9AC00804070BD9D7A0020D02600203E7900205A
:10D9BC0024260020BF7A0020CA270020CD27002073
:10D9CC009C7A0020A86D00207C0520432DE9F84F9F
:10D9DC004FF00054002A994616460F46804618BF51
:10D9EC004FF080444D1C1BF001FF824635B1404680
:10D9FC003946002214F090FA07460FE03C48816C3F
:10DA0C0011B10969414506D0C16C11B10969414593
:10DA1C0003D0876B02E0876C00E0C76C37B197F9D5
:10DA2C003300B0F1FF3F03DD04245BE0032459E035
:10DA3C00DFF8BCB00A9DDBF84800874218D0DBF851
:10DA4C004C00874229D0404639464A462B460BF0BB
:10DA5C0015FC0028E8D02748017E012941D0007E22
:10DA6C0004283ED02448254928301CF05DFA38E0C3
:10DA7C00DBF848000022234619F0CCF81BF046FFD7
:10DA8C001F48002E18BF00F580301AF063F8F5B16E
:10DA9C00DBF848001CF0AEF80CE01BF037FF184820
:10DAAC00002E00F100501CBF0120C2F202401AF0FF
:10DABC0051F865B1DBF84C001CF09CF838690E4944
:10DACC00086291F8240040F0010081F82400B9F1BB
:10DADC00000F06D0DBF83810404601222B460BF025
:10DAEC00CDFB832450461CF03CF92046BDE8F88F52
:10DAFC0030210020D01E00207020002002000040A9
:10DB0C0001000104F0B58DB0044603200D468DF8DC
:10DB1C0030000AAE30461CF09CF91BF0E7F90146C8
:10DB2C00304619F014FF50B1287D40F00201032952
:10DB3C0005D1297A09B1FF2914D1822000E0842073
:10DB4C008DF82700E289207C0DF127010123CDE916
:10DB5C00001004F11100A11C42F4004213F0E2FD8C
:10DB6C000DB0F0BD032804D1A87DFF28E5D0002816
:10DB7C00E3D0304F4FF0FF300822CDE9060006A964
:10DB8C003E1D30461AF0A6FB18BB2B486188C08A94
:10DB9C0081421ED03878FF280AD0297A814207D0DA
:10DBAC0078884FF6FF71884202D06989884210D17B
:10DBBC000020314608228DF8080002AF381D1BF0FA
:10DBCC003FFC38460DF05EFD6088BDF80A108142BE
:10DBDC002DD1E08905F10C0621281CD18C206989F6
:10DBEC00AB7D32468DF82700287A17F04FFB0028C2
:10DBFC00A8D11BF0F5FF287D0328A3D102A930463C
:10DC0C0017F074FB00289DD1304600210022002320
:10DC1C0010F066FB96E76989287AAB7D32461AF0DC
:10DC2C00BFFA08B188208BE71BF0DAFF8AE78D205A
:10DC3C0086E700BF0C260020A86D0020F0B589B047
:10DC4C000546002001F108060C468DF80F00304601
:10DC5C001AF02EFA18B9284631460DF02BF804ADFF
:10DC6C000DF10F0130462A460BF06CFD3B4E4FF682
:10DC7C00FF7731784A1E9DF80F10012A10D879B918
:10DC8C0000200DF10F01CDE90000684604AA0BF04D
:10DC9C0059FDB8421ABF01218DF80F109DF80F10D5
:10DCAC00B1B1B84214D09DF8201099B3FF2926D0F9
:10DCBC00022918BFFD2912D12A4900EB400001EBC3
:10DCCC008000A16950F8042F91420FD2A22042E0AB
:10DCDC00307810B91BF098FEC0B1A1203BE00129AF
:10DCEC0038D130780138012806D90FE001310160B4
:10DCFC003078411E02291ED24FF0817007E0307837
:10DD0C00013801289CBF012084F826001448C4F86F
:10DD1C0012001FE0052060829DF8230000F07F00B8
:10DD2C00A08212480078002818BF012084F8270030
:10DD3C0084F826000EE030B90B48C4F812009DF8A8
:10DD4C00220084F8280004F11E0005F108010822C5
:10DD5C001BF076FB002009B0F0BD00BF242600208C
:10DD6C0000000301F033002000000101A427002073
:10DD7C002DE9F047816A91F90120002A28D48246C6
:10DD8C0002F01F0000EB40049AF81C300234A3424E
:10DD9C001ED18B1CD2B24FF6FE784FF6FE7C08B12A
:10DDAC00B1F802C0DFF8F49000264FF6FE770021A0
:10DDBC00B9F81650814210D29C7814F0880F07D114
:10DDCC0033F8037BAF4208BF04F007060131F1E7DB
:10DDDC00D320BDE8F0470CF00ABC300606D11FFA80
:10DDEC008CF0B9B214F0EAFF002849D0BAF80C0054
:10DDFC001BF051FF80B10021027AC17128490978CA
:10DE0C008A4206D3013149080172F1B2072938BFA1
:10DE1C0001364672BDE8F08708F10101BAF80C0032
:10DE2C0089B217F0C9F820B105461D48297C007845
:10DE3C0015E015F0DDFC18B31C2105461BF068FF3E
:10DE4C004AF60120A5F81100BAF80C002880B9F8A0
:10DE5C002400688112480078411C490829748142C9
:10DE6C0006D3013040082874F0B2072838BF0136B9
:10DE7C0000206E742873023528461AF019F908B17F
:10DE8C00BDE8F0879AF808000028F9D0DAF81810E5
:10DE9C002846BDE8F0471BF0DCBF00BFA86D002092
:10DEAC00CDBA02002DE9F84F1D4600928B468146F3
:10DEBC001BF09CFC444A82464FF4A06000210127D1
:10DECC0005F1010C002392F86040602935D007FA67
:10DEDC0003FE1EEA040F0AD0BCF1000F18BF9D42CE
:10DEEC0005D1561896F80A80B8F1000F04D02031ED
:10DEFC0000F580700133E8E724EA0E040125737203
:10DF0C0082F8604092F86240B572013482F8624047
:10DF1C009EB142F801902D49BBF1020F86F808B072
:10DF2C00716011D0BBF1010F34D1591DB1740A21AC
:10DF3C0031820A99896871612CE0FE2450461BF0ED
:10DF4C0010FF60B2BDE8F88F718A5A1D0A9B02F06F
:10DF5C000F0221F4706141EA0221718221F0F80173
:10DF6C005A7902F01F0241EAC201718221F4C041C8
:10DF7C009A7902F0030241EA423140F203623282A2
:10DF8C0071824EF6FF721140DA7902F0010241EA19
:10DF9C00023171820B9A42B111785278920042EAA6
:10DFAC00411108430A49084300E000200099B06180
:10DFBC0001B171600748416809B9C0F804900FF0CD
:10DFCC0003FC747ABAE700BF206E0020236E0100B8
:10DFDC0001000406D01E00202DE9F04F8BB04A4FF3
:10DFEC00B868D0F80001807AC0001BF087FF0028C9
:10DFFC0009907DD000244FF6FF7B1BF0F7FB0090BF
:10E00C0001AD0DF114094FF0FF3AB868A2B2D0F887
:10E01C0000110B899A4263D24FF001080026C97A8D
:10E02C00F2B28A4222D2D0F88824D02029468DF828
:10E03C000660ADF80440904720B1B8680136D0F8BE
:10E04C000011ECE79DF810004FF000080128F4D106
:10E05C009DF80F000028F0D103200B2809D0295C73
:10E06C000130FF29F9D04FF00008E6E7B8F1000FB6
:10E07C0001D00134C9E70026B868F1B2D0F800210C
:10E08C00D2888A42F5D9D0F88824ADF80610D12070
:10E09C002946ADF80440904700BBBDF80800584530
:10E0AC001CD0ADF81400B8684946D0F88824D420A8
:10E0BC009047F8B9B8684946CDE907AAADF81AB047
:10E0CC00ADF818B0D0F89424D4209047B8682946FD
:10E0DC00ADF808B0D0F89424D12090470136CBE7A6
:10E0EC0000981BF03EFE09981BF006FF002008E08C
:10E0FC001A2006E000981BF034FE09981BF0FCFE79
:10E10C0019200BB0BDE8F08F0C0100207CB5044643
:10E11C008078022820D0012840F08C80267D0020B9
:10E12C008DF8060006F1180019F002F9054610B931
:10E13C0001208DF80600607940F00200022824D1FD
:10E14C00002D4CD0E078002818BF01201BF08CFA71
:10E15C0023D01BF06DFA25E000208DF807002C2051
:10E16C0019F0E6F8054610B901208DF80700607922
:10E17C0040F0020002280CD1002D54D0E0781BF0A6
:10E18C0073FA31D01BF054FA33E002208DF80600FC
:10E19C0025E002208DF8070045E0A01D042118F0B1
:10E1AC00E7FAA860A07C32462874E07C6874207D75
:10E1BC0015342146A87505F117001BF041F9A05D37
:10E1CC00A874A01941786975817829750521C078E2
:10E1DC0029802946E8741848007810F0BFFF0DF12B
:10E1EC0006037520012122E0A01D042118F0C0FABD
:10E1FC00A860A07C04F1150110222874E07C28751D
:10E20C00207D687505F11C001BF01AF904F125003E
:10E21C00042118F0ADFA0821A86107482980294685
:10E22C00007810F09BFF0DF10703752002210122ED
:10E23C0014F0A4FA00207CBDA87A00202DE9F04F40
:10E24C008BB04248DFF80CB100240DF11C0A4FF0E2
:10E25C0000084FF0000900270078019000EBC00087
:10E26C0086003B48007801304008029046455CD05F
:10E27C001FFA89F1032000221023CDF800A018F01A
:10E28C00C7F900284CD19DF821300BEB0801BDF8E3
:10E29C001C009DF820200C82CC60CC724B714AF68D
:10E2AC0001232BF80800BDF81E000A71A1F80930F3
:10E2BC00029B48800B72BDF82230CB800A9B5D1C00
:10E2CC0004D081F82040C1E9063315E0013A012A57
:10E2DC0009D8214A12784AB1204B53F82220C2EBBC
:10E2EC000212920004E06FF0010203E01B4A126874
:10E2FC0081F820408A61CA614FF6FF7188420FD0C5
:10E30C00ADF8180001208DF80C0003A811F02AFEBE
:10E31C0028B11348818CBDF81C0017F0C6FD0137DD
:10E32C0008F1240809F10109A0E7002004210024C8
:10E33C0015F054FC0199884224BF0A48047006F079
:10E34C0013FBF8B20BB0BDE8F08F00BFE3BA0200CC
:10E35C00CDBA020020450020D827002090B402003E
:10E36C00A86D0020972700202DE9F041414F04466D
:10E37C007878C8B1DFF80081B8F85400B8F85610B6
:10E38C0088421ED008F13801204619F07AFA80B97B
:10E39C00D8F8480010B10069A04207D008F140013C
:10E3AC00204619F06EFA03E0BDE8F081D8F8480079
:10E3BC0038B1B0F9301020460A224FF0E04307F094
:10E3CC0045FF1BF013FA2D4D0646284602C8A14204
:10E3DC0008BF284600210160787801387870000663
:10E3EC0036D17C60387E02280ED1082016F040FB16
:10E3FC0030461BF0B6FC04F150004FF0FF311BF01F
:10E40C0017FC1BF0F3F9064605F128001BF08AFDFA
:10E41C0040461BF04FFD1A481BF084FD08F11C0010
:10E42C001BF048FD17481BF037FD17481BF034FD57
:10E43C001648416811B107F15000884707F12800D0
:10E44C0019F028FC1248807810B10D2007F0A8FEB6
:10E45C007868A04204BF0020786030461BF081FC35
:10E46C0004F150001BF05AFD04F1B800BDE8F04176
:10E47C001BF012BDD01E0020302100207020002087
:10E48C00407200207C710020387100208026002012
:10E49C009CB902002DE9F0478EB080460E2016463E
:10E4AC008A468DF81A308DF818208DF81900012045
:10E4BC008DF81C003E48B8F1000F077B8DF81B70DF
:10E4CC0020D00AEB0605687B11F014FE034620F001
:10E4DC00010000243A280AD10DF104090020112171
:10E4EC004A4619F0A3FE002808BF09F10104287858
:10E4FC000994384305F8050B0DF12B0029461BF048
:10E50C00A8FC36E001AD002011213A2300242A4654
:10E51C0019F08CFE08B109942BE0DFF898906C1C74
:10E52C00012101220994D9F80430581CC9F80400BF
:10E53C000AEB06000090384612F031F81AF0D6FCBF
:10E54C0001460DF12B001BF084FCB9F800001A49B0
:10E55C0001300968A9F8000080B2814203D3D9F8D0
:10E56C000400012805D115484FF4007100780FF014
:10E57C00C7FD0DF12B000AEB06050422691C0830BF
:10E58C001AF05EFF1AF806008DF837005CB106A988
:10E59C000DF12B024046534606F05EF8297801F047
:10E5AC00F801297000E0A1200EB0BDE8F08700BF93
:10E5BC00A86D002014250020A8BA02009D7A002026
:10E5CC002DE9FE431BF012F9DFF80C91804699F807
:10E5DC000100B8B14148032201688260C80711D01C
:10E5EC003F4C2068416802208847019020684168B0
:10E5FC000120884702903B4801A91C3011F09AF881
:10E60C0017F09EFDD9F80450EDB13649686A01AF98
:10E61C0001F11C06A96A884219D23046394612F01B
:10E62C00D5F9013011D0D5E90912E869541A08441A
:10E63C003946082C28BF082422461BF085FC686A42
:10E64C0020446862E6E700240CE0D5E909010024C7
:10E65C00884207D309F10400294618F0FFF985F820
:10E66C003240012499F8010088B9D9F8040018B196
:10E67C0080681AF069FB0AE01A481C301BF025F878
:10E68C0028B9194A4FF0FF30012110F067FA4046C3
:10E69C001BF067FBF4B1A86800220168CA628A69A2
:10E6AC000AB10223137091F83030012B07D0022BE2
:10E6BC0010D101F134001BF033FCBDE8FE8322B114
:10E6CC00CB6800219847BDE8FE830C69CA698B6A48
:10E6DC000021A047BDE8FE831823002008800240DB
:10E6EC00CC0100107422002080A9030070B586B004
:10E6FC00454D0446A868D0F8F41091F84420B2F1C6
:10E70C00820318BF531C81F84430D0F8F40090F801
:10E71C00441000EBD10090F82C104A0880F82C2003
:10E72C00C807A86809D1D0F8F41091F94420531CFB
:10E73C0012F1020F81F84430E7DCD0F8F4201146D6
:10E74C0011F8443F802B25D8D0F83024E120904795
:10E75C00AA6802208DF814004FF0FF30D2F8F43084
:10E76C00ADF80C009878022823D0012824D030BBB7
:10E77C001BF094FB4FF47A71244B0022B1FBF0F0A8
:10E78C0023490BF0B5FBE0B3A8681A21D0F8F400CC
:10E79C00417004E0907810B91C4814F04FF82A200E
:10E7AC002070A868D0F84013204606B0BDE8704031
:10E7BC000847D2F86814F7E70820802101E0072009
:10E7CC008321D2F8786303F149020023CDE90032AA
:10E7DC0003AA4FF6FF73B047A0F1DB01182910D83C
:10E7EC00012202FA01F10B4A11420AD0A968D1F8B0
:10E7FC00F41048702A202070A868D0F840132046E6
:10E80C00884706B070BD00BF0C0100205C7A002068
:10E81C003D2D0100112400012DE9F04389B004467F
:10E82C004648807860B9E07AFE2809D168462421F0
:10E83C001BF06EFA208B10F00D0F06D0B62400E002
:10E84C000124204609B0BDE8F083207A0028F5D0D9
:10E85C0001288DF8080011D002281CD003281ED0E6
:10E86C000F2820D102204FF000080B264FF0000992
:10E87C008DF808002088ADF8000019E0B4F800808D
:10E88C004FF6FF700F26ADF8000002204FEA182952
:10E89C008DF808000CE02088ADF8000003E0684615
:10E8AC0021461BF0D6FA4FF0000803264FF0000962
:10E8BC0006F00C0707200C2F08BF0920A17C084488
:10E8CC008DF81F00C0B21BF019FBA0B305460C2F2E
:10E8DC000890867011BFE81C85F8049085F80380B9
:10E8EC00681DA17B0170E17B4170217C8170617C92
:10E8FC00C1700430628A61691AF0A2FD1AF0A6FF99
:10E90C0081098000033069702870B7FA87F04009DC
:10E91C00ADF80E0003208DF80C00A07E8DF80D00D4
:10E92C00A089ADF80A0068461BF078FA0446284620
:10E93C001BF0E2FA85E7102483E700BFCC26002009
:10E94C002DE9F04F85B0054691460E46C80731D1EA
:10E95C002846314612F0C6FD404FF98A884242D013
:10E96C002846022132460CF0C1FBE0B328464FF694
:10E97C00FE7102223346FEF7C1FB90BB4FEA15280D
:10E98C0006F0DF0A70061ED402A9284617F0BEF95D
:10E99C0068B9B98C284616F00FFBA0B1871C384615
:10E9AC0019F086FB78B102A839461BF052FA46F0F2
:10E9BC00200A08E0B0074FF0FF084CBF46F0100AE1
:10E9CC0046F0080AFC25264800220778791C0170BD
:10E9DC002248012100913946C08A034608F0EAFF1B
:10E9EC0018B1C72037E0002035E01AF020044FF0B2
:10E9FC000E0008BF06208DF8110004A818F06AF864
:10EA0C0040B34FF0010B064680F81EB01AF06EFAB8
:10EA1C0070623069002141710AF078018770C5700D
:10EA2C0080F8048080F800B041701CB1063002A957
:10EA3C001BF00FFA6FF00300B9F1000F708005D0D6
:10EA4C0008480078484588BF86F81A9030460FF081
:10EA5C00CDFF00E0102005B0BDE8F08FA86D0020C0
:10EA6C00C07A0020CBBA02002DE9F04788B0444DA3
:10EA7C000A4604461046A98C14F0D8FE40B14178E1
:10EA8C0031B9072141703F490978013149080170BA
:10EA9C00A06A477817F08F0F18D1F9064FF01002C3
:10EAAC0058BF0822BB0648BF0832237F93420DD1C2
:10EABC0090F8029090F80780B0F805A0B0F80360C9
:10EACC00002909D407F0700708200DE0D32008B006
:10EADC00BDE8F0470BF08BBD00F1080106A81BF058
:10EAEC00B8F907F060071020B90606D5A16A0144F1
:10EAFC0004A81BF0AEF907F05007B6B249463046F1
:10EB0C0015F0EAFF2049097888421ED21F4900EB14
:10EB1C00800001EB400010F8061F41452CD980F80D
:10EB2C000080E88A864213D0A1891FFA8AF4012258
:10EB3C003B462046FEF7E2FAF0B904A806A9029774
:10EB4C00CDE900103046214612E0E88A864207D112
:10EB5C00A1891FFA8AF001223B46FEF7CFFA0BE09F
:10EB6C0004A806A90297CDE900101FFA8AF13046D5
:10EB7C0042464B4603F0C4F908B0BDE8F08700BF2D
:10EB8C00A86D0020CDBA0200D5BA0200B25C0020FC
:10EB9C002DE9FE4F8A4683461AF0ACFDDFF808914A
:10EBAC00DFF8FC803F4E99F8001098F80200B07323
:10EBBC0039B1000713D501200DF10A018DF80A00B7
:10EBCC000AE0002000240EF06FFBB07B000706D596
:10EBDC008DF80B400DF10B01522013F0CFFA0EF013
:10EBEC0083FF19F02DFF38B105460EF0F3FC13F03E
:10EBFC0005FE0CF051FF08E008F028FF0546307EBA
:10EC0C00012101FA00F0294908604FF6FE74012D2C
:10EC1C002FD10FF0D5FA1AF0F7FF074624482349F5
:10EC2C0000680860FF20022114F02CFF601C748324
:10EC3C00F482B084002013F0A3F807F07F0058444E
:10EC4C0000F164061B480078012808D10020BAF1B5
:10EC5C00010F1CBFCDE90000684615F0B3FA114A4C
:10EC6C00212074211AF02AFF0020022114F00AFF3F
:10EC7C0000E0002628460CF09BFE601C80B2834509
:10EC8C0007D0012089F8000017F0D8FFB0B219F0B6
:10EC9C00CBFE98F8020019F0D7FA2846BDE8FE8F93
:10ECAC003E790020A86D0020D0260020747A002028
:10ECBC0078270020242600202DE9F0438FB014F093
:10ECCC0003FB3F4F97F82600082806D00120C7E920
:10ECDC000C003C480078F87078710DF11408242170
:10ECEC0040461BF015F839480F25374EDFF8E090F9
:10ECFC000DF13B018DF83B5000783570013818BF91
:10ED0C0001208DF81E004620C847324800248DF89B
:10ED1C00004000788DF801001AF098FD8DF8020083
:10ED2C0097F838008DF80640ADF8034007F139012B
:10ED3C000F2838BF05468DF805506D46E81D1BF0B1
:10ED4C0088F84FF0FF303278234EADF80F008DF875
:10ED5C00110097F8720031468DF81200284610F019
:10ED6C0014FD45203146C84705F0FEFDB88D97F8D7
:10ED7C002F108DF820408DF834408DF82940ADF8D7
:10ED8C001C00387E8DF81F1007F116018DF81A0043
:10ED9C00B88CADF818005320C84707F11A014B2066
:10EDAC00C847F879642100FB01F20C48082100786F
:10EDBC001BF00AF8404606F03DFA0FB0BDE8F083B0
:10EDCC00A86D0020E3BA0200B927002024260020F9
:10EDDC0089210200E8270020207900209C7A00205D
:10EDEC002DE9F0410546880058BFBDE8F0810020B0
:10EDFC00002410F0DFF93D493D483E4FCC610860DE
:10EE0C0040F60A008846B887FC8797F8480000F05F
:10EE1C00F00087F848003C6497F8490000F0F000D7
:10EE2C00013087F84900284607F00AFEAC6801203B
:10EE3C0021460E46496849B10A88A2F60302072A00
:10EE4C00F7D800FA02F212F0830FF2D0707B00F0C8
:10EE5C00F000707307F13C0070602748806B28B19C
:10EE6C00C0680088A0F6030002281AD3284630F8A0
:10EE7C00381FB1B10021E9636987386495F8440003
:10EE8C0095F8451000F0F00085F8440001F0F00012
:10EE9C00013085F8450097F8490000F0F00087F83C
:10EEAC0049001AF04BF81548F86197F8250030B175
:10EEBC0017F09CFE0028FBD012F0CCFA0BE00120DE
:10EECC001AF03CFD012806D0707B00F0F0000130F8
:10EEDC0070730B48F86100202146C8F81C00C8F874
:10EEEC0000400120BDE8F04118F004BF00100440C0
:10EEFC0001010E04D01E00203021002095370000A7
:10EF0C008D0902002DE9F84F0746087A0C4640F0AF
:10EF1C000201032917D10025B7B1FF2F14D09A464F
:10EF2C0016460AB903280ED00FF00AFA204610F044
:10EF3C00C8FF8146207A4FF6FE71B0F1010B18BF65
:10EF4C00B346894503D100252846BDE8F88F013822
:10EF5C00DDF82880314EB0FA80F044092E48017853
:10EF6C000020814230D03278BA4208D17278A24265
:10EF7C0005D17288914502D13279934502D00E3673
:10EF8C000130EEE706B32649C7B23546B1F800901A
:10EF9C00BAF1000FD8D0B8F800402846214619F035
:10EFAC00BFFA60B92846214618F03CFB30B102206C
:10EFBC0039464A46334617F041FB00E0002508F17C
:10EFCC000208AAF1010AE3E70DF1030017F0ECF9CE
:10EFDC0005460028B8D0134885F804B0A5F802906F
:10EFEC006C702F7041460078504538BF8246A81D82
:10EFFC004FEA4A0285F805A01AF022FA9DF8031090
:10F00C00064AC1EBC10002EB40030548028802200E
:10F01C0017F014FB98E700BFDFBA0200307900202C
:10F02C004EB20200CFBA02002DE9F84380460068C8
:10F03C003B4BD8E9012118603A4802603A4820223B
:10F04C001AF082FFD8F80C003849DFF8E89090E805
:10F05C00FC00FCC1D8F80C00354990E8FC00FCC160
:10F06C00D8F81000494690E8FC00FCC1324D402213
:10F07C0099F80C00D8F8141040F0800089F80C00B6
:10F08C0028461AF061FFE87BD8F81810202240F0CF
:10F09C00A500E873294D28461AF056FF40F20540AA
:10F0AC00697BAA7CEB7DC5F8049028820320287527
:10F0BC00287B40F08000287301F0F00020490230DA
:10F0CC00687302F0E0000A460130A87403F0F00007
:10F0DC000130E875D8F81C0090E8F800F8C2087BFD
:10F0EC00CB7B4A7B40F08000087303F070008430C7
:10F0FC00C87302F0F000013048734FF45860086197
:10F10C00D8F820000F4908600F48C06840690078A3
:10F11C0008B111F005FBBDE8F84315F097BE00BF30
:10F12C00687A00206C7A0020D87500209077002037
:10F13C00A8770020C077002000720020B87500204E
:10F14C0048780020647A00200C0100202DE9F0435F
:10F15C0087B0DFF8FC8081462025EFF3118085F322
:10F16C001188D8F830501DB180F3118800256AE061
:10F17C00C8F83090374F80F311880020C9F80C1074
:10F18C004FF48031C9F81C20002BC9E91200C9E9E1
:10F19C00080118BF1F46D7E90116C9F81810397BAA
:10F1AC00012905D1C9E91060C9F8146030460DE099
:10F1BC00294A002031460023002519F041FFC9E9F6
:10F1CC0010012649C9F814008E423CD80021DFF802
:10F1DC0090E0C9E9160197F800C0C9F85410BCF1C9
:10F1EC00020F08BF0146BCF1000FC9F8501001AB6B
:10F1FC009EE8F5001946F5C108F11C001A4ACDF835
:10F20C0008900090174808BF024609F12800142105
:10F21C0018F0CEFA05462020EFF3118180F3118807
:10F22C0081F3118899F8100010B9484612F04EFC81
:10F23C0035B108F12800494619F036FA4D4602E07E
:10F24C000025C8F83050284607B0BDE8F08300BF51
:10F25C00A01F00200CB7020040420F003F420F00DD
:10F26C00E8B70200ED3802008D950200F8B50446AF
:10F27C000020A5782075C4E9030045F0020000F0D9
:10F28C00030002280CD115F00C0005F0030218BF86
:10F29C00042809D1022A05D1E90601D402210FE084
:10F2AC00012619E0022106E00C2803D00828F1D031
:10F2BC00012100E00321022A02D1EA060E460BD4FA
:10F2CC0048B10E1D0C2807D8012202FA00F041F2B9
:10F2DC001012104200D04E1D68B2B0F1FF3F0ADC94
:10F2EC00E078800706D0A8074FF0030058BF022033
:10F2FC00064400E0013627881AF0AEFA87420BD09C
:10F30C00A80609D51F48416920468847206918B9C5
:10F31C00A07800F0DF00A070207D00B1F8BD61790D
:10F32C005020751C8DF8000020798DF80210216991
:10F33C0028448DF8010029B10A7F497F1044084404
:10F34C008DF80100684613F037FEA0B1012180F85A
:10F35C004850417621884180618801872179226952
:10F36C0080F8421001692944416412B1127F1144A2
:10F37C004164E060F8BD20461AF0E7FB10202075D0
:10F38C00F8BD00BF502400202DE9FC47434FDFF8A7
:10F39C0010810DF1070A4FF0000918F0FBFB002853
:10F3AC0000F079805046012114F030FD38780528A2
:10F3BC00F3D8DFE800F003090F1928469DF8070081
:10F3CC00FE28EAD1032462E0B8689DF807100224F5
:10F3DC0041705CE0B8689DF807100424817078785F
:10F3EC00002808BF052452E09DF8070088F800901B
:10F3FC007870033017F09CFF0028B86049D07978FA
:10F40C000124017043E098F80000411C88F80010BA
:10F41C00B96808449DF80710C17018F0BBFB05468D
:10F42C0098F8000079780A1AB9680844E9B20330F0
:10F43C008A421ADA91B214F0E9FC787888F8000064
:10F44C001FE07878BD689DF807400330C6B22846A7
:10F45C00314619F06DFBA04215D17B68B3B1304633
:10F46C00294600220024984711E014F0CFFC98F8AC
:10F47C0000007978284488F80000C0B288427FF4F4
:10F48C008CAF052403E0284618F030FE00243C70B5
:10F49C0083E700203870BDE8FC8700BFF42500200E
:10F4AC00967A0020F8B504464048C16819B1204648
:10F4BC00BDE8F84008473E4E3068074658B105464F
:10F4CC0060882988814203D12079A978814216D09D
:10F4DC00A8692F46F2E71C201AF010FD002863D013
:10F4EC001C2105461AF014FCFF20E8724FF6FE7042
:10F4FC0028813068002818BF07F11806356020797C
:10F50C00217A627A237BA87060880129AA716971BB
:10F51C002B75288005F10C0007BF4FF0FF31C0E9B7
:10F52C00001104F10D011AF094FC2249A07A09781B
:10F53C00884239D96179012903D01AF06BFA98B352
:10F54C00A07AA97A884202D9E27A102A05D3884295
:10F55C0006D1E97AE27A8A4202D20022012101E044
:10F56C0001220021144B1B78022B01D2A31D01E0B8
:10F57C0005D1E31D1B7813B172B9228808E00F4A3C
:10F58C00538B2288D31AB3FA83F35B09194203D045
:10F59C00A872E07A2A81E872E07908B1012028711A
:10F5AC00A07908B10120E870F8BD00BF54750020A7
:10F5BC00E8790020A327002024260020A86D002035
:10F5CC001EF0040F14BFEFF3098169468869A1F19D
:10F5DC00480214BF82F30988954621ED100BF1EE19
:10F5EC00102A41F8082DEFF3118102B400B5DFF8B1
:10F5FC00D8E0F047374A1268116801EA0000106041
:10F60C005DF804EB1EF0080F09D101BC80F31188E2
:10F61C005DF8080BE1EE100ABDEC100B704704BC52
:10F62C001EF0040F14BFEFF309816946A1F120010C
:10F63C0014BF81F309888D464A604FF08070C86111
:10F64C0025488861234B1B681868086040F201103C
:10F65C001860704702B401B4EFF3148100291CBF89
:10F66C00002282F3148802B402B4DFF860E0F047A1
:10F67C0001BC01BC00281CBF022181F3148801BC11
:10F68C00DFF84CE0F0470F484FF08051016001BCAF
:10F69C0080F3118800BF00BFFFF7FEBF1EF0040F00
:10F6AC0014BFEFF30981694601F1200151F8080BF1
:10F6BC00E1EE100AB1EC100B14BF81F309888D46F2
:10F6CC00704700BF04ED00E0CDCD01006B9E020041
:10F6DC00719E0200B4BA020060F600002DE9FF41F1
:10F6EC003B4E96F8420100286AD1012086F842016F
:10F6FC001AF030F9374F86F87001374D7868C6F834
:10F70C006C01387B86F84101A86810F4402F13D1A6
:10F71C00386988B128686421C0F3066000FB01F4E5
:10F72C001AF0BCFBB4FBF0F22C4906F19400002358
:10F73C0015F06CFE19F094FE01AC20461AF00FFA8D
:10F74C002749A846002506F10C00002219F05BFFA2
:10F75C0020461AF004FA234906F15000082219F049
:10F76C0052FF214A06F1D8003221002313F0F8FC95
:10F77C001E4C1F4A06F1F4002C210023256045463F
:10F78C0013F0EEFCD8F80800797BC0F3815021B15E
:10F79C00032804BF012186F83911032803D040F057
:10F7AC000200022810D1206840F0400020600220A6
:10F7BC0015F07CFF6868400702D4002015F076FF36
:10F7CC00002004B0BDE8F08114F0E4FBF2E700BFC8
:10F7DC00D81B002018B80200AC4F005063970200F1
:10F7EC00ABDD01000929020061CD01009022084027
:10F7FC0091A700002DE9F8431D46434BDDF820800E
:10F80C0043F606061C68038814F0007411D0B3424A
:10F81C0027D0B3F5C15F33D040F60206B3423ED1D8
:10F82C0000F112030B604169116081692960C169A3
:10F83C002EE0B3420AD0B3F5C15F03D040F6020606
:10F84C00B34203D100F11203143002E000F11A03A9
:10F85C001C300B600068106000202860C8F80000A5
:10F86C004BE000F11A034FF000090B60C169116005
:10F87C00016A2960416AC8F8001000F118011CE007
:10F88C0000F112030B6041691160416A2960816AC1
:10F89C00C8F8001000F1100190F80F900DE000F185
:10F8AC001A030B60C1691160816A2960C16AC8F8CA
:10F8BC00001000F1180190F82490286868B10E88A7
:10F8CC0019F0C4FE042808D8074606F0070148467C
:10F8DC000EF0A4FF296841F82700D8F8000060B1A9
:10F8EC0019F0B4FE042808D805464846FF210EF04E
:10F8FC0095FFD8F8001041F82500002C18BF012402
:10F90C002046BDE8F88300BF941200502DE9FE4F4D
:10F91C00D0E90085994614460F46834613B1002062
:10F92C00C9F8000074B119F061FF064698F8070099
:10F93C0058B198F8E80070B130461AF012FA6FF02E
:10F94C0008046CE06FF0090469E030461AF009FA1B
:10F95C006FF00E0463E000200121C8E93B74C8F885
:10F96C00F440C8F8FC0088F8E810C8F83C0088F8A7
:10F97C000D0088F80B00284601951AF027F8304640
:10F98C001AF0EFF908F1D0060DF1080A19F02EFF64
:10F99C0004463046514616F043FAD8F8F450D8F8DD
:10F9AC00FC10A842394438BF054602982A461AF082
:10F9BC00CBFA3046294614F041FBD8F8F400D8F8BD
:10F9CC00FC10401BC8F8F4004819C8F8FC0020468D
:10F9DC001AF0C7F9012D03DBD8F8F4000028D5D1B3
:10F9EC0019F004FF0746D8F8FC0050B1019819F043
:10F9FC00EDFF584605F0F2F9D8F8FC0010B10024E0
:10FA0C0002E000206FF00F04B9F1000F18BFC9F825
:10FA1C000000002088F8E80038461AF0A2F92046C9
:10FA2C00BDE8FE8F2DE9F041047B06468846204652
:10FA3C0019F08AF8054610B168892C4625E07289C0
:10FA4C003068214617F074FB002700286AD0044662
:10FA5C00078116F8100F207470886082304619F0F8
:10FA6C00F3FB6061308961892083B07AA07621F440
:10FA7C0060704907608105D42C490978013140EA4E
:10FA8C00C11001E040F080006081C0F3C211B8F1F8
:10FA9C00000F12D0022262732268D289520702D55B
:10FAAC00234A128A228169B36FF07F0220F46070BE
:10FABC0002EBC1110843608124E039B1810607D4FF
:10FACC00C1060BD440070FD4012013E000271AE025
:10FADC001AF09AF800F07F005F300BE01AF094F8FF
:10FAEC0000F00F000A3005E0124806881AF08CF876
:10FAFC0030400230208110480421617320210078AD
:10FB0C000EF0FEFA01276DB92289617B20460CF0BC
:10FB1C00DDFC38B1606908B11AF0EEF920461AF034
:10FB2C00EBF900273846BDE8F08100BFD52700204F
:10FB3C00A86D0020B8BA02009C7A00207CB504465F
:10FB4C00007A022803D3208814F0F0F810B10226B2
:10FB5C0030467CBD207A032806D10DF102012046E7
:10FB6C0015F0C4FB18B9F2E72088ADF80200608AE2
:10FB7C0044301AF0C3F9002864D0442105461AF029
:10FB8C00C7F8A07A694617F0AFFE9DF800009DF803
:10FB9C00011085F83A0085F839102846012117F034
:10FBAC00F9FE05F110002146242219F049FC628A65
:10FBBC00616905F144002864AA8719F041FCBDF87D
:10FBCC000200A88020480178E971013101701AF017
:10FBDC0067F906461AF062F970434FF47A71002601
:10FBEC00B0FBF1F0FF218DF80460288095F8390006
:10FBFC0001FA00F0217E85F8370085F83600207A6E
:10FC0C008DF8060001F001008DF8050001A819F02F
:10FC1C002BFA298D023885F83400C0B241F0080166
:10FC2C0083B22985A98F8AB2B2FBF3F202FB1010C2
:10FC3C000004064818BF013201212A7200780EF028
:10FC4C005FFA85E7102683E7987A00204826002083
:10FC5C002DE9F04F85B0044600880DF1060117F030
:10FC6C0051F8054618201AF049F94FF6FE7768B19D
:10FC7C00182106461AF04CF860881821324619F003
:10FC8C001DFF781C608030461AF036F90020278062
:10FC9C00002D207160D1DFF8C8A0BDF80640DAF85D
:10FCAC000000D0B314201AF029F9B0B3834604AB8A
:10FCBC004C2000210222002719F058FA009404EB82
:10FCCC00440402AE0BEB44004FEA4408851C122F8F
:10FCDC0018D0B84505D1DAF8000000EB44012846ED
:10FCEC000BE007F102094C20062233461FFA89F17A
:10FCFC0019F03CFA09EB0B003146062219F0A0FB77
:10FD0C000637E4E74C2014215A4619F0D7FE584622
:10FD1C001AF0F2F8009C4FF6FE7704AB4C20002151
:10FD2C00022219F023FAB8B9DAF8000050B104EB4A
:10FD3C00440130F81100B84204D1BDF8100030B1C4
:10FD4C00013802E0BDF810000130ADF8100004AA33
:10FD5C004C20022119F0B2FE05B0BDE8F08F00BFB7
:10FD6C00EC2600202DE9F04788B0DFF8FCA0D0F895
:10FD7C0004803E4E7F2400217F23DAF8280020EAFD
:10FD8C000800CAF828001B2915D020FA01F2D20766
:10FD9C000FD00027324612682AB19578A94208BFC5
:10FDAC0001371832F7E7DAB2FDB295423CBFCCB25C
:10FDBC003B460131E7E7B8F1000F15D0CAF82880AF
:10FDCC0001AC1821201D19F0A3FF0120CDF80480EF
:10FDDC008DF808009AF82E008DF8090020460EF0D8
:10FDEC00EBFE08B0BDE8F087204EDFF884804FF6BC
:10FDFC00FF7930460768BFB13888BAF824108842BA
:10FE0C000FD1B978A1420CD1B8F8001049451DD1D9
:10FE1C001AF05AF8AAF82400398881423046E9D100
:10FE2C0002E007F11800E5E78AF81840FEF744FFF6
:10FE3C000028D6D000208AF826000E480168002938
:10FE4C00CFD0C42008B0BDE8F047084700208AF89E
:10FE5C0026000848016809B1C4208847002008B072
:10FE6C00BDE8F04716F08ABAA86D0020E8790020AA
:10FE7C0090270020102500202DE9F04389B03F4A3F
:10FE8C001278824209D93C4A3D4F002952F8306021
:10FE9C0018BF0F4696F8521021B10025284609B01C
:10FEAC00BDE8F08302EBC009D9F804406078022861
:10FEBC0026D1022086F8520011F0EAFF0DF10C0851
:10FECC00404619F0C5FA3868002541468DF81450A3
:10FEDC0006958DF80C500490207812F0EFFC002859
:10FEEC007060DBD019F082FFF87988B1B879396885
:10FEFC0048436421B0FBF1F1706819F074FF07E01E
:10FF0C0000F0EEFC012086F85200207886F85400B0
:10FF1C006D46284619F023FE002000212A46CDF814
:10FF2C0008908DF800000190164813F0DDF8B060D1
:10FF3C0070B138683060B97986F85310F8790228B6
:10FF4C000CD0012812D0A0B9484613F016F810E0D6
:10FF5C0070680028A1D019F043FF9EE7B8884FF6CF
:10FF6C00FF72410848460BF02DFF02E0484613F0A3
:10FF7C006DFE4D4692E700BFF4B80200C3B8020014
:10FF8C001CBA0200092C0200F0B58BB0364D286863
:10FF9C0070B9364C206828B935488068D0F84C05C3
:10FFAC0080472068334C016A204688473248E0611C
:10FFBC0032480068016931B12D488068D0F8D4000E
:10FFCC0090F8530088472A4EB068D0F8D40090F9C6
:10FFDC00420010F02FF9411C03D0294940EAE0708F
:10FFEC004882274C002060606080207B617B40F061
:04FFFC0080002073EE
:020000021000EC
:1000000001F0F00001306073B068D0F8C40380479D
:1000100030B91F4810210170F06814214068017048
:100020002868D8B10020002614F0CEF9124F3868A5
:10003000416E03A8884717480696806808B1804734
:1000400009903968286800230D6D0821CDE9001654
:1000500003AA2146A8471048046009E00F480B4A4C
:10006000074B01680448006804680D48A0472860F1
:100070000BB0F0BDE4260020347A00200C010020F3
:10008000F875002054F10080607A0020D8750020B7
:10009000B47A002054B5020030250020687A002090
:1000A000B06500202DE9F0418AB03E4E054630682B
:1000B00020B13D490978A94209D82DE013F038FF55
:1000C0003068002448B338490978A94225D94FF04F
:1000D000FF3119F0B3FD354905EB450001EB800414
:1000E00067683878A8B9A568A9682A6848424B1E8D
:1000F0001A42B8600DD16A688A420AD3104082421F
:1001000007D1686910B10068786029E0298B04295B
:1001100007D3306819F00AFF002420460AB0BDE872
:10012000F08106EB81000069A8B90DF10408404692
:1001300019F02EFC002041468DF810008DF80400C7
:10014000E8690590287E12F03FFC0028E1D0298B59
:1001500006EB81021061786031440A7B01320A7338
:10016000298CC6E90101204617F0C4F80120387037
:10017000AB2031898DF82700204619F01AF80DF1CF
:10018000270001210FF07EFD31890546204619F038
:1001900019F815B920460EF09FFD306819F0C6FE1B
:1001A000BBE700BF0C2400208DB9020028B7020075
:1001B0002DE9F84F3C4C3D4E3D4D42F62A294FF07B
:1001C000010A4FF0030B00274FF00508D4F83C015B
:1001D000062833D8DFE800F00433183B203D4B00FD
:1001E0000F20F060C6F8109013F00AF945F804AC3F
:1001F00055F8040C8007FBD5C6F81CA094F839010B
:1002000090B10120EF6210E02F60C4F83CB1286883
:100210008007FCD40320DBE72F60C4F83C8128680A
:100220008007FCD40520D3E70320C6F800B0C4F84B
:100230003C012F6029688907FCD4C9E7FEE7012645
:10024000022084F83A6112F07FFB2E6009E0022060
:1002500000E0032084F83A01002012F075FB012031
:10026000286004F15000BDE8F84F19F027BE0020C7
:1002700045F8040C286055F8040C8007FBD4286866
:100280008007FCD40B480025012105600A48016065
:100290000D2005F08BFF022014F0D6FBC4F83C5172
:1002A00084F83B51BDE8F88FD81B002000400C407B
:1002B00058600C403C500C4004800C4070B5C16844
:1002C0000C6991F8381041F00203224603F0030351
:1002D00002F8011B022B3BD111F00C0301F00305C6
:1002E00018BF042B2DD1022D01D1CE0630D4C26807
:1002F00092F83B2062700234022D01D1CA0626D446
:10030000C26892F83E202270C26892F83F20627064
:10031000C26892F84020A270C26892F84120E27050
:100320004BB1221D0C2B13D8012505FA03F341F222
:1003300010152B420CD0C26892F83A202271621D2F
:1003400006E00C2B32D0082BCDD01446D4E7224641
:10035000C46801F0020394F8395005F003051D4309
:1003600009D1658D2D0606D4154E357884F849508F
:100370006C1C347001E094F8495049B21570B1F129
:10038000FF3F00DD70BDC16891F839105170C16840
:1003900091F83940A407F5D091F84B10002B9170DB
:1003A000F0D0C06890F84C00D07070BDC26892F870
:1003B0003C206270C26892F83D20A27003349BE733
:1003C000987A00202DE9FE4FDFF8F4B001219BF868
:1003D0000C4001AA204619F00EF96A462046022177
:1003E00019F009F9DFF8DC909BF80EE09BF80D009E
:1003F000BDF800C099F800100EF101030746B3FBE9
:10040000F1F404FB11359DF80240ADB2FEB2B542E5
:100410000FD0A642634618BF1023720052FA87F22B
:100420000BEB82029383721CB2FBF1F303FB1127E7
:10043000ECE7DFF894A0002401270DF1080857FA33
:100440008EF2C9B2C5B2B2FBF1F303FB1121A9428E
:1004500032D0690051FA80F00BEB800232F81C0FA9
:10046000102806D1284607F013FA8AF80000013454
:1004700017E028460421022313F03EFD8AF800000D
:10048000284600214246042318F0A8FF9DF80800E2
:100490007C2802D0FE2804D10DE02846782114F0F3
:1004A00051FA99F80010681C9BF80EE0B0FBF1F2CD
:1004B00002FB1100C3E7FEE7E0B2BDE8FE8F00BF1C
:1004C000B87200209B7A0020A02300202DE9FE4F67
:1004D00005460F465818AE687168884202D96FF019
:1004E000030564E0DFF8E8800C9C4FF0FF3199468B
:1004F0009246D8F8000019F0A1FBE00711D1A0073F
:100500001ED5306851464A463844CAB110F8013BFE
:1005100011F8014B013A23409C42F6D06FF00605DA
:1005200041E0D8E90101CB4301EA090213EA090FCE
:1005300018BF02443940284609F060FE054690BBCA
:10054000306802970196074412F07EFBCB46554671
:100550000090BBF1000F16D0BBF1080F5E4628BF1C
:10056000082619F049F9804628463946324617F0E0
:100570007FFE0446404619F0FAFB2CB93744354457
:10058000ABEB060BE5E70024009817F005F9DFF860
:100590004080DDE901210C9814B14FF0FF3502E0F5
:1005A000400707D40025D8F8000019F0BFFC284602
:1005B000BDE8FE8F10680844B9F1000FF2D010F8C2
:1005C000011B1AF8012BA9F101098A42F4D0E4E7D2
:1005D000DC250020B0B50C46880722D4600758BF40
:1005E000B0BD354D0120A870042015F065F83348E2
:1005F0000068006B8047E8602D48806BF0B1696847
:10060000046961B1A1420AD094F82800400704D5DA
:10061000636A2046042100229847012060766C60BE
:100620000DE0FCF7CBFC2248006CE0B3214844F01D
:1006300002012830BDE8B04019F07CBC6C686068ED
:100640001F4900780860022015F036F8102005F0E8
:1006500047FB012028761B48807810B90D2005F053
:100660003FFB6868416818488A680AB9C96821B1BF
:1006700000218160154940F8141C154907220A60C1
:10068000016800210160426841601249124AE96133
:100690000168114301601A2019F016FC1920BDE809
:1006A000B04019F011BCBDE8B0400DF093B800BFE8
:1006B0003021002070200020D01E00208C0100106E
:1006C000D02108409CB902001410044051000706D4
:1006D00000000460EDED0000024000402DE9F84FFD
:1006E0003A48DFF8EC90DFF8ECB0DFF8EC80002659
:1006F0004FF0060A00210078C700B74242D009EB4C
:100700000605A878E0B30138A870687918F022FAD5
:10071000A8B30446A87800B3A87948B3287970B381
:10072000E9780139E970090629D19BF801100138EF
:100730002871E970617B032921D100061BD00420B8
:10074000607319F067FA00F00F002021013020815A
:1007500098F800000DF0DAFC11E0607B84F80DA041
:1007600002280CD02068F021407B11F001F906E04E
:10077000607B032803D12846214610F095FE012115
:100780000836BAE798F8000001290BD1402112F091
:1007900019FEC0B998F8000040216422BDE8F84F66
:1007A00019F015BB40210FF01DF90C480178012903
:1007B00009D1002101700A48007806F023FCBDE849
:1007C000F84F12F059BEBDE8F88F00BFCEBA020054
:1007D000AA680020A86D00209C7A0020EA2700204B
:1007E000EB27002070B58AB04FF48061041D458866
:1007F000ADF826108189807B0894ADF82450032839
:10080000ADF81C1034D0022806D0B0BB40F6010071
:100810000026ADF826005AE03248007801285FD162
:100820000DF11B0101AA204608F092FF04469DF835
:100830001B00012854D19DF81400022850D101ADAD
:100840001421284619F06AFA274904EB44000022D3
:100850002B4641F8202001EB800021464260427285
:10086000FF2014228DF81400042015F0EDFE37E06F
:10087000102000268DF8270029E00DF11B0101AAA8
:10088000204608F065FF01469DF81B0001281DD198
:100890009DF81400022819D1134A002301EB4100EE
:1008A000CDE9013342F8203002EB8000142243608E
:1008B000FF208DF814009DF81600013000F00F00A5
:1008C0008DF8160001AB042015F0BEFE012607A826
:1008D00001F05AFD26B118B92846214602F04EF91A
:1008E0000AB070BDCB270020F03300202DE9F0477F
:1008F000A4B018F081FF34490A78012A04D124B049
:10090000BDE8F04719F033BA4FF0010981F80090C3
:1009100019F02DFAFEF7E8FE082005F0E1F921AC08
:10092000204618F003FDDFF8A4A02A4A1021234630
:10093000DAF80C002290264812F018FC2648002510
:1009400001AF0478254890F800804646A64213D8A7
:10095000DAF8000050F8261021F0FF0047F82600D2
:10096000880707D4F0B201F0010118F0CFFC09FAB2
:1009700006F005430136E9E7194805601948C168E2
:1009800001F44001B1F5800F09D10068000E18BFD5
:10099000012057F8201041F0070147F820101248B5
:1009A000A4EB0802042307EB880103EB820240EA70
:1009B000880019F0CFFA0D482022016862F30D215A
:1009C000016024B0BDE8F087A6270020E4B802004B
:1009D00078760020491D020017B802000BB702000C
:1009E000D0200240A84F00500010084000300940BD
:1009F000FEB5D0E9005401A818F078FC95F8340051
:100A00003649374A384E085C95F83510515C354AFE
:100A1000084395F83610515C2A6B40EA01033168AF
:100A200020684F680299B847206840F2F272E16985
:100A30002E4B2F4F426494F854209A5C94F8553012
:100A4000FB5C1A430129426311D10146D4E90A2310
:100A500051F8307FFF2A27F4004718BF07F50047F9
:100A6000FF2B0F6009D00A6842F4804208E001467B
:100A700051F8302F22F400420A600A6822F48042C2
:100A80000A60C16A41F01001C162016B41F00101CD
:100A90000163E16B09B3A16BF9B1012118F0EAF828
:100AA000D5F85801E16B40680068C162C0F80415D0
:100AB00091FAA1F17268B1FA81F153680222984764
:100AC0007068A16B02224368D5F8580191FAA1F130
:100AD000B1FA81F1406800689847FEBDA4BA0200EF
:100AE000C2BA020083BA0200D00100108DBA02001F
:100AF00088BA02002DE9F8430546007F04282FD16B
:100B0000A86A4678B0F802900E2E38D80C46012715
:100B1000DFE806F008080841414141414141412ACE
:100B20002A38410031480078012833D83048807B8A
:100B300080072FD51FFA89F80021404609F01EFAD8
:100B400000283FD0817911F0180F3BD0AA89438843
:100B5000698900880027009200220FF08FF91AE0BF
:100B6000D32009F04AFD29E020480078012811D857
:100B70001F48807B80070DD519F0E6F90AE00127B0
:100B8000002408E019480078012803D81848807B21
:100B900080071DD4012768891FFA89F2314619F0B0
:100BA000A5F9688913F0C8F840B1A87C022805D3DC
:100BB00027B10F48A989C08A814200D1002420466C
:100BC000BDE8F88340460121012716F04BFBE2E720
:100BD0001FFA89F8404618F099F940460DF0A6FC36
:100BE000B0F1C50718BF0127D5E700BF24260020B4
:100BF000A86D00202DE9F04186B018F041FF0446B1
:100C0000002718F03DFF10B180690137FBE7DFF8DE
:100C1000C88098F80000012831D818F031FF2F4E15
:100C2000B18C28B102888A4229D080690028F8D185
:100C30001C2019F069F910B30546B08C2880307E6D
:100C4000A87018F009FE6871254806F1390100788E
:100C5000A87105F10C0019F002F90DF117014120FE
:100C600015F050FB1F489DF81710AC612C4600880A
:100C7000002908BF6FF001000137288100E000253E
:100C80001948FBB200210278934201D200260BE002
:100C9000B81A0026F7B2974202D2A4690136F9E7E2
:100CA000C6B2052E28BF05261048CDE902411049DD
:100CB000CDE900260022007803F072FC98F80000CD
:100CC00008B1012803D115B1284619F01BF916F017
:100CD00027FF06B0BDE8F08124260020A86D002083
:100CE000E827002088790020C77A0020C67A0020F3
:100CF0009C7900202DE9FE4F4FF4804018F056FB00
:100D0000A0B1354C35496068D1F8132009786FF3EC
:100D10009F5201F00401806842EA417101AA03F088
:100D20001DF960688168012016F0EAFF2E482C4FFB
:100D30002C4D44F2020B00244FF0000A00F1400950
:100D4000BAF1020F3CD055F82A80D8F80000A0B3C1
:100D5000D8F80000806918F029FB0646D8F8000092
:100D60000023324615F05CFF16F00A0F1ED0D8F8AB
:100D700000008069B9686BEA00000840B860D8F8E4
:100D80000000C069396821EA000038601020D8F8F6
:100D9000001016F0B5FFD8F80010484616F03EFADD
:100DA000002044F00204C8F8000006E02EB1D8F894
:100DB00000000D4944F4804408650AF1010ABFE7C8
:100DC00024B10A482146283019F0B4F806F0BEFFD5
:100DD000BDE8FE4FF7F768BCD01E00208503002158
:100DE0000C10044004BA02003021002070200020C2
:100DF0002DE9FC473A4D0446286810B194B1BDE88E
:100E0000FC87122019F080F800282860F7D04FF6F0
:100E1000FE720021531C1229F0D0461842520631AE
:100E20007380F8E701AB4C200021022218F0A4F9EE
:100E300000284CD1BDF80400002848D0032846D82B
:100E4000182019F061F8DFF89C90044600264FF650
:100E5000FE784FF0020A0027032F34D028680622BC
:100E6000831907EB47000AEB400081B24C2018F0D1
:100E700083F928BB2868815B414518BF002C1FD02F
:100E800030440022182341880620009415F0C6FB48
:100E90002868D4E90423304402F2E932418822610F
:100EA00001EB410049F8202009EB80001822436043
:100EB0000620234615F0C8FB2046182118F02EFF07
:100EC00006360137C8E714B1204619F01BF8064B67
:100ED00071200021082218F04FF9BDE8FC8700BFFF
:100EE000EC26002030750020B8260020F8B5044616
:100EF00018F004FA07464568204617F0B7FFB8B166
:100F0000D7E9014618F078FC0546D4F8C000B8B11E
:100F100004210174384606F005FAD4F8C800B0B1CF
:100F2000014640690028FBD1D4F8C000486112E0B6
:100F300018F062FC0446D5F8C00078B3103034E0F5
:100F40003068416821F002014160284630E0D4F861
:100F5000C000C4F8C800416900274761C4E934777C
:100F6000C4E93677C4F8C01031B320463146FAF7E9
:100F700069FFD4F8C000C4F8E0700068B0F5806F75
:100F800003D920463146FAF75DFF94F8FE0010BB06
:100F90003068416841F0020141601CE095F8FB00B7
:100FA000002114F051FA05F1FC00012101702046E6
:100FB000BDE8F84018F0DBBE94F8FB000021C4F84F
:100FC000C47014F041FA012084F8FC003068416AD2
:100FD00021F003014162284618F0C9FE04F13000F7
:100FE000BDE8F84018F0A8BFF8B53948394D0121DF
:100FF000394E0768E868C0680170002002F00201FD
:10100000F07003F0E040401817D096F90600012870
:1010100002DBB0790138B07196F90500012802DBD6
:101020007079013870712D48426803F0807082B188
:10103000D8B10020002190470CE01446500223D480
:10104000E00326D4A00330D50020387111F002F956
:101050002BE050B196F90700012802DBF079013846
:10106000F0710120307118F04BF8002038710BF04E
:10107000C3F97079F8B196F90500002823DCA86857
:10108000D0F84C0580471EE0002038710BF0B4F911
:101090000BE01348007820B1052018F013F813F086
:1010A0003FFE00203871F1F72DFEA00648BF18F072
:1010B00087FF707938B900200021B070A868D0F897
:1010C000582400209047E8680021C0680170F8BDEE
:1010D000787A00200C0100202425002054B502005D
:1010E000A0270020B0B58CB004464089ADF80000C0
:1010F00060684178821C019206298DF8021003D0A5
:10110000042907D0012936D1817C13228DF80310E0
:101110001B2101E01A211222851801440391029536
:1011200031D0284616F0CAFF01282CD117F0E4FE72
:101130000146284616F011FC28BB264800780128F5
:1011400024D8684618F00CFD01281FD102980DF133
:10115000160114F0D1F8012818D10021BDF81600AD
:1011600061721D496081097891B16168097805292A
:101170000ED101210DE00021029100F11201807ECB
:1011800003918DF81000684610F056FD0CB0B0BD0C
:10119000002100222173CDE90622ADF81800207A43
:1011A00008928DF81D108DF81C0001208DF81A0092
:1011B00006A8FEF761F89DF82C000028E6D10998F2
:1011C000227A6168406C18F041F906A811F01CFA07
:1011D000DCE700BF24260020E02700202DE9F041B5
:1011E0000E46054610463421144618F097FD082E89
:1011F0004ED326702146288812F030F88046688841
:1012000008216081A888A081A879A074E87961701C
:10121000E074E07920B1102105F10800617060618F
:10122000207A28B101F1080029446070A16100E032
:1012300008460021616284F82010617919B1295CA7
:10124000013060706171617FF1B1421C6270295C94
:101250000230607084F82010AA5C914284F821204A
:1012600010D9194A4F00194E1278914288BF182799
:10127000291830463A4618F0E9F860786662384432
:10128000607001E0002161772178C2B2914203D2FF
:1012900000263046BDE8F081B8FA88F2091A55FAFE
:1012A00080F05609A2792177A062002AF1D00E3091
:1012B000A062A1F10E0020770548007B18F016F916
:1012C000217F081A2077E4E7D8BA020008780020C6
:1012D000A86D00202DE9F04105460026806A1C46D5
:1012E000174688461680007817F0FCFA40B16889E6
:1012F00012F022FD022811BF002668893880264698
:10130000A86A007801380A2846D8DFE800F0060C01
:101310001116242C45383C4A5200284641463A468C
:10132000F7F75AFE41E028464146FDF7A3FB3DE0B2
:1013300028463146FFF7DEFB37E0287F02282BD115
:1013400026B920486989C08A814228D13046294679
:1013500000F068FD29E0688912F0EEFCE0B928464B
:10136000F4F7C8FD22E017486989C08A814213D189
:10137000287F022810D128460CF008FE16E02846E7
:10138000FCF7FCFC12E00F486989C08A814203D156
:1013900028460BF027FA09E0D32009F02EF90026A1
:1013A00004E0304629460FF05FFF06463046BDE8B0
:1013B000F081054800780128F1D128460CF0B6FDEF
:1013C000F4E700BFA86D0020CA27002070B586B0E2
:1013D0003449002808705DD1344C207830B9324946
:1013E000097819B9082016F0DBFC207801284ED8BE
:1013F0000020CDE90300CDE9010017F06FFF0028C0
:1014000045D02B4D05F13904204617F0A1FE18B93F
:101410002849204618F023FD05F11601532010F04D
:10142000B3FEA87B0DF11701C0F3C0008DF81700C3
:10143000522010F0A9FE082085F8260003F09AFA41
:1014400004F036FA1C48016809B9012101601B4803
:101450004FF4407100780CF059FE01AC204614F0B6
:101460007BFA20460021002616F02EF895F8410060
:1014700010B9002005F0C6FD1148CDE90366CDE99D
:101480000166807B012802D0012014F07DFF01203D
:1014900015F08EFC0948022100780CF037FE06B0EA
:1014A00070BD00BFBF7A0020D02600202426002077
:1014B000A86D0020B6790020182500209D7A002014
:1014C000CC2200202DE9F84F8A468DF8030062B146
:1014D000384851460123406802700DF1030048F27C
:1014E00031020DF0F9FF044660E00B9F1624052041
:1014F0001E4617FB0400C0B218F006FD002854D0A9
:10150000814604220C980A9917FB04280024CB4634
:101510000BF8014F00F119058BF801600BF104067F
:101520008BF803708BF80210E0B2B84229D2A5F113
:101530001701304618F093FC06F10800A5F10F01E1
:1015400018F08DFC15F8071C861D0134017015F884
:10155000061C417015F8051C817015F8042C41EA31
:101560008201817015F8032C41EA0211817015F88F
:10157000021CC17015F8011C017129781A354171DE
:10158000D2E70C4D5FFA88F30DF10300514648F2A3
:101590003102C5F804B00DF09FFF0446484618F02C
:1015A000B1FC05480130686000E010242046BDE829
:1015B000F88F00BF88260020447000202DE9F041FC
:1015C000056804464FF0FF30E86218F015F98046D0
:1015D00095F83000042809D13249497831B13249AF
:1015E00003228A604A6822F003024A602D4F6B6929
:1015F0002E4E00217A68B34204D01AB979780029B6
:1016000018BF01210023042804D11AB17B78002BD4
:1016100018BF012341EA0300012808BF14F096FD1A
:1016200095F8320030B1404618F0A1FB4FF0FF3082
:10163000BDE8F08195F83000042804D1381D294612
:1016400015F0FEFD03E0381D294615F0E7FD0120E9
:1016500085F83200404618F08AFBFCF7B7FF246893
:1016600094F83000012811D0022812D00428DDD1CE
:101670000D4DD4E90901884210D2012018F080FBF9
:1016800028688007F9D0FCF7A1FFF2E70020BDE849
:10169000F081216A04F1340018F0D0FAE06ABDE864
:1016A000F08100BF182300200880024080A90300B9
:1016B0002DE9F04F85B0044610F000FD00286ED0F3
:1016C00026468346471C00244FF000084FF00009CF
:1016D0009BF80000844222D2384618F03FFBD8B174
:1016E00001790139012917D890F82000A0B10C2008
:1016F00018F00AFC80B13946054618F0B0FB00200E
:1017000009F10109A860B8F1000F28461CBFCAF80A
:1017100008504046AA46804608370134D8E75FEAB9
:10172000096039D002205FFA89F937468DF8100038
:101730007088ADF808004FEAC90018F0E5FBC0B1A9
:1017400005460024B8F1000F17D0E0B2414605EB82
:10175000C00018F084FBD8F80860404618F0D2FBAF
:101760000134B046EEE7D8F80840404618F0CAFB0E
:10177000A046B8F1000FF6D10EE0002048F21F019C
:101780004A462B46CDE9001007F1110002A902F0EC
:10179000AFFC284618F0B6FB584618F0B3FB05B06E
:1017A000BDE8F08FF8B53B4E0446B068D0F8B810ED
:1017B000097859B194F8982004F190014AB11522A2
:1017C00017F0B8FB58BF25229A5C09E0012121756A
:1017D00014E0252217F0AEFB58BF25229A5C023296
:1017E00084F86A20002284F86920042284F86B209F
:1017F00004F1700228C928C209881180254615F80D
:101800002C1FB5F872200F2925F8162CB5F8742076
:1018100025F8112C0CD0D0F80473B4F8A800294690
:101820000023B0FA80F042092046B84700B1F8BD65
:10183000214611F83C0FFF2801D1A06D30B1B068EE
:10184000D0F8FC22204690470028F0D1B06805F17E
:101850006402B4F89A3094F89C10D0F874530020C5
:1018600000902046A8470028E1D1B0682189D0F82F
:101870000021D289914205D9E5206070B06800F559
:101880001B7001E000F51E700168204688470020AB
:10189000F8BD00BF0C0100202DE9F04385B00646DD
:1018A00000200D46049017F0A7FF334CDFF8C490DA
:1018B00080462168D9F80000CB6C04AA052198471E
:1018C00001A817F001FF2D48019626F001060395A7
:1018D00020F00107BE420AD12B490878FE281BD010
:1018E0002068826BD9F8000091F900100EE02448BE
:1018F00020F0010086421BD123494878FE280BD0F6
:101900002068826BD9F8000091F901109047812876
:1019100002D01C4818F0EDF92168D9F80000002227
:10192000CB6A01A998470546B0F1FF3F07DC03E009
:10193000144818F0DEF9FE25124818F0DAF9BE4214
:1019400001D1114806E00E4820F00100864202D184
:101950000D4801300570012021680490D9F800007D
:10196000CB6C04AA05219847404618F000FA05B050
:10197000BDE8F083E4260020347A0020BD64020034
:10198000F14D02000C010020242500202DE9FC4728
:1019900006680446707A00286BD0D4F80490D6F814
:1019A0005801D0F80480D9F8347020460BF016FBAB
:1019B000706F20B306F14C05284618F0B3FA316F6A
:1019C000884221D2307902281ED0B06E002850D033
:1019D00020460BF003FB346F284618F0A3FA201AB8
:1019E000D6F868A0B46F7067284618F09BFA0021FB
:1019F000F1740AEB040108440190706F0CE0B06EC2
:101A000010B1306F0028D5D106F14C0001A914F0B7
:101A10000DFA01217067F17458B30021B0F5806FA1
:101A2000B17384BF4FF48060706701230199014452
:101A3000013979601049B96043F6F07101EB00108B
:101A40000840B9680843B860D9F83C10D9F80000DC
:101A500091FAA1F2B2FA82F203FA02F2D8F8003057
:101A60009A61D6F85821526812689162012117F0E4
:101A70000DF9BDE8FC8700BF0180000C2DE9F0479F
:101A800088B004466FF00100A081002004F1040832
:101A90008DF8100004AD4146281D17F09EFD284624
:101AA00009F0F6FD012809D1BDF81C00BDF812109F
:101AB000A0816088814222D004AD01E060880025C9
:101AC000EA46ADF8020000264FF6FE7950468DF842
:101AD000006007F0C9FA0128074608BF5646B5B1AD
:101AE000A88901210125A081204610F0C7F8012F07
:101AF00006D1ADF802903046022110F0BFF8012562
:101B0000204611F0D9FA284608B0BDE8F087012F29
:101B100013D1BDF80C00A0810AF1040016F0CEFA32
:101B2000012817D1204609F007F905463046022161
:101B3000ADF8029010F0A2F8E2E76088484504D1C1
:101B4000404616F0BBFA01280CD1204609F0F4F803
:101B50000546D5E7404616F0B1FA0128CFD1204618
:101B60000321CAE70025CBE72DE9F0438FB080467B
:101B7000374800240394CDE90144077814F0FAFEB5
:101B80004FFA80F901ADBC4212D2E6B207200C2216
:101B90002B4631460EF048F940B9B9F1FF3F05DC5C
:101BA000072031460C222B4614F04EFD0134EAE7A3
:101BB0004FF0FF300C22CDE90200781E01AB85B258
:101BC000072029460EF030F940B9B9F1FF3F05DC96
:101BD00001AB072029460C2214F036FD04AD182174
:101BE000284618F09BF8822018212A4617F066FF35
:101BF000B8F1010F08BF002804D104AA82201821DF
